S011000000486578766965772056312E3036D3
S224018000F0FF0220F52C02007B1A02003F1D0200C73F02009B43020097450200000000006B
S22401802000000000000000000000000017120200BB2A020000000000171202002961020071
S2240180401712020017120200171202001712020017120200171202001712020017120200C2
S22401806017120200171202000D640200415B020017120200171202001712020017120200E7
S224018080171202001712020017120200171202001712020017120200171202001712020082
S2240180A0171202001712020017120200171202001712020017120200171202001712020062
S2240180C0171202001712020017120200171202001712020017120200171202001712020042
S2240180E0171202001712020000000000000000000000000017120200B5EB0100B5EB0100B7
S224018100B5EB0100B5EB01002DED01002DED01002DED01002DED0100171202001712020055
S2240181201712020017120200171202001712020017120200171202001712020017120200E1
S224018140171202001712020017120200171202001712020017120200000000000000000017
S2240181600000000000000000000000000000000000000000000000001712020011160200A5
S2240181801712020017120200171202001712020000000000A15D02004D6102001712020052
S2240181A0171202001712020017120200171202001712020017120200171202001712020061
S2240181C0171202001712020017120200171202001712020017120200171202001712020041
S2240181E01712020017120200171202001712020017120200255702001712020017120200CE
S22401820017120200000000000000000017120200171202001712020017120200E166020038
S22401822017120200155B020017120200171202001712020017120200171202001712020099
S2240182401712020017120200171202001712020017120200171202001712020017120200C0
S224018260F8B500BFF8BC08BC9E467047ED4D0200F8B500BFF8BC08BC9E467047C94D0200A6
S224018280843D00201C00000000000000BC340020D000000000000000113F0020010000008A
S2240182A000000000A43F00200800000000000000AC3F00200800000000000000B43F002087
S2240182C00800000000000000943E00201000000000000000BC3F002008000000000000006B
S2240182E0A03D00201C000000000000001F3F00200100000000000000203F00200C00000055
S224018300000000008C3C00202C00000000000000B83C00202C0000000000000025100020AE
S22401832001000000000000002C3F00200C00000000000000C43F0020080000000000000074
S224018340CC3F00200800000000000000D43F002008000000000000002D200020010000003B
S22401836000000000913E00200100000000000000B14000200100000000000000D5410020BF
S2240183800100000000000000E43C002020000000000000009C400020060000000100000073
S2240183A01000803000070000D439002060000000000000008C350020C000000001000000C1
S2240183C0000000000000008000020305000000000080000000020305000000000000020081
S2240183E0000203050000000000001000000203050000000000000002000203050000000047
S22401840002000000000203050000000020000000000203050000000008000000000203050E
S224018420000000000004000000020205000000000008000000020205000000000010000008
S22401844000020205000000000020000000020205000000000040000000020205000000009B
S224018460000000400002030500000000000020000002030500000000000001000002030577
S224018480383F00200C000000010000009C4000208C350020D4390020343A0020600000003A
S2240184A00000000000420020030000000100000000010200443F00200C000000010000009D
S2240184C010000300A040002000420020503F00200C0000000100000000000000343A0020D7
S2240184E0D4390020DC3F00200800000001000000503F0020443F0020803F00200A000000CA
S22401850001000000100003FA0301140514010000E43F002008000000000000004C36002028
S224018520C0000000000000005C3C002030000000010000003002003002003602003D0201B0
S2240185403C02013902013F02014802013102013602012F02013702013B0201300200300292
S224018560003C0200A43E00201000000001000000E43F0020803F00204C3600205C3C002028
S224018580B43E00201000000001000000080005000300058103138C004C3600205C3F00201D
S2240185A00C00000000000000EC3F002008000000010000005C3F0020B43E0020B440002074
S2240185C004000000000000006C3900206800000000000000AC26002014000000000000005E
S2240185E0F43F00200800000000000000D94100200100000000000000DD41002001000000A0
S22401860000000000E14100200100000000000000B84000200400000000000000FF41002095
S2240186200100000000000000103E00201800000000000000E5410020010000000000000066
S224018640E94100200100000000000000ED4100200100000000000000F14100200100000027
S22401866000000000BC4000200400000000000000F54100200100000000000000043F00201A
S2240186800D0000000000000020000020051000000000000028100020051000000000000005
S2240186A0FC4100200300000000000000E64100200200000000000000EA41002002000000BE
S2240186C000000000F94100200100000000000000C0400020040000000000000003420020B0
S2240186E00100000000000000044200200100000000000000054200200100000000000000A4
S224018700064200200100000000000000074200200100000000000000084200200100000015
S224018720000000000942002001000000000000000A4200200100000000000000C440002036
S22401874004000000000000008C3F00200A00000000000000C84000200400000000000000EE
S224018760683F00200C00000000000000AC4000200500000000000000842B0020100200002E
S224018780000000006C3800208000000000000000542F002048010000000000000B42002036
S2240187A00100000000000000AC23002000030000000000009C300020400100000000000093
S2240187C0C43E00201000000000000000CC4000200400000000000000D040002004000000FD
S2240187E000000000D44000200400000000000000FC3F002008000000000000000C4200206A
S22401880001000000000000000D42002001000000000000000E420020010000000000000070
S2240188200F4200200100000000000000EE4100200200000000000000F2410020020000001A
S22401884000000000F64100200200000000000000D84000200400000001000000000000205C
S224018860104200200100000000000000114200200100000001000000010000001242002095
S2240188800100000000000000FA4100200200000000000000134200200100000000000000FE
S2240188A0803E00201100000000000000DC4000200400000000000000A44000200600000079
S2240188C000000000D43E00201000000000000000E43E00201000000000000000F43A0020B0
S2240188E05A0000000000000044290020400200000100000086F10100010000005D780200F8
S22401890090F11100010000006F70020099F1040001000000937002008AF1060001000000C7
S2240189201D6F020087F11500010000004545020098F1100001000000C970020093F1100020
S224018940010000006D67020095F1100001000000415E02000070020001000000D971020043
S2240189600170020001000000E97102000270020001000000F97102000370020001000000CA
S2240189800972020004700200010000001972020005700200010000002972020006700200C3
S2240189A0010000003972020007700200010000004972020008700200010000005972020084
S2240189C00970020001000000697202000A70020001000000797202000B7002000100000050
S2240189E0897202000C70020001000000997202001070020001000000A972020011700200C5
S224018A0001000000B97202001270020001000000C97202001370020001000000D97202008D
S224018A201470020001000000E97202001570020001000000F97202001670020001000000CE
S224018A400973020017700200010000001973020018700200010000002973020019700200C6
S224018A6001000000397302001A70020001000000497302001B70020001000000597302009A
S224018A801C700200010000006973020020700200010000007973020021700200010000004E
S224018AA08973020022700200010000009973020020900200010000009F68020021900200A0
S224018AC001000000B96802002290020001000000D36802002390020001000000ED6802006D
S224018AE024900200010000000769020025900200010000002169020026900200010000004A
S224018B003B6902002790020001000000556902000290010001000000B973020003900100D9
S224018B2001000000C973020001A0010001000000DB7002000C370020C000000001000000DC
S224018B4090F11100030100008170020099F1040003010000A570020098F110000301000040
S224018B60B77002002090020003010000316F02002190020003010000456F0200229002004D
S224018B8003010000596F020023900200030100006D6F02002490020003010000816F0200BE
S224018BA02590020003010000956F02002690020003010000A96F020027900200030100005B
S224018BC0BD6F02000190010003010000D16F020002900100030100002955020003900100DE
S224018BE003010000B562020004900100030100004558020001A00100030100008967020082
S224018C00CC370020A00000000100000000AE0000030000006B7802000000000000000000F4
S224018C2001AE00000300000079780200000000000000000002AE00000300000087780200D5
S224018C40000000000000000003AE00000300000095780200000000000000000004AE000099
S224018C6003000000A3780200000000000000000005AE000003000000B178020000000000ED
S224018C800000000006AE000003000000BF780200000000000000000007AE00000300000026
S224018CA0CD78020000000000000000006C3E00201200000000000000F84100200100000031
S224018CC000000000F44100200100000000000000043D002020000000000000001442002041
S224018CE00100000000000000154200200100000000000000D83D00201A00000000000000A6
S224018D00F43D00201A0000000000000016420020010000000100000001000000D641002030
S224018D200200000000000000174200200100000000000000DA410020020000000000000074
S224018D40DE4100200200000000000000E2410020020000000000000018420020010000000C
S224018D6000000000F04100200100000000000000EC4100200100000000000000E841002004
S224018D800100000000000000E44100200100000000000000E0410020010000000000000044
S224018DA0DC4100200100000000000000D84100200100000000000000D441002001000000FF
S224018DC0000000000440002008000000000000001942002001000000000000000C40002039
S224018DE008000000000000001A42002001000000000000001440002008000000000000006C
S224018E001C40002008000000000000002440002008000000000000002C40002008000000A8
S224018E20000000003440002008000000000000003C40002008000000000000004440002048
S224018E4008000000000000004C400020080000000000000054400020080000000000000094
S224018E605C40002008000000000000006440002008000000000000006C4000200800000088
S224018E80000000007440002008000000000000007C40002008000000000000008440002028
S224018EA008000000000000008C40002008000000000000001B420020010000000000000032
S224018EC01C42002001000000000000001D42002001000000000000001E420020010000000C
S224018EE000000000E04000200400000000000000E44000200400000000000000E840002098
S224018F000400000000000000EC4000200400000000000000F04000200400000000000000A3
S224018F20F44000200400000000000000F84000200400000000000000FC4000200400000017
S224018F400000000000410020040000000000000004410020040000000000000008410020D4
S224018F6004000000000000000C410020040000000000000010410020040000000000000001
S224018F801441002004000000000000001841002004000000000000001C4100200400000054
S224018FA0000000002041002004000000000000001F42002001000000000000002042002022
S224018FC0010000000000000021420020010000000000000022420020010000000000000081
S224018FE02342002001000000000000002442002001000000000000002542002001000000D6
S2240190000000000026420020010000000000000027420020010000000000000024410020B2
S2240190200400000000000000583E00201400000000000000283E00201800000000000000BE
S224019040284100200400000000000000284200200100000000000000294200200100000066
S224019060000000002A42002001000000000000002B42002001000000000000002C42002041
S22401908001000000000000002D4200200100000000000000522F0020020000000000000096
S2240190A04E3B00200200000000000000F23D002002000000000000000E3E00200200000040
S2240190C0000000007E3E002002000000000000008A3F00200200000000000000963F0020CC
S2240190E00200000000000000A23F00200200000000000000A2400020020000000000000061
S224019100AA40002002000000000000002610002002000000000000002E2000200200000075
S22401912000000000923E00200200000000000000B240002002000000000000007241002050
S22401914002000000000000007441002002000000000000002E42002001000000000000009F
S2240191607641002002000000000000007841002002000000000000007A4100200200000058
S224019180000000007C41002002000000000000007E41002002000000000000008041002028
S2240191A00200000000000000824100200200000000000000844100200200000000000000DB
S2240191C08641002002000000000000008841002002000000000000008A41002002000000C8
S2240191E0000000008C41002002000000000000008E41002002000000000000009041002098
S22401920002000000000000009241002002000000000000009441002002000000000000005A
S2240192209641002002000000000000009841002002000000000000009A4100200200000037
S224019240000000009C41002002000000000000009E4100200200000000000000A041002007
S2240192600200000000000000A24100200200000000000000A44100200200000000000000DA
S224019280A64100200200000000000000A84100200200000000000000AA41002002000000A7
S2240192A000000000AC4100200200000000000000AE4100200200000000000000B041002077
S2240192C00200000000000000B24100200200000000000000B441002002000000000000005A
S2240192E02F42002001000000000000003042002001000000000000003142002001000000AF
S224019300000000003242002001000000000000003342002001000000000000003442002086
S2240193200100000000000000354200200100000000000000364200200100000000000000F5
S224019340374200200100000000000000384200200100000000000000394200200100000036
S224019360000000003A42002001000000000000003B42002001000000010000000F0000009C
S2240193803C42002001000000010000000F0000003D42002001000000010000000100000076
S2240193A02C4100200400000001000000FFFFFFFFA03B00204000000000000000E03B0020A3
S2240193C0400000000000000030410020040000000000000034410020040000000000000019
S2240193E03E4200200100000001000000010000003F42002001000000000000004042002080
S2240194000100000000000000B64100200200000000000000942D0020BE010000000000008C
S224019420302000207C03000001000000000000000000B8420080B74300C0494400E0AF44A2
S22401944000E004450070384500906F45004894450028B0450040CA450050E14500C0F345B1
S2240194600074004600840346000003460070FC450060EA450028CF450038AB4500207D4590
S22401948000E013450080E24300C0CEC4008074C500F0C3C5008407C600E42CC600FC50C62D
S2240194A000F872C600DC88C6002A96C600F0A0C600C4A8C60050ADC6003EAEC60064ABC6F4
S2240194C0008AA4C600C099C600F08AC600C870C6007444C600B011C60098B2C50040E2C43B
S2240194E000A010450010C94500D8224600085E4600548A4600EAA2460042B84600E4C9463E
S2240195000088D74600DAE04600AEE54600F4E546009EE14600C4D84600A2CB460062BA46EC
S2240195200078A54600368D46004C644600A429460028D74500702D4500A0ADC400B8ACC550
S224019540004015C6003451C6007A84C600BA9DC600D0B3C6004EC6C600E0D4C60026DFC656
S2240195600004E5C6004AE6C600F6E2C60020DBC600EACEC6008CBEC6006CAAC600DC92C643
S22401958000BC70C6001037C60010F3C5004067C50000E94300108F450074054600CC3F4672
S2240195A00058754600A69246004AA746004EB8460058C546004CCE4600EED246005CD34653
S2240195C00086CF46009CC74600E8BB460094AC4600209A4600E6844600B85A460034284628
S2240195E00038E64500C072450000C24300303FC50038C7C500A414C600AC41C600206AC60D
S224019600008886C6000095C6003EA0C6000CA8C6005CACC60028ADC60074AAC60072A4C6CE
S224019620003E9BC600248FC6007280C600EC5EC6004C39C600B010C60048CCC500B069C5BC
S224019640008068C40080E54400C88C450050DB4500F4114600543246008C4E4600D06546F4
S224019660000C7846006482460002864600DA864600FC8446007A8046001C734600A4604655
S22401968000444A460068304600A8134600C0E94500F8A84500904D450000924400C066C45C
S2240196A0007036C5005096C50038CCC50088FCC5001413C6004424C6008C31C600DC3AC602
S2240196C0000440C6002441C600643EC600B837C600C82DC6007C20C6009810C60088FCC55E
S2240196E00048D4C50058A9C5002079C500C01EC5008088C4008098430000CD4400E033452C
S22401970000F0794500D09B4500E0B54500E0CA450098DA450000E54500D8E94500D0E94537
S2240197200098E4450000DB450060CD450000BC450008A84500809145001073450000414536
S22401974000A00E450080B94400003444000000C000C023C400A09AC400C0D8C400A005C5F0
S224019760001019C5005026C500C02DC500702FC500702CC500F023C500D018C5002009C5D0
S2240197800040F1C40000CBC400C0A5C4000080C400803AC40000FAC3008091C3000009C3F7
S2240197A0000020C200000000983F00200A000000000000004142002001000000000000001C
S2240197C0B84100200200000000000000384100200400000000000000424200200100000026
S2240197E0000000004342002001000000010000000300000044420020010000000000000012
S224019800DC320020F000000000000000CC330020F000000000000000203C00203C0000005D
S22401982000000000454200200100000000000000464200200100000000000000BA410020B6
S2240198400200000000000000BC41002002000000000000003C410020040000000000000040
S224019860404100200400000000000000444100200400000000000000243D002020000000F3
S22401988000000000443D00202000000000000000403E00201800000000000000F43E0020F9
S2240198A01000000000000000944000200800000000000000743F00200C00000000000000B7
S2240198C0704100200200000000000000474200200100000000000000484100200400000058
S2240198E000000000484200200100000000000000BE4100200200000000000000C041002075
S22401990002000000010000005E010000C24100200200000001000000AF000000494200205F
S22401992001000000000000004A42002001000000000000004B4200200100000000000000C5
S2240199404C42002001000000000000004D42002001000000000000004E42002001000000F1
S224019960000000004F4200200100000000000000504200200100000001000000500000002B
S224019980514200200100000000000000524200200100000001000000FF00000053420020A3
S2240199A00100000001000000FF000000C44100200200000000000000C64100200200000050
S2240199C000000000C84100200200000000000000643D00202000000000000000CA4100204A
S2240199E00200000000000000CC410020020000000000000054420020010000000000000079
S224019A00CE410020020000000000000055420020010000000000000056420020010000009E
S224019A200000000057420020010000000000000058420020010000000000000059420020F0
S224019A4001000000000000005A42002001000000000000005B420020010000000000000084
S224019A605C42002001000000000000005D42002001000000000000004C41002004000000B0
S224019A80000000005041002004000000000000005441002004000000000000005E42002092
S224019AA001000000000000005F4200200100000000000000D04100200200000000000000AA
S224019AC0584100200400000000000000C02600208402000000000000943A002060000000E9
S224019AE000000000DC3100200001000000000000EC38002080000000000000005C410020B1
S224019B000400000000000000604100200400000000000000644100200400000000000000AD
S224019B2060420020010000000100000001000000BC3D00201C0000000000000010000020F5
S224019B401000000000000000D24100200200000000000000123F00200D000000000000003C
S224019B60684100200400000000000000503B002050000000000000006C4100200400000046
S224019B80000000000000000000000000222222222DE9F043ABB008F029F901200DF082F9E0
S224019BA0852839D0AF4B00221A7000200DF07AF985283DD0AC4B00221A7002200DF072F9CC
S224019BC0852840D1A94B03221A70A94B01221A70A84B1B7813F0010F3ED10023A64A13703F
S224019BE0A64A1370A64A1370A64A1370A64A1370A64A1370A64A13709C4B1B78013B072BC5
S224019C0000F25C81DFE813F05201A301AC01B501BE01C701D001D9010E200DF043F9852805
S224019C20C0D1924B02221A708E4B01221A70BCE70D200DF037F98528BCD101238B4A1370C9
S224019C40894A1370B9E70F200DF02CF98528B9D0874B00221A70BBE702AC8E4D0FCD0FC429
S224019C6095E80F0084E80F000AAC8B4D0FCD0FC495E80F0084E80F0012AC884D0FCD0FC451
S224019C8095E80F0084E80F001AAC854D0FCD0FC495E80F0084E80F0022AC824D0FCD0FC41D
S224019CA095E80F0084E80F007F4B5A7800EE902A1B7800EE103AB8EE400A8DED000AF8EE2E
S224019CC0600ACDED010A9DED084ADDED094A9DED063ADDED073A9DED042ADDED052A9DED46
S224019CE0021ADDED031A0AF03FF988B15F4B1B78013BDBB2022B7FF67FAF5C4B04221A70C3
S224019D0001235D4A13705D4A1370614A137073E79DED104ADDED114A9DED0E3ADDED0F3A4F
S224019D209DED0C2ADDED0D2A9DED0A1ADDED0B1A9DED000ADDED010A0AF016F990B14B4B76
S224019D401B78013BDBB2022B7FF656AF474B05221A700123484A1370494A13704C4B0222AD
S224019D601A7049E79DED184ADDED194A9DED163ADDED173A9DED142ADDED152A9DED121A8E
S224019D80DDED131A9DED000ADDED010A0AF0ECF890B1364B1B78013BDBB2022B7FF62CAFE4
S224019DA0324B07221A700123334A1370354A1370374B04221A701FE79DED204ADDED214AE6
S224019DC09DED1E3ADDED1F3A9DED1C2ADDED1D2A9DED1A1ADDED1B1A9DED000ADDED010A71
S224019DE00AF0C2F890B1214B1B78013BDBB2022B7FF602AF1D4B06221A7001231E4A137024
S224019E00214A1370224B03221A70F5E69DED284ADDED294A9DED263ADDED273A9DED242A31
S224019E20DDED252A9DED221ADDED231A9DED000ADDED010A0AF098F800283FF4DDAE0B4B07
S224019E401B78013BDBB2022B7FF6D6AE074B08221A700123084A13700C4A13700C4B052224
S224019E601A70C9E656420020574200205242002058420020484200204942002059420020B4
S224019E805A4200205B4200205C4200205D420020534200206C2202008C220200AC22020001
S224019EA0CC220200EC220200704100200CF034FFA74B18800CF09CFDA64B188003F07CFF86
S224019EC0A54B1870A54B93F800805FFA88F8B8F1010F7BD0A24B1B78012B00F0E982A14B39
S224019EE09B79042B00F0F2829F4B1A789F4B19789F4B18789F4B1B78DBB2022B00F0EA82B1
S224019F009C4B1B7843B99C4B1B782BB19B4B01241C709B4B00241C70964B1B78DBB2964C5F
S224019F202370984B1B78DBB2012B00F0F482012A00F0F182012900F0EE82012800F0EB8255
S224019F40904B1B78DBB2012B40F0FA82F3E20CF0EFFE7F4B18800CF058FD7E4B1880ADE7C2
S224019F600CF0F2FE7A4B18800CF070FC794B1880A4E70CF0F5FE764B18800CF053FD754BEF
S224019F8018809BE70CF0F8FE714B18800CF057FD704B188092E70CF0FBFE6D4B18800CF0FE
S224019FA05BFD6C4B188089E70CF0FEFE684B18800CF05FFD674B188080E70CF001FF644B8D
S224019FC018800CF063FD634B188077E76E4F6F4E0024A5B228460CF051FF27F8020F284696
S224019FE00CF056FF26F8020F0134102CF1D10DF0C5FC674B187010F0010F1CD1594B9B79FB
S22401A000032B00F08880012B02D0564B00229A71544A00231371537193609370D370137083
S22401A0205370D3605B4A137053705B4F3E4600254FF00109B8E000200CF03EFF0446012041
S22401A0400CF03AFFC1B2E0B208F07AFB514A137844490B7052784A70898811B941490B71C0
S22401A0604A7140498D79ADB90C4608794F7989680131A160E6680136E6601C460646181AC0
S22401A0800E301C2840F29C823649002088718870C8702EE0334CA078E778A1680131A160E0
S22401A0A0E6680136E6601C460646181A0E301C2818D89446BE46D01B0E301C2812D869B12E
S22401A0C04DB928493019401088700EEB0C004010C8700120887123490120886021490B7170
S22401A0E04A7109E005F0FD05012DCDD11D49032088711C490B714A711A4BDA684EF65F2368
S22401A1009A426DD9174B4EF66022DA6004229A714FF0000889E7134B9878D9781A795B79A7
S22401A120141A0E341C2C07D85C1A0E341C2C03D80C4B02229A716BE705F0A8FE084B187257
S22401A14000283FF465AF1E225A6001221A705FE7C0410020C241002047420020B14000209F
S22401A160743F0020F43E00205642002058420020574200204B4200204C4200204E4200207E
S22401A1804D42002049420020223D0020423D0020484200207041002094400020204607F075
S22401A1A0CDFE307001350136ECB2022CF6D94946204609F051FA30700134E4B2072CF1D985
S22401A1C0B54B1B78013B072B00F23D81DFE813F00B00310057007D00A400CB00F100160177
S22401A1E04FF0000821E7002007F0A8FE0446AB4B1870002840F0468100264FF001090DE00A
S22401A200284607F09BFE387030B90134E4B20135EDB2072D00F2348101360137F5B2022DE9
S22401A220EED94946284609F017FA38700028ECD0EDE7012007F082FE0446984B5870002835
S22401A24040F0208100264FF001090DE0284607F075FE387030B90134E4B20135EDB2072D8E
S22401A26000F20E8101360137F5B2022DEED94946284609F0F1F938700028ECD0EDE70220E9
S22401A28007F05CFE0446854B9870002840F0FA8000264FF001090DE0284607F04FFE3870BD
S22401A2A030B90134E4B20135EDB2072D00F2E88001360137F5B2022DEED94946284609F07F
S22401A2C0CBF938700028ECD0EDE70121032009F0C3F90446714BD870002840F0D38000263B
S22401A2E04FF001090DE0284607F028FE387030B90134E4B20135EDB2072D00F2C1800136C8
S22401A3000137F5B2022DEED94946284609F0A4F938700028ECD0EDE70121042009F09CF99B
S22401A32004465E4B1871002840F0AC8000264FF001090DE0284607F001FE387030B9013491
S22401A340E4B20135EDB2072D00F29A8001360137F5B2022DEED94946284609F07DF938702C
S22401A3600028ECD0EDE70121052009F075F904464A4B5871002840F0858000264FF00109FD
S22401A3800CE0284607F0DAFD387028B90134E4B20135EDB2072D73D801360137F5B2022DA2
S22401A3A0EFD94946284609F057F938700028EDD0EEE70121062009F04FF90446374B9871C9
S22401A3C000285FD100264FF001090CE0284607F0B5FD387028B90134E4B20135EDB2072D50
S22401A3E04ED801360137F5B2022DEFD94946284609F032F938700028EDD0EEE70121072058
S22401A40009F02AF90446254BD87100283AD100264FF001090CE0284607F090FD387028B90E
S22401A4200134E4B20135EDB2072D29D801360137F5B2022DEFD94946284609F00DF9387090
S22401A4400028EDD0EEE7002634464FF00109F5B2022D07D8284607F071FD387068B90134CD
S22401A460E4B206E04946284609F0F6F838700028F5D06B1CDBB2072B02D801360137E6E785
S22401A480082C11D0B8F1000F02D0054B00229A71044B00221A701DE55242002094400020F5
S22401A4A0F43E0020B1400020494BFF221A70E9E7484B5B682BB1013B464A5360002B7FF4D5
S22401A4C00EAD444B00221A721A7008E5424B00229A7109E5414B1B78DBB2022B3FF410AD96
S22401A4E03F4B1B78042B3FF60BAD3E4C24789C427FF406AD3C4B1B78042B3FF601AD3B4C40
S22401A50024789C427FF4FCAC394B01241C70394B00241C7000E5384B1B78DBB2022B1BD097
S22401A520364B1B78DBB2012B05D0012A03D0012901D0012804D12E4B1B78DBB2012B13D0D4
S22401A5402C4B1B78DBB2012B1ED0214B1B78FF2B32D02BB0BDE8F083294B1B78012BDFD143
S22401A560284B01241C70DBE7254B1B78012BE7D1254B01221A70254B197831200BF022F884
S22401A5801B4B00221A70E0E71E4B1B78DBB2012BDBD11D4B1B78012B05D00023154A13707A
S22401A5A0184A1370D1E7184B00221A70174B197831200BF007F8F0E7114B01221A70C8E71C
S22401A5C09446BE46D01B0E301C283FF65DAD76E552420020743F0020F43E00204C42002009
S22401A5E02A4200202D4200202B4200202C4200204D4200204E4200204B4200204942002068
S22401A6002E4200204A420020514200204F420020A0F580500138642800F25084DFE810F0DD
S22401A620B300A60099008D00BE007F027202650259024E024102340227021B020E020302FC
S22401A640F801E601C001B301A801EC01900183019B01B102A502980292028C02B702760112
S22401A66069015E0151014B0145013F01390133012D012701210110010A010401FE00F800EA
S22401A680F200EC001601C402CD0286038F039803A103AA03B303BC03C503CE03D703E00358
S22401A6A0E903F203FB03D602DF02E802F102FA0203030C0315031E032703300339034203F7
S22401A6C04B0362036B0374037D03DB00D500CF00C900E1003004880083007E007900740089
S22401A6E06F006A00650004041A040A78B24B1A70002070470A78B14B1A70002070470A78AF
S22401A700AF4B1A70002070470A78AE4B1A70002070470A78AC4B1A70002070470A78AB4BAA
S22401A7201A70002070470A78A94B1A70002070470A78A84B1A7000207047A74A137803F096
S22401A740FC031370097801F003010B43137000207047A148037803F0F30303700A7892007F
S22401A76002F00C0213430370002070479A48037803F08F0303700A78120102F0700213438F
S22401A780037000207047944A137803F07F031370097843EAC1131370002070478E4A537889
S22401A7A003F07F035370097843EAC1135370002070478A4B0020D8700A78DA707047874BAD
S22401A7C0002098700A789A707047844B002058700A785A707047814B002018700A781A70CE
S22401A7E070477E4A137903F07F031371097843EAC113137100207047794B0020D8700A78C4
S22401A800DA707047764B002098700A789A707047734B002058700A785A707047704B002081
S22401A82018700A781A7070476D4B002098710A789A7170476A4B002058710A785A71704700
S22401A840674B002018710A781A717047644AD37903F07F03D371097843EAC113D37100203A
S22401A8607047604B002018710A781A7170475D4B0020D8700A78DA7070475A4B00209870A3
S22401A8800A789A707047574B002058700A785A707047544B002018700A781A707047514B3C
S22401A8A00020D8710A78DA7170474E4B002098710A789A7170474B4B002058710A785A71D3
S22401A8C070474948C37903F0EF03C3710A78120102F010021343C37100207047424AD37903
S22401A8E003F01F03D371097843EA4113D371002070473D48037903F0EF0303710A781201ED
S22401A90002F0100213430371002070473648037903F0F10303710A78520002F00E0213430B
S22401A9200371002070473048837803F0CF0383700A78120102F030021343837000207047C2
S22401A940294A937803F03F039370097843EA81139370002070472448037903F0BF0303710E
S22401A9600A78920102F0400213430371002070471D4A537903F03F035371097843EA811379
S22401A9805371002070471848437903F0CF0343710A78120102F030021343437100207047E7
S22401A9A0114A537903F0F0035371097801F00F010B43537100207047F0410020EC410020B7
S22401A9C0E8410020E4410020E0410020DC410020D8410020D4410020144000201C40002007
S22401A9E0244000202C40002034400020B64B002098710A789A717047B34A137903F0FE03C2
S22401AA001371097801F001010B43137100207047AD4A137903F07F031371097843EAC11391
S22401AA20137100207047A84A137803F03F031370097843EA8113137000207047A24803797E
S22401AA4003F0DF0303710A78520102F0200213430371002070479C4A537803F0FC035370B7
S22401AA60097801F003010B435370002070479648437803F0FB0343700A78920002F0040229
S22401AA8013434370002070478F48437803F0E70343700A78D20002F0180213434370002025
S22401AAA070478948437803F0DF0343700A78520102F020021343437000207047824A537865
S22401AAC003F03F035370097843EA81135370002070477D4A137803F0FE031370097801F061
S22401AAE001010B431370002070477748037803F0F90303700A78520002F006021343037073
S22401AB00002070477048037803F0F70303700A78D20002F0080213430370002070476A4823
S22401AB20037803F0CF0303700A78120102F030021343037000207047644B002018710A7829
S22401AB401A717047614B0020D8700A78DA7070475E48437803F0CF0343700A78120102F0B6
S22401AB6030021343437000207047584A537803F0F0035370097801F00F010B4353700020F4
S22401AB807047524B002098700A789A7070474F48037803F0FB0303700A78920002F004026E
S22401ABA01343037000207047494B002058704A785A7018700A781A707047454B0020D870A4
S22401ABC04A78DA7098700A789A707047414B002058704A785A7018700A781A7070473D4B45
S22401ABE00020D8704A78DA7098700A789A707047384B002058714A785A7118710A781A7101
S22401AC007047344B0020D8714A78DA7198710A789A717047304B002058704A785A701870BE
S22401AC200A781A7070472C4B0020D8704A78DA7098700A789A707047274B002058714A78F8
S22401AC405A7118710A781A717047234B0020D8714A78DA7198710A789A7170471F4B00201B
S22401AC6058704A785A7018700A781A7070471B4B0020D8704A78DA7098700A789A7070470A
S22401AC80164B002058714A785A7118710A781A717047124B0020D8714A78DA7198710A782C
S22401ACA09A7170470E4B002058704A785A7018700A781A7070470A4B0020D8704A78DA70EB
S22401ACC098700A789A707047344000203C400020444000204C400020544000205C40002033
S22401ACE064400020764B002058714A785A7118710A781A717047724B0020D8714A78DA71D3
S22401AD0098710A789A7170476E4B002058704A785A7018700A781A7070476A4B0020D8704B
S22401AD204A78DA7098700A789A707047654B002058714A785A7118710A781A717047614B97
S22401AD400020D8714A78DA7198710A789A7170475D4B002058704A785A7018700A781A707A
S22401AD607047594B0020D8704A78DA7098700A789A707047544B002058714A785A71187115
S22401AD800A781A717047504B0020D8714A78DA7198710A789A7170474C4B002058704A784A
S22401ADA05A7018700A781A707047484B0020D8704A78DA7098700A789A707047434B002078
S22401ADC058714A785A7118710A781A7170473F4B0020D8714A78DA7198710A789A7170477D
S22401ADE03B4B002058704A785A7018700A781A707047374B0020D8704A78DA7098700A7888
S22401AE009A707047324B002058714A785A7118710A781A7170472E4B0020D8714A78DA713C
S22401AE2098710A789A7170470A782A4B1A704A785A708A789A70CA78DA700A791A714A7949
S22401AE405A718A799A71CA79DA71234B08221A70002070470A78214B1A704A785A708A7886
S22401AE609A70CA78DA700A791A714A795A718A799A71CA79DA711A4B08221A70002070470E
S22401AE80184B002018700A781A7058704A785A7098708A789A70D870CA78DA7018710A794D
S22401AEA01A7158714A795A7198718A799A71D871CA79DA710C4B08221A7070470120704722
S22401AEC0644000206C400020744000207C4000208440002004400020194200200C400020FD
S22401AEE01A4200208C4000201B4200202DE9F04F85B00CF05BFDADF80E000CF051FDADF8E7
S22401AF000C000CF059FD83B201930DF10E0141F23400FFF77DFB03A941F23500FFF778FBA5
S22401AF201C4E1D4D0024DFF87490A246DFF870B00EE001228BF800202AE0C5F800A03368A3
S22401AF400BB1013B33600134043604350F2C29D01FFA84F840460BF091FF074640460BF010
S22401AF6097FF04EB440313F8093018448742E4DD2B6801332B6046F2A8129342DFD933468B
S22401AF803268002AD5D14DF2D8623260C5F800A01B68D6E7E03B0020A03B00205C3C0020AB
S22401AFA0294200200024E5B2A0B20BF071FF002800F0B8820135EDB20134102CF3D1102DEF
S22401AFC000F0CE82974B1B68002B40F0BC8200200BF054FF944D288001200BF04FFF934BEE
S22401AFE0188002200BF04AFF914B188003200BF045FF904B188004200BF040FF8E4B188035
S22401B00005200BF03BFF8D4B188006200BF036FF8B4B188007200BF031FF8A4B18800820B5
S22401B0200BF02CFF884B188009200BF027FF874B18800A200BF022FF854B18800B200BF0F1
S22401B0401DFF844B18800C200BF018FF824B18800D200BF013FF814B18800E200BF00EFFF0
S22401B0607F4B18800F200BF009FF7E4B188000200BF00EFF7C4C208001200BF009FF7B4B5B
S22401B080188002200BF004FF794B188003200BF0FFFE784B188004200BF0FAFE764B1880B0
S22401B0A005200BF0F5FE754B188006200BF0F0FE734B188007200BF0EBFE724B1880082032
S22401B0C00BF0E6FE704B188009200BF0E1FE6F4B18800A200BF0DCFE6D4B18800B200BF06E
S22401B0E0D7FE6C4B18800C200BF0D2FE6A4B18800D200BF0CDFE694B18800E200BF0C8FEB4
S22401B100674B18800F200BF0C3FE664B18802B882288934286BF9B1A9BB20023624A1380D0
S22401B120424B1B88514A1288934286BF9B1A9BB200235E4A13803E4B1B884D4A12889342F8
S22401B14086BF9B1A9BB20023594A1380394B1B88484A1288934286BF9B1A9BB20023554A18
S22401B1601380354B1B88444A1288934286BF9B1A9BB20023504A1380304B1B883F4A12883E
S22401B180934286BF9B1A9BB200234C4A13802C4B1B883B4A1288934286BF9B1A9BB20023C9
S22401B1A0474A1380274B1B88364A1288934286BF9B1A9BB20023434A1380234B1B88324A4A
S22401B1C01288934286BF9B1A9BB200233E4A13801E4B1B882D4A1288934286BF9B1A9BB23C
S22401B1E000233A4A13801A4B1B88294A1288934286BF9B1A9BB20023354A1380154B1A88A7
S22401B200244B1B889A4286BFD21A92B20022314B1A80114B1A88204B1B889A4284BFD21A76
S22401B22092B259E034410020522F00204E3B0020F23D00200E3E00207E3E00208A3F00202C
S22401B240963F0020A23F0020A2400020AA400020261000202E200020923E0020B240002020
S22401B260724100207441002076410020784100207A4100207C4100207E41002080410020F8
S22401B280824100208441002086410020884100208A4100208C4100208E4100209041002058
S22401B2A0924100209441002096410020984100209A4100209C4100209E410020A0410020B8
S22401B2C0A2410020A4410020A6410020A8410020AA410020AC41002098BF0022A24B1A8038
S22401B2E0A24B1A88A24B1B889A4286BFD21A92B20022A04B1A80A04B1A88A04B1B889A423A
S22401B30086BFD21A92B200229D4B1A809D4B1B8898423ABF1B1A9BB200239B4A13809B49AF
S22401B32041F24500FFF774F9994941F24700FFF76FF9984941F24900FFF76AF9964941F2AA
S22401B3404B00FFF765F9954941F24D00FFF760F9934941F24F00FFF75BF9924941F2510094
S22401B360FFF756F9904941F25300FFF751F98F4941F25500FFF74CF98D4941F23700FFF712
S22401B38047F98C4941F23900FFF742F98A4941F23B00FFF73DF9894941F23D00FFF738F91F
S22401B3A0724941F23F00FFF733F9734941F24100FFF72EF9734941F24300FFF729F9DFF8CA
S22401B3C038B2594641F24400FFF722F97C4941F24600FFF71DF97B4941F24800FFF718F9C6
S22401B3E0794941F24A00FFF713F9784941F24C00FFF70EF9DFF804A2514641F24E00FFF73E
S22401B40007F9734941F25000FFF702F9DFF8F091494641F25200FFF7FBF8DFF8E8814146DA
S22401B42041F25400FFF7F4F86A4F394641F23600FFF7EEF8684E314641F23800FFF7E8F8B2
S22401B440664D294641F23A00FFF7E2F8644C214641F23C00FFF7DCF8454941F23E00FFF742
S22401B460D7F846494FF48250FFF7D2F85D4941F24200FFF7CDF85C4BBBF800201A80504A0F
S22401B48012885A804F4A12889A804F4A1288DA804E4A12881A81BAF800205A814C4A1288AE
S22401B4A09A81B9F80020DA81B8F800201A823A885A8232889A822A88DA8222881A83334A8D
S22401B4C01288DA83324A12881A84324A12885A84314A12889A84314A1288DA84304A12880D
S22401B4E01A85304A12885A852F4A12889A852F4A1288DA852E4A12881A862E4A12885A866C
S22401B5002D4A12889A862D4A1288DA86BDF80E209A87BDF80C20DA87019AA3F8402005B0F2
S22401B520BDE8F08F314A13680133136046F2A81293427FF644AD2E4B1B6843B12D4A01218E
S22401B5401170102D0CD0013B294A13603FE5284B4DF2D8621A6008F037FD0BF0B1FA2EE5BA
S22401B560224B00221A602DE5AE410020B240002090410020B04100207241002092410020C1
S22401B580B241002074410020B4410020522F00204E3B0020F23D00200E3E00207E3E0020C7
S22401B5A08A3F0020963F0020A23F0020A2400020AA400020261000202E200020923E0020E6
S22401B5C0784100207A4100207C4100207E41002082410020884100208A4100208C41002051
S22401B5E08E41002094410020F43A00203041002034410020294200207641002080410020AA
S22401B60084410020864100202DE9F047B8B005460F46164600248DF8DF40ADF8DC40369454
S22401B620FF238DF8D730ADF8D4408022214615A80CF0E2F8282221460BA80CF0DDF86B1E43
S22401B640092B00F29982DFE813F00A00350097029100970269019702970297024002012E31
S22401B66006D0132528460AF0DDFD38B0BDE8F0873C78012102910023019300910B460A461E
S22401B680204609F033FD08B13125EBE737A809F031FF08B11025E5E7C14B01225A709C706D
S22401B6A0DA70BDF8DC20110A19715A7105200BF073FDD7E7012E01D01325D3E70121029124
S22401B6C00023019300910B460A46387809F00EFD08B13125C6E70DF1D7000CF0B4F910B1CC
S22401B6E000238DF8D73037A809F004FF9DF8D73063B901250024AA4B02225A70FF229A70AA
S22401B700A000023080B20BF047FDABE70DF1DF0136A807F081FD054618BB00242346A04E84
S22401B7200EE00134A4B20DF1DF0136A807F074FD0546B8B92346BDF8DC10621E91420EDB64
S22401B740B4F5806FEDD2369A06EB8303110CD970110A19715A719DF8DF209A71E1E73125B2
S22401B760C9E70024012D18BF3125C4E73B787C78240204EB0344BB781C440DF1DF02012152
S22401B78020460AF08DFA002840F0F881042E01D0132567E7824B220C9A70220ADA701C715A
S22401B7A09DF8DF205A7104225A7005200BF0F4FCFF78FF2F07D07B1EDBB2012B01D9312526
S22401B7C050E7002600E000264FF400790DF1D40814E00DF153030DF12B020DF1670013F887
S22401B7E0011F02F8011F8342F9D106E00023ADF8D4300135EDB2022D20D80136F5B2ADF849
S22401B800D490CDF8008015AB2A460121204606F019FE0028EAD1012DDBD0022DE6D10DF114
S22401B82053030DF13F020DF1670013F8011F02F8011F8342F9D10023ADF8D430022F24D043
S22401B840FF2F33D0564A012302F8063F0BAB0DF13F0013F8011F02F8011F8342F9D11420B3
S22401B8600BF09AFC4E4B0521D971B0221A7201255D721A7303205873DA73042018749A744F
S22401B880D9749A750622DA75ECE6454A022302F8063F10AB0DF1530013F8011F02F8011FB9
S22401B8A08342F9D114200BF077FCDBE73C4A012302F8063F0DF13F000BAB13F8011F02F88E
S22401B8C0011F8342F9D10DF13F03364A0DF1530013F8011F02F8011F9842F9D1304B02221A
S22401B8E09A760521D976B0221A770120587783F82020032083F8210083F82320042083F893
S22401B900240083F8262083F8271083F82A20062283F82B2028200BF03FFCA3E7042E01D0CC
S22401B92013259FE63B787D782D0205EB0345BB781D440DF1DF02012128460AF0B1F9002866
S22401B94040F01E81164B2A0C9A702A0ADA701D719DF8DF205A7106225A70FF78FF2F05D09A
S22401B9607B1EDBB2042B01D931257BE6002306930793089309930A9301248DF81C40022386
S22401B9808DF81E3003238DF8203004268DF8226005238DF8243040F2FF1A0DF1160907E052
S22401B9A028100020411000200134E4B2062C1CD0AAEB0603ADF81630B046731CCDF800906C
S22401B9C006AA134422460121284605F0B9FB0028EAD1BDF81630002BE6D038AA904408F844
S22401B9E0C84C01331E44F6B2DEE7032F42D027D9052F54D048D3FF2F5CD1624B9DF81C209A
S22401BA009A719DF81D20DA719DF81E201A729DF81F205A729DF820209A720022DA729DF815
S22401BA2022201A739DF823205A739DF824209A739DF82520DA730F200BF0AEFB012511E68F
S22401BA40012F0CD0022F35D14E4B9DF81E209A719DF81F20DA7107200BF09EFBEEE7494BE3
S22401BA609DF81C209A719DF81D20DA7107200BF093FBE3E7434B9DF820209A710022DA7172
S22401BA8007200BF089FBD9E73E4B9DF822209A719DF82320DA7107200BF07EFBCEE7394BD8
S22401BAA09DF824209A719DF82520DA7107200BF073FBC3E7334B9DF81C209A719DF81D2011
S22401BAC0DA7107200BF068FBB8E70EB11325C9E5012102910020019000910B460A4609F0BB
S22401BAE005FB08B13125BDE50DF1D7000BF0ABFF10B100238DF8D73037A809F0FBFC9DF841
S22401BB00D7305BB901251F4B0A225A70FF229A70B000023080B20BF03FFBA3E50DF1DF01A4
S22401BB2036A807F079FB054610BB0023154C0EE00136B6B20DF1DF0136A807F06DFB054629
S22401BB40B0B93346BDF8DC10721E91420EDBB6F5806FEDD2369A04EB8303110CD970110AF1
S22401BB6019715A719DF8DF209A71E1E73125CAE7012D18BF3125C6E7122573E5312571E5B9
S22401BB8031256FE5281000202DE9F04F054685B0002800F05582D0F804A04FF00008C1461F
S22401BBA0C3460322CDF80880BAF800300193BDF80810019B99421AD32A68137819060AD542
S22401BBC000214FF00C0E019C88B2844200F20C8103F07F031370BBF1000F40F017811378C3
S22401BBE0B9F1000F00F0658143F0010363E1029B0C20AF6800FB03F6BC196068037813F046
S22401BC001E0E1CBF0123BB55BB5D042B7CD00AD8022B32D044D8012B25D0029B08F1030861
S22401BC2001330293C3E7852B00F09280862B00F0B480072BF1D121894388994269D9C91A9B
S22401BC40EB689AF805E089B213F8083043FA0EF3DBB28B425DD86378002B77D14FF0010338
S22401BC60BB550270D9E7BEF1000F03D10221B955082161704FF0010BCFE7617871B1042996
S22401BC8003D9438823810139F3E7238940888342F9D08CBF03F1FF330133F3E7BA55BCE70C
S22401BCA02389B0F802E07345B7D0E86813D910F80810A3EB0E039AF805009BB20141C9B26D
S22401BCC09942AAD89AF80430002BA6D04FF00701B9556370CEE7AEEB030300EB080C10F817
S22401BCE008009BB2984298D89CF8023033B12846039207F001FC039A00288ED14FF0040394
S22401BD00BB559AF80230E4E7B4F808E043889E4504D9BA554FF0000363707EE7E868A3EBF8
S22401BD200E0300EB080C9BB210F808009842F0D29CF802303BB12846039207F0DDFB039AD3
S22401BD4000287FF46AAF6378002B42D0013BC0E72B689AF8081019712389B0F802E0734579
S22401BD6008D96FF07903BB559AF8023063704FF001097FE7E968AEEB030301EB08009BB27A
S22401BD8011F808104078013041FA00F0091AC9B29942E6D24FF001093FE72389B0F802E092
S22401BDA0734506D963780BB9BA55F3E7013B6370F0E7E968AEEB030301EB08009BB211F83E
S22401BDC008104078013041FA00F0091AC9B2994205D26FF07A03BB559AF80330E7E7637887
S22401BDE0002BE1D0013BC1E70EFB01F6AF68B8194468207810F0010F06D1BE5D16F0F70F43
S22401BE001CBF40F0010020700131DCE69AF8091000293FF4E4AE1378012963F07F031370E6
S22401BE207FF4DDAE00210C27019B1FFA81FE73457FF6D5AE07FB01F3AC6804EB030CE35C7F
S22401BE4013F0F70F27D0852B01D0032B2BD1D5F80C8001EB4103434493F802A0BAF1000F3A
S22401BE6019D0002003469E450FD007FB03F6A65D042E01D0862E08D103EB43064644B6782B
S22401BE805645019E04BF012033460133019E9BB29E42E8D838B9DCF80400037823F00103EA
S22401BEA003700131C0E7DCF80400037843F00103F6E723F001031370624B51881B8801F114
S22401BEC0C802934254D95B1A9AB20C2401260327C82A4FD92B68C83A92B25988C8315980A8
S22401BEE01979002940F08680597909B101395971997909B101399971D5F804E09EF80690CE
S22401BF00B9F1000F08D0597931B9BEF800A088B250453DD383F805909EF807C0BCF1000F70
S22401BF2008D0997931B9BEF8008088B2404548D383F806C06B68D9780029C9D0B3F800C085
S22401BF40002104FB0CF88BB26345C1D204FB01F9AB6803EB090E13F80900852806D19EF800
S22401BF600100002849D001388EF801000131EAE78B4203D3002005B0BDE8F08F03F57F4261
S22401BF80FF32521AC82AF5D95A1E521A92B29CE704FB01F0D5F808C00CEB00081CF80000FB
S22401BFA0032801D008280AD1D8F80400B8F808C04088604584BF0CF1010CA8F808C00131D4
S22401BFC0A5E704FB01F0D5F808E00EEB00091EF80000032801D008280AD1D9F80400B9F885
S22401BFE008E0408870453CBF0EF1FF3EA9F808E001319AE7013919719CE703F80960DEF8E2
S22401C000040001EB410E0770E86886449EF80290B9F1000FAAD003EB080A9A45A6D090F812
S22401C02002E0CE4509D1D3F804E09EF800B01BF0010F1CBF1E708EF800700C330330ECE777
S22401C0400B2098E7D2410020A74B2DE9F04F87B05B7A002B00F0DE81A44B4FF0000BCDF832
S22401C06000B01B6801931B6802931B880393A04B1B680493039B1FFA8BF0984206D39A4BD3
S22401C08002225A72009807B0BDE8F08F049B0C2633F81B10062303FB0BF4019B5A689D6887
S22401C0A006FB0B262F5D05EB040AC7F3820796F80B80042F00F2AD81DFE817F0050020001C
S22401C0C07E014801F300B27A02F00F0290450CD9A8EB0200B8F1040FC0B20DD9A8F1030869
S22401C0E0804502DCC2F10407FFB241FA07F8AAF802800BF1010BBDE70746F6E7B8F1040F38
S22401C100029B28BF4FF0040841FA08F8B8F5007FBAF804101FFA88F2AAF80220B5BFC2F59B
S22401C120FF726FF4FF7E0132724493F802E0A7BF384692B292B20020BEF1400F4FEA52023B
S22401C14092B21BD1E0B1F9B1092A21D9C1F30134C1F30320C1F3031501F00F06002F43D06D
S22401C160CF2A01D9002C70D1152A78D9002871D1002C7DD0013C0A20E4B272E00028E2D0DD
S22401C18043F6FF70814208D181220E232A5500932A5D570603D501220CE00027D4E71006AC
S22401C1A009D4029BDA7802F00302032A06D13F22327211222A55AAF804109AE7022A05D1C2
S22401C1C0727A22F00F0272720922F3E7012AE2D1727A02F00F0242F0700272720D22E9E70D
S22401C1E00134CF3AE4B292B2CF2A01D9032CF7D1152A0DD90F2806D1032C1BBF01340520C1
S22401C2000F20E4B206E00130153AC0B292B2EFE70F28F1D0022A12D90F2D0BD10F2800F013
S22401C220FC800130032C4FF00505C0B20BD0022ADAD826E0691C023ACDB292B2EAE70F2D11
S22401C240ECD0032C1DD10324F1E7013CCF3AE4B292B285E70138153AC0B292B284E70028A3
S22401C26086D0022A0BD92DB998B90646054608E02046F6E7691E023ACDB292B2F1E7002DCE
S22401C280F2D0210389B241EA0021314341EA051191E70138022A4FF00A05C0B23FF660AF95
S22401C2A0EFE7B8F1040F96F8089028BF4FF00408B9F13F0F41FA08F81FFA88F71AD1AAF836
S22401C2C002701F2232722A5D012A7FF412AFB8F5007FB5BFC7F5FF776FF4FF730137FF1825
S22401C2E0BFB20A2F5CE000BFBC3D0020180000201C000020002229FA02F1C9075CBF92460B
S22401C300062202F1010248BF4FF0000AD2B2052AF1D9394606F03EFB30B1012202FA0AF282
S22401C32049EA020986F808900122BAF1000F0BD00AF1FF3A5FFA8AFA02FA0AFA327A22EA22
S22401C3400A0A86F808A0BEE72A55BCE796F8099041FA08F81FFA88F84FEA1917072F29D043
S22401C360414606F017FB00BB013701222A5509F00F0949EA07177772AAF802802A5D012A72
S22401C3807FF4B7AEB8F5007F35BFC8F5FF786FF4FF7208F1010890441FFA88F8B8F10A0F66
S22401C3A07FF6A7AE45222A55A3E6002FDDD0013FFFB2DCE70627DAE7B8F1040F727A28BF31
S22401C3C04FF0040812F00F0941FA08F81FFA88F71CD03946059206F0DDFA059A70B909F18E
S22401C3E0FF395FFA89F90121295522F00F0249EA020986F80990AAF8027064E7B9F1070FED
S22401C400F1D009F101095FFA89F9EEE74FF00109EBE7FEE70323009334E6032C01D0054683
S22401C42005E7022A8BBF054605460646064628E700B583B0A64B1B7813F0010F1CD0A54BFC
S22401C4401B78032B0FD1A24A137803F0FE0313709F4B1B78002B40F0C7819F4B187800307D
S22401C46018BF0120C1E19D4B0093082334220121002008F08FFAE6E7954B1B7813F0020F09
S22401C48013D0944B1B78032B05D1914A137803F0FD031370DCE7924B009308234FF440720E
S22401C4A00121002008F076FAEFE7894B1B7813F0040F13D0874B1B78032B05D1844A1378D4
S22401C4C003F0FB031370C3E7864B0093082340F205320121002008F05DFAEFE77C4B1B787F
S22401C4E013F0080F13D07B4B1B78032B05D1784A137803F0F7031370AAE77B4B009308230A
S22401C5004FF45C720121002008F044FAEFE7704B1B7813F0100F13D06E4B1B78032B05D113
S22401C5206B4A137803F0EF03137091E76F4B009308234FF45D720121002008F02BFAEFE716
S22401C540634B1B7813F0200F13D0624B1B78032B05D15F4A137803F0DF03137078E7644BA1
S22401C560009308234FF45E720121002008F012FAEFE7574B1B7813F0400F17D0554B1B7827
S22401C580032B03D05B4B1B78012B05D0504A137803F0BF0313705BE7574B009308234FF418
S22401C5A080620121002008F0F5F9EFE7484B1B7813F0800F12D1484B1B7813F0010F2FD0C2
S22401C5C0444B1B78032B03D04A4B1B78012B1DD0414A137803F0FE03137039E73D4B1B7829
S22401C5E0032B03D0434B1B78012B05D0384A137803F07F0313702BE7404B0093082340F280
S22401C60001420121002008F0C5F9EFE73C4B0093082340F202420121002008F0BBF9D7E79C
S22401C6202D4B1B7813F0020F17D02A4B1B78032B03D0304B1B78012B05D0274A137803F0E7
S22401C640FD03137004E72F4B0093082340F203420121002008F09EF9EFE71F4B1B7813F010
S22401C660040F17D01B4B1B78032B03D0214B1B78012B05D0184A137803F0FB031370E7E692
S22401C680214B0093082340F204420121002008F081F9EFE7104B1B7813F0080F38D00D4B00
S22401C6A01B78032B03D0134B1B78012B05D00A4A137803F0F7031370CAE6144B00930823D2
S22401C6C040F205420121002008F064F9EFE700BF1C420020164200201D42002014400020C6
S22401C6E03C400020344000202C400020244000201C4000205E420020444000204C40002068
S22401C700544000205C400020644000206C400020374B1B7813F0100F17D0364B1B78032BB3
S22401C72003D0354B1B78012B05D0314A137803F0EF0313708CE6314B0093082340F2064278
S22401C7400121002008F026F9EFE7294B1B7813F0200F17D0274B1B78032B03D0264B1B787A
S22401C760012B05D0224A137803F0DF0313706FE6234B0093082340F207420121002008F02D
S22401C78009F9EFE71A4B1B7813F0400F17D0194B1B78032B03D0184B1B78012B05D0144A3D
S22401C7A0137803F0BF03137052E6164B009308234FF481620121002008F0ECF8EFE70C4BE8
S22401C7C01B7813F0800F3FF443AE0F4B009308234FF4C4620121002008F0DCF8044A1378A2
S22401C7E003F07F03137033E6012003B05DF804FB1D420020164200205E420020744000206F
S22401C8007C400020844000208C40002070B58AB0BA4BDB78012B40F28580B84B1B79042B86
S22401C82002D80133B54A1371B44B5B79092B02D80133B24A5371B14B9B79132B02D8013330
S22401C840AE4A9371AD4BDB79182B02D80133AB4AD371AA4B1B88B3F57A7F02D20133A74ACE
S22401C8601380A64BDB78022B60D0A44B1B79052B00F0B480A14B5B790A2B00F0C7809F4B91
S22401C8809B79142B00F031819C4BDB79192B00F049819A4B1B88B3F57A7F00F04881974BA0
S22401C8A0DB78022B00F04881944B1B79052B00F04781924B5B790A2B00F046818F4B9B7953
S22401C8C0142B00F045818D4BDB79192B00F044818A4B1B88B3F57A7F00F04281884C207AFE
S22401C8E009F010F8E07A09F025F8A07A09F03AF8607A09F04FF8207B09F064F8A07907F062
S22401C90021F820790AF040F8E0780AF04AF8607908F064FCE07909F06DF8607809F082F866
S22401C9200AB070BD0133754AD37076E709F0C4FA744C21460BF0E0F809F0D2FA611E0BF087
S22401C940D1F809F0E1FAA11E0BF0CEF809F0F0FAE11E0BF0CDF809F0FFFA211F0BF0C0F82D
S22401C96009F022FB684A611F0BF038F809F008FBA11F0BF0B1F809F02BFBE11F0BF0AEF81E
S22401C98009F03AFBA4F108010BF0B0F809F0AEFDA4F109010BF0AEF807F054FA054600F0BE
S22401C9A0AFFEA4F10A03A4F10B02014628460BF075F80C3C069463790593E3790493A379FE
S22401C9C0039323790293E3780193237A0093637AA27AE17A207B08F05BFC46E706F076FE96
S22401C9E00DF127010BF074F806F070FE0DF126010BF070F845480BF00EF89DF827209DF8B9
S22401CA0026103F4B18780AF001FB33E709F0E6FE05460BF075F83E4C3E4E009623460DF10D
S22401CA2027020146284609F033FA0BF069F8032500952B46F21EE11E05F0F6FF0BF060F816
S22401CA4000952B46B21F211F05F0EEFF14F8043C002B42D0A6F112039B788DF826309DF81F
S22401CA602620264B9A70264C2B4D029504F112030193237A0093637AA27AE17A207B05F0BC
S22401CA8003FB043D029504F111030193237A0093637AA27AE17A207B05F047FB237C0BB36A
S22401CAA000201E4B9DF82620011C18BF01219DF8270005F0EFF9124C254615F80E0F0AF070
S22401CAC0D7FF0BF01BF80AF0CFFF2B4604F10D02A17860780AF013FBD1E609F09BFE8DF868
S22401CAE02600BCE709F088FEDBE7054B597B18780AF0FCFA0A4809F058FDC5E6283E0020B1
S22401CB00583E0020643E0020C4790200C57902006B3E00203A3E0020CB790200303E0020E3
S22401CB20C6790200104B18780AF0DEFEB1E60E4B18780AF0D2FEB2E60C4B0022DA70B3E6AF
S22401CB400A4B00221A71B4E6084B00225A71B5E6064B00229A71B6E6044B0022DA71B7E6E5
S22401CB60024B00221A80B9E6583E0020283E0020F0B583B0984B5B7B022B47D0974B5B7940
S22401CB80022B5FD00023964A1370964A13801E461D460020944B1870044607F063FE924B6D
S22401CBA01B78103B2E2B00F26381DFE813F052006F0061016101EB006101610161016101A0
S22401CBC0F80061016101610161016101610161016101A300610161016101610161014E016B
S22401CBE061016101610161016101D0000A0161012501610161016101610161016101610134
S22401CC00610161016101610161018200774B01221A70714B5D685E89714B00221A70714BA7
S22401CC201E80002EB5D0002DB3D02B786E4A1370687800F07F0440336D4A13706D4B012234
S22401CC401A80AAE7694B00221A70644B1D681E79E2E7B8B1012E40F2FD806B78DB09604AF7
S22401CC601370624B1B780BB9022C04D0F1B2204606F014FAF1E0022E00F2EC80122009F08E
S22401CC80D1FAEAE07F2009F0CDFAE6E010F0170F0BD0022E40F0DE806B78DB09504A137031
S22401CCA00121204608F066FBD7E07F2009F0BAFAD3E0D8B1022E06D0012E40F2CB80002C70
S22401CCC000F0C88000E01CB1122009F0ABFAC4E06B78DB09424A1370454B00225A70012082
S22401CCE00AF05AFA012009F09DFAB6E07F2009F099FAB2E038B3032E08D0042E40F2AA805A
S22401CD0016F0010400F0A680312708E0A97868780AF09DFE09F086FA9FE0212F11D02B19A9
S22401CD205978285D0AF093FE0234A4B2012800F0A380212802D0B442EFD3384609F072FA8E
S22401CD408BE03846FAE77F2009F06CFA85E010F0140F13D0012E7DD9244B1B78012B09D10D
S22401CD60032E77D9F31E9BB2EA1CA97868780AF072FE72E0222009F055FA6EE07F2009F09B
S22401CD8051FA6AE038B1042E64D1EA78A978687808F040FD61E07F2009F044FA5DE060B1AB
S22401CDA0012E57D96B78DB090D4A1370B21E92B2A91C2046FEF728FC4FE07F2009F032FA22
S22401CDC04BE010F0140F02D0022E46D842E07F2009F028FA41E000BFAC260020F43F0020DE
S22401CDE0E5410020E6410020E9410020F541002028100020EA41002010F0140F21D0012E1A
S22401CE0028D9204B1B78012B17D1E0B2431EDBB2022B0ED8032E1DD96B78DB091A4A137091
S22401CE20EA78A978331F9BB200932B1D0AF016F913E0122009F0F6F90FE0122009F0F2F9D4
S22401CE400BE07F2009F0EEF907E010F0140F0BD0032E04D0132009F0E5F903B0F0BD6B782B
S22401CE60DB09094A1370F8E77F2009F0DBF9F4E7112009F0D7F9F0E7B442BFF45FAF0746F7
S22401CE804DE700BFF5410020E54100202DE9F04F85B0002800F07E814568EB79CF2B00F25F
S22401CEA077810468002C00F07581D5F80CA0BAF1000F00F06F81AB780C202E880093002328
S22401CEC00099324606EB01091FFA89F74A451DDB4BB332464FF6FF774FF00008914542DCB4
S22401CEE0AB794FF6FF78B5F804B00193002301995A465944029102998A4241DB4FF6FF7390
S22401CF00984501D09F424AD1002319E000FB02F11AF80110852908BF3A4602F1010208BF82
S22401CF20012392B2D2E7A9790C27AA8811441FFA81FE8A420ADB002BCBD12278D007C8D4D1
S22401CF4063810020237005B0BDE8F08F07FB02F01AF80000852808BF724602F1010208BF6C
S22401CF60012392B2E5E7114650460AF0E3F8002803DD4045C4BF17468046013292B2ADE777
S22401CF801146504603930AF0D5F8039B002803DD9842C4BF90460346013292B2ABE7BE4216
S22401CFA04CD84F454ADA3B46009A3146504607F09DF98146C34544D8029B984541DA4346D1
S22401CFC0019A5946504607F091F9484480B2237813F0010205D020B1B4F80A904844C0F370
S22401CFE04E006B89608183424FF00003A9D8DFF8A89102B9012389F80C3099F80C30002BDC
S22401D00061D195F8099019F0030302931BD13B46009A3146284603F073FC4346019A5946FD
S22401D0206080284603F06CFCE0806E7A618816F0100667D0002007F0D5FD64E04FF0000948
S22401D040B8E70020C3E731463B46009A284603F057FC4346019A5946B4F80290B4F806A0C8
S22401D0600646284603F04CFC029909EB0602012992B20AEB00039BB212D102EB460203EB65
S22401D080400392B2B1459BB217D2023292B2824516D202339BB292089B086280E380C4E701
S22401D0A0029902290BBF520002EB49025B0003EB4A030CBF92B292B2E4E7E8D9013AE5E7D4
S22401D0C0E9D9013BE6E73B46009A3146284603F017FC4346019A59466080284603F010FC69
S22401D0E06388A380E0802081A9F80030A9F80230A9F804308123A9F80600A9F80800A9F80D
S22401D1000A001EE70846A288237890421ED2190703D4297A121A8A4212DD8B27A080E18869
S22401D12006BB084623892278984224D2960603D4297A1B1A8B4219DD208147F0220300E7D2
S22401D14003F0040363F07E03DFB2E8E75F0703D4297A821A8A4202DDA0808727DFE703F0ED
S22401D1600803EFE7012007F03DFDDBE702F0100242EA0703E5E6D10603D4297AC31A8B42B4
S22401D18003DD208147F01203DBE602F02002EFE70220D8E60B20D6E6123F0020B64B1B7845
S22401D1A0012B00D07047B54B1B688342FAD010B5B24B1860B24B984200D0F8B9B14B1B6B90
S22401D1C013F4803F0AD100EB8003C0EB0313AE4AA2FB0323C3F38F13AA4A1367FA2404FBDB
S22401D1E000F46409A94BA3FB0434C4F3C714204609F05AFA204609F065FA10BD40F2712368
S22401D200984255D040F2D923984260D040F2A93398426BD040F27A43984276D040F24A53D0
S22401D220984200F0818040F21B63984200F08B8040F25373984200F0958040F6F4039842BA
S22401D24000F09F8040F6FD23984200F0A98040F60553984200F0B38040F6DF73984200F093
S22401D260BD80B0F5995F00F0C88041F23273984200F0D28041F61443984200F0DC8042F2BA
S22401D280C613984200F0E78042F6B1039842B4D17C4B1B6B13F4803F03D17A4B40F29B12A8
S22401D2A01A670D2009F000FA0D2009F00BFAA4E7744B1B6B13F4803F02D1724B18221A67BB
S22401D2C0012009F0F1F9012009F0FCF995E76D4B1B6B13F4803F02D16A4B1C221A6701204D
S22401D2E009F0E2F9012009F0EDF986E7654B1B6B13F4803F02D1634B24221A67022009F088
S22401D300D3F9022009F0DEF977E75E4B1B6B13F4803F02D15B4B2D221A67022009F0C4F9D5
S22401D320022009F0CFF968E7564B1B6B13F4803F02D1544B35221A67022009F0B5F9022093
S22401D34009F0C0F959E74F4B1B6B13F4803F02D14C4B3D221A67032009F0A6F9032009F0CE
S22401D360B1F94AE7474B1B6B13F4803F02D1454B4A221A67032009F097F9032009F0A2F93B
S22401D3803BE7404B1B6B13F4803F02D13D4B5A221A67032009F088F9032009F093F92CE7DE
S22401D3A0384B1B6B13F4803F02D1364B6F221A67042009F079F9042009F084F91DE7314B89
S22401D3C01B6B13F4803F02D12E4B83221A67042009F06AF9042009F075F90EE7294B1B6B8F
S22401D3E013F4803F02D1274BA0221A67052009F05BF9052009F066F9FFE6224B1B6B13F40B
S22401D400803F02D11F4BC1221A67072009F04CF9072009F057F9F0E61A4B1B6B13F4803F4A
S22401D42002D1184BEA221A67072009F03DF9072009F048F9E1E6134B1B6B13F4803F03D127
S22401D440104B40F21B121A67092009F02DF9092009F038F9D1E60B4B1B6B13F4803F03D1C3
S22401D460084B40F255121A670B2009F01DF90B2009F028F9C1E600BF164200202C4100204F
S22401D480A086010000600141D34D6210C55A7C0A08B58A4B1B7813F0200F26D0884B1B68E3
S22401D4A0884A12681344B3F5C87F77D2844A1360854B1B68834A12681344B3F5C87F78D220
S22401D4C0814A1360814B1B687E4A12681344B3F5C87F79D27D4A13607D4B1B68794A126824
S22401D4E01344632B7BD87A4A13607A4B1B68754A12681344312B7DD8764A1360764B1B68B7
S22401D500704A12681344312B7FD8734A1360734B1B686C4A12681344312B00F281806F4AC7
S22401D52013606F4B1B68674A12681344312B00F282806B4A13606B4B1B68624A1268134485
S22401D540312B00F28380674A1360674B1B685D4A12681344312B00F28480634A1360634B83
S22401D5601B68584A12681344312B00F285805F4A13605F4B1B68534A12681344312B00F257
S22401D58086805B4A13605B4B1B684E4A12681344312B00F28780574A136008BD484B0022F2
S22401D5A01A60554A137843F001031370FEF740FF7EE7454B00221A604F4A137843F02003C8
S22401D5C01370FEF735FF7DE7404B00221A604A4A137843F010031370FEF72AFF7CE73C4B1E
S22401D5E000221A60444A137843F008031370FEF71FFF7AE7374B00221A603F4A137843F0D6
S22401D60040031370FEF714FF78E7334B00221A60394A137843F080031370FEF709FF76E71C
S22401D6202E4B00221A60354A137843F001031370FEF7FEFE75E72A4B00221A602F4A1378A9
S22401D64043F002031370FEF7F3FE74E7254B00221A602A4A137843F004031370FEF7E8FE25
S22401D66073E7214B00221A60244A137843F008031370FEF7DDFE72E71C4B00221A601F4AF3
S22401D680137843F010031370FEF7D2FE71E7184B00221A60194A137843F020031370FEF758
S22401D6A0C7FE70E7134B00221A60144A137843F040031370FEF7BCFE6FE700BF184200202E
S22401D6C0E040002024410020E4400020E8400020EC400020F8400020FC4000200041002092
S22401D6E004410020084100200C4100201041002014410020184100201C4200201D4200208D
S22401D700F0B58DB07E4B1B88ADF824307D4B1B88ADF826307C4B1B88ADF828307B4B1B8886
S22401D720ADF82A307A4B1B88ADF82C30794B1B88ADF81830784B1B88ADF81A30774B1B886D
S22401D740ADF81C30764B1B88ADF81E30754B1B88ADF82030744B5A7AADF80C201A7BADF885
S22401D7600E20DA7BADF810209A7CADF812205A7DADF814201A7EADF80020DA7EADF8022032
S22401D7809A7FADF8042093F82120ADF8062093F82430ADF808300022644B1A7009A86C4690
S22401D7A00DF12E072146034694464FF0010E01E0BB4209D033F8026B31F8025BAE42F7D9C3
S22401D7C00132D2B2F446F3E7BCF1000F01D0574B1A700023564A1370DDB230F8021B34F879
S22401D7E0022B914273D80133052BF5D10022514B1A7006A803AC0DF1220721460346944658
S22401D8004FF0010E04E04A4B1D70EFE7BB4209D033F8026B31F8025BAE42F7D90132D2B26D
S22401D820F446F3E7BCF1000F01D0424B1A700023414A1370DDB230F8021B34F8022B9142F9
S22401D8402BD80133052BF5D1384B1B78042B1FD8374A12789A4204D000201AE0364B1D7076
S22401D860F2E7344B1B78042B15D8334A12789A4201D000200DE0314B1B78012B01D00020AE
S22401D88007E02F4B1878032894BF0020012000E000200DB0F0BD0020FBE7042DD4D86A1C03
S22401D8A0D2B2520006AB991803AB1A44C5F10505EDB200230133DBB2AB42CFD031F8024BD9
S22401D8C032F8020B8442F5D81B4A1370BCE7042D8CD86A1CD2B2520009AB99186A44C5F133
S22401D8E00505EDB200230133DBB2AB428BD031F8024B32F8020B8442F5D80D4A137075E7D7
S22401D9009C4100209E410020A0410020A2410020A4410020A6410020A8410020AA410020E1
S22401D920AC410020AE4100205C3C00202A4200202D4200202B4200202C4200203242002043
S22401D9405242002030B591EA030F00F18280841A71EB030C05D2121953EB0C03001B71EBD9
S22401D9600C0140F2000CCFF6E07C1CEA430F52D0BCEB410F5FD90C0DA4EB135E5FF0010C17
S22401D9806CF31F516CF31F53DEF1200C2AD303FA0CF5401941F1000122FA0EF5401923FACA
S22401D9A00EF5694112FA0CF2CD0208D349085FEA30005FEA320228BF42F001020134013C2B
S22401D9C05FEA500C72F1004250F1000051EB04514FF4001313EB410F38BF30BD090D090579
S22401D9E0002030BDBEF1200EBEF1200F1ED223FA0EF5401941F10001CEF1200C124218BFA7
S22401DA00012203FA0CF52A43CEE711EA5C0F04BF0020002130BD1CEA410F04BF01F000411B
S22401DA20002030BD01F00041002030BD21F4801101EB045130BD004218BF41F00101BCEBCD
S22401DA40410F08BF30BD4FF0FE4141F47801002030BD83F00043841A71EB030E07D28EF06B
S22401DA60004E001B71EB0E01121953EB0E0340F2000CCFF6E07C1CEA430FC6D0BCEB410F0E
S22401DA8072D90C0DA4EB135EC90241EA5051C00241F00041DB0243EA5253D20243F0004358
S22401DAA0DEF1200C41D312FA0CF522FA0EF203FA0CF542EA050218BF42F0010223FA0EF3CD
S22401DAC0801A9941E30AC4F30A0411F0404F03D418D0013C40004941013C23D44205C00A7F
S22401DAE040EA4150C90A51EAC3715FEA500C72F1004250F1000051EB045130BD01002FD01A
S22401DB000020203C0029F9D0B1FA81FCDCF1200E11FA0CF130FA0EF510FA0CF02943A4EB38
S22401DB200C04D9E70020D90730BDAEF1200EBEF1200F0DD2CEF1200C03FA0CF533FA0EF381
S22401DB402A4318BF43F00103C01A61F10001B9E721F00041C00A40EA4150C90A01EB04518C
S22401DB6030BD0020002130BD004218BF41F00101BCEB410F7FF467AFBCEB430F3FF463AF7A
S22401DB8030BD00BF006A70472DE9F04F59EC118B2DED028BC9F30A51013940F2FD70814222
S22401DBA083B011EE104A4D465BEC10AB64D8CBF30A51013981425E465ED82BF000438DED3A
S22401DBC0000A0193204625F00041DDE9002307F025FC70B152465B464046494600F0BEFCCB
S22401DBE021F0004319466EA3D3E9002307F016FC70BB42464B465046594600F0AFFC41EC32
S22401DC00100B00F055FE4046494600220023B0EE408AF0EE608A07F001FC40B9B0EE480A39
S22401DC20F0EE680A03B0BDEC028BBDE8F08F0022002351EC180B07F0D5FBC8B15AA3D3E9E3
S22401DC40002351EC180BFFF77DFE41EC180BE5E749A3D3E9002306F0004646F07F5343F468
S22401DC60641343F4075343F03B0343EC182BD5E74FA3D3E90023E4E72219414945EB05035E
S22401DC800020994208BF90423BD31AEB0A0300934BEB0B030193DDE90023994208BF904202
S22401DCA05E464BD32BF00043CDF800A00193DDE90023344900208B4208BF824230D0002245
S22401DCC000235046594607F097FCE8B92D4B00229D4208BF94424BD02B4B00229D4208BF4C
S22401DCE0944213D0002200234046494607F084FC00283FF467AF20A3D3E900230BF0004640
S22401DD00ABE749EC188B89E7E80F31D01F48204906F00046024686EA010343EC182B7DE78D
S22401DD20194625F0004310468B4208BF84420BF0004606D010A3D3E900238EE74BEC18AB5E
S22401DD406CE7494600220023404607F067FB114F1149124D0D4C002808BF39464FF0000296
S22401DD6081EA060314BF2A46224643EC182B55E70146CDE7AFF30080182D445400000000D6
S22401DD800000E0FF0000F07F0000F0FF182D4454FB210940FB21E93F7CD90240D221337F7E
S22401DDA02342920CA19CC73B182D4454FB2109C0182D4454FB2109402DE9F04F85B0664BDC
S22401DDC0B3F800A0654BB3F800B0654BB3F80090644BB3F80080644B1F88644B1E88644BC8
S22401DDE01D88644B1B880193634B1B880293634B1B880393624B1B78FF2B07D0614B1A8836
S22401DE00614B1A80614B1A88614B1A80614B1B78022B02D95F4B00221A7009F0C1FD044684
S22401DE2009F0E2FD052830D15B4B1C885B4B1C8007EE904AB8EE677ADFED597A87EE270AAF
S22401DE40584B83ED000A012002F0E4FB564B1878002854D14E4B1B8807EE903AF8EE677A6D
S22401DE60DFED4F6A87EEA67AB4EEC07AF1EE10FA21DB00234D4A13704D4A1370464B1C803D
S22401DE80444B187005B0BDE8F08F09F0ADFD0428CAD014F4006F0CBFC4F30B0400243E4B6E
S22401DEA01A88A31A002BB8BF5B4240F674118B42C8BF1446BAE7B4EEC07AF1EE10FA17D800
S22401DEC0314B1B8807EE903AF8EE677ADFED346A87EEA67AB4EEC07AF1EE10FA08DD334B70
S22401DEE01B78012B0CBF02200120314B1870C5E72E4B01221A7002202D4B1870BEE70AEBBD
S22401DF000B034B4443443B4433442B44019A1A441346029A1A441346039A1A4493B2642BFE
S22401DF2005D80020214B1870214B1870A6E7643B9BB2632B08D81D4B1B78012B0CBF0220FB
S22401DF4001201B4B187099E7184B01221A700220174B187092E700BF9C4100209E410020DC
S22401DF60A0410020A2410020A4410020A6410020A8410020AA410020AC410020AE4100205B
S22401DF8052420020C0410020CA410020C2410020CC41002054420020CE410020BE41002027
S22401DFA000007243484100200D420020554200204B42002008B5A0F5805001385A2800F25B
S22401DFC0E280DFE800F03734312E3AC7C4C0BDBAB7B4B1AEABA7A49E9B9895A18E8B92D614
S22401DFE0D3D0CDCAD98885827F7C7975726F6C6966605C595653504D63E0E0E0E0E0E0E096
S22401E000E0E0E0E0E0E0E0E0E0E0E0E0E0E0E0E0E0E0E0E0E0E0E0E0E0E0E04743403D4A09
S22401E020DD0009F001FA08BD09F006FAFBE709F00BFAF8E709F010FAF5E709F015FAF2E7CC
S22401E04009F01AFAEFE709F01FFAECE74F4B1878C009E8E709F020FAE5E709F025FAE2E770
S22401E06009F02AFADFE709F02FFADCE709F034FAD9E709F039FAD6E709F03EFAD3E7444B88
S22401E0801878C009CFE709F03FFACCE709F044FAC9E709F049FAC6E709F04EFAC3E709F0D2
S22401E0A053FAC0E709F058FABDE709F05DFABAE7384B1878C009B6E709F05EFAB3E709F029
S22401E0C063FAB0E709F068FAADE709F06DFAAAE709F072FAA7E709F077FAA4E709F07CFA0F
S22401E0E0A1E72D4B1878C0099DE709F07DFA9AE709F082FA97E709F087FA94E709F08CFAE5
S22401E10091E709F091FA8EE709F096FA8BE709F09BFA88E7214B1878C00984E709F09CFAD1
S22401E12081E709F0A1FA7EE709F0A6FA7BE709F0ABFA78E709F0B0FA75E709F0B5FA72E780
S22401E14009F0BAFA6FE7164B1878C0096BE709F0BBFA68E709F0C0FA65E709F0C5FA62E7AD
S22401E16009F0CAFA5FE709F0CFFA5CE709F0D4FA59E709F0D9FA56E70A4B1878C00952E79A
S22401E18009F0DAFA4FE700204DE700BF1F42002020420020214200202242002023420020D4
S22401E1A024420020254200202DE9F7430025714C294609F011FB704FA946A846238865F307
S22401E1C04103238009F008FB0C2509F005FB3B685B6845432B445B68A36209F0FDFA3E6871
S22401E1E073685A195B59636206235843B3681C181E5CA488B60744BF05261E541B5C5F4E18
S22401E20013F01C0F11BF44F47C14907A5C4B03EB1013107A01BF1B7A63F313441B0963F36A
S22401E220155409F0D9FA534B3A289BBF0430DA7ADA7A60F3050288BF42F03F02DA7209F014
S22401E240CBFA4C4BDC6109F0C7FA3B6872685B682B44DB7A12B1042B28BF0423454C63F37A
S22401E2600308022363F3C409042363F30A2909F0B3FAA4F8069009F0AFFA6FF3061884F81F
S22401E2800A804FF000083B685B682B44587A000909F0A2FAA36960F31653A3613B685B6830
S22401E2A01D446B7A63F30A2141F040016FF3C71141F4004141F0040109F08EFA072389B253
S22401E2C0218084F82E3009F087FA238843F00203238086F8088009F07FFA7368002B38D037
S22401E2E009F07AFAE07A00F03F0009F075FAA169C1F3032109F070FA278809F06DFA2388BB
S22401E300C7F3022768F34103238009F065FAA57809F062FA45F01205EDB2A57009F05CFAB9
S22401E320184BA57A1A68EDB2137843F00803137009F052FAA37A3A4668F30303A372124B33
S22401E34000957568A84709F047FA238843F00203238009F041FA074A237D43F002032375A1
S22401E36092F82F30DB0702D4337A012BF8D103B0BDE8F083001C004318000020BC3D0020D9
S22401E380E45A0200100000200A1C004338B5044609F030FB614B1B7813F0100F51D0B0F51C
S22401E3A0E46F53D040F2FF73984200F08180302802D05B4B1B7848E00221204609F020FB4A
S22401E3C0C0F3C710574B18700221204609F018FBC0F38010544B18700021204609F010FBF9
S22401E3E0C0F34010514B18700021204609F008FBC0F387104E4B18700021204609F000FB87
S22401E400C0F300104B4B18700021204609F0F8FA00F00F00484B18700521204609F0F0FA1A
S22401E420C0F38000454B1870454B00221A600521204609F0E5FAC0F3C000424B187009F07A
S22401E44032FB374B1B78002B64D038BD0021204609F0D6FA3C4D28700121204609F0D0FA64
S22401E46068700221204609F0CBFAA8700321204609F0C6FAE8700421204609F0C1FA2871EC
S22401E4800521204609F0BCFA68710621204609F0B7FAA8710721204609F0B2FAE8712B4B10
S22401E4A008221A702A4A137843F001031370C8E70021204609F0A4FA264D28700121204689
S22401E4C009F09EFA68700221204609F099FAA8700321204609F094FAE8700421204609F0B3
S22401E4E08FFA28710521204609F08AFA68710621204609F085FAA8710721204609F080FAF3
S22401E500E871154B08221A70114A137843F00203137096E7024B01221A7096E71842002079
S22401E5201E420020F0410020EC410020E8410020E4410020E0410020DC410020D841002072
S22401E54020410020D44100200440002019420020274200200C4000201A4200202DE9F04366
S22401E56091EA030E0EF0004E40F20007CFF6E07717EA41051EBFBD4217EA4305BD4200F00D
S22401E5809F807F0D17EA135623EA475343F4801317EA115521EA475141F48011AD1B05F260
S22401E5A0FD354FEAD31C1CF1010C4FF00047B7FBFCF77F01A2FB079C0024E3FB07C4D9F15F
S22401E5C000096CEB4C0CA0FB07620020E1FB072000275FEAC628E0FB0987760D46EAC226F2
S22401E5E0520DF61900277A41E0FB0C625FEAC823E2FB09375FEA585848EAC628760D18EB8C
S22401E600070800214E41E2FB0C8602EBC020DA02E6FB09215B0D43EAC8235FEA58585B1826
S22401E620002758EB0708E6FB0C38D102E8FB0917520D42EAC3225B0DD21900277B41E8FBD7
S22401E6400C2308EBC6265FEAC128E3FB0987490D41EAC221520DC91942F10002E3FB0C1230
S22401E660470019EB08095CEB010C72EB040453EBC62047EB56530026B3F5000F7641AD1926
S22401E6800236D6F1200910FA09F4F04013FA09F21043F340E40F001943F10003B3F5001F7D
S22401E6A024BF5B08013540F2FE77BD4204D24EEA05511944BDE8F0832D4224D5714626E034
S22401E6C0004218BF41F00101124218BF43F00103B7EB410F2CBFB7EB430F1BE0B7EB410FC8
S22401E6E004BFB7EB430F15E017EA410F04BF17EA430F0FE017EA410FE0D017EA430F02D0EC
S22401E700B7EB430FDAD04EF0FE4141F470010020BDE8F08340F20001C7F6F871F7E700BF04
S22401E720F8B5002006F077F806F0D0FD032008F03FFA09F005F90130524B18600021524892
S22401E74009F004F908F086FB08F026FA00224F49104607F047FF00214D4808F0FDFC4D48A3
S22401E76003F0E6F9002003F089F903F09DFF03F02DFD06F00DFF08F03FFC02F03DF907F02C
S22401E78063FC08F0A9F90021434809F0BBF84FF4C051062007F092FC08F0AAF904F0B8FDDF
S22401E7A008F0D6F908F0E0F9002007F07DFF002007F088FF07F008FB002003F091FE07F0F7
S22401E7C01FFD02F029FD05F0B9F9344C08221146204609F09DF800224FF40051204609F04E
S22401E7E097F82F4C0122214640F2837006F0CAFA2378012B01D9012222702A4B01221A7028
S22401E80000241F46284E294D2CE007F02DFB06F003FD3B78012B0AD03B78032B10D103F0EE
S22401E82075FD00221821012008F06AFA1DE0FBF7AFF900F0A5FC04F063F8FCF757FBEBE7FA
S22401E840002007F095FC08F09FFC06F083F9E6E706F020FF286008F0B7F9FDF7D7FF07F032
S22401E86075FE013414F0010FCFD0A6FB04239B0803EB83039C42EBD100F03AFD07F016FE8C
S22401E880E6E700BF4C410020C977020095420200357A0200C0260020A53E020000800041C1
S22401E8A05E42002016420020CDCCCCCC644100202DE9F04759EC108B594F18EB080029F02B
S22401E8C0004343EB030100268F4208BF864282B0C0F0848053490020994208BF404510EE70
S22401E8E0102ACA467DD310EE104A1D460127002643A1D1E900019042994126DA42A3D3E983
S22401E90000232046294601F095F90022464B09F0BBF80022444B09F0B7F822462B46FFF7F3
S22401E92011F83BA3D3E900238046894620462946FFF708F802460B4640464946FFF70EFEFB
S22401E9403E4604460D4602460B460FF2CC09D9E9008923F00041894508BF904527D22246B7
S22401E9602B462046294601F065F902460B46804689462E48042106F059F94246CDE90001AC
S22401E9804B4604212A4806F051F802460B46DDE90001FFF7E3FD22462B4601F04BF902467E
S22401E9A00B4620462946FEF7CDFF04460D46012E22DD05F100431D461E4B03EBC60620467A
S22401E9C02946D6E90023FEF7BDFF04460D460AF0004A22468AEA050343EC102B02B0BDE8A9
S22401E9E0F08700200F49FFF7B9FD032704460D4602460B4602267BE7002EE8D0DCE700BF24
S22401EA0058CD9E5E1426D13F5499B0D0F56CE73FAA4C58E87AB6FB3FBBBDD7D9DF7CDB3D56
S22401EA200000E0FF0000F03F0000E03F283F0200483F0200083F020038B55C4A682303FB4C
S22401EA4000235A8A5B6D934217D900EB8003584A02EB83035B7B042B4AD000EB8002544B6E
S22401EA6003EB820303225A73504A682303FB0020002343650123437038BD00EB80034C4A4D
S22401EA8002EB83035B7B052B12D0042B30D0474A682303FB002393F82830012B18D9022B7C
S22401EAA036D0424A682303FB002002234370E3E700EB80023E4B03EB820303225A733B4A93
S22401EAC0682303FB00200023436501234370D3E700EB8002364B03EB820303225A73334A5B
S22401EAE0682303FB00200023436501234370C3E700EB80022E4B03EB820302225A732B4A5C
S22401EB00682303FB00200023436501234370B3E70446264A682303FB00231B7E5BB31146A6
S22401EB20682202FB0012D18C5A1E91420DDB1F49682202FB0012958C00EB80021C4901EBC6
S22401EB4082025289073A954224DB1849682202FB0412D28C013B9A420DDB144A682303FBF6
S22401EB600423998C04EB8403114A02EB83035B89073B994295DB204603F04AFD0B4A68230E
S22401EB8003FB0424E38C0133E384002363650223637071E707F0FEFA044A682303FB042416
S22401EBA0002363650323637066E700BF6C390020AC26002008B55A4B9B7D002B58D0584A39
S22401EBC0536803F00703127E12F0040F62D0544A906A544A5169D26891425BD2002B48D132
S22401EBE0504B59685A6988545A6901325A614C4B1B7E13F0010F1AD0494B01221A75494B5C
S22401EC009A699B689A425FD2464B19689A69895C434A91629A6901329A61424B9A699B689D
S22401EC209A426AD03F4B5A69DB689A4272D03C4B1B7E13F0020F15D03B4B1B78C3B1394BE0
S22401EC405A69DB689A4210D1364B00221A7734490720087534490A701B6A4BB1314B1A6A1E
S22401EC60586A9047304B1B7813B12D4B02229A7508BD2C4B5A68596922F811005A69013297
S22401EC805A61274B1B7E13F0010FD0D0244B01221A7509E0224A127E12F0010FC7D0204ADC
S22401ECA001211175002BAAD01E4B9A699B689A4216D21C4B1A68996932F81110184A916243
S22401ECC09A6901329A61A8E7164B1B69002BA4D0134BFF229A62134A1369013B13619CE763
S22401ECE0104B1B69002B98D00D4B4FF6FF729A620C4A1369013B13618FE70A4B1B69002B96
S22401ED0090D1094B01221A70054B1B7E13F0020F95D1AAE7024B01229A7504221A7586E7F6
S22401ED2000300040B83C0020251000205A4B9B7D002B00F0B08010B5574B5B8B13F0020F8B
S22401ED4019D0564B022283F82120544B002283F82020514A536843F440335360D369002BAD
S22401ED60FCD14D4B83221A764C4B5B6A43B34B4A906A984724E0484B5B8B13F0010F04D0CF
S22401ED80464B022283F82120DFE7434B5B8B13F0040F04D0414B012283F82120D5E73F4B27
S22401EDA093F92030032B56D0042B19D0022B08D03A4B93F92030B3F1FF3FC6D0062B3AD0EC
S22401EDC010BD364B1B692BB10021344B988806F091FCEDE70121314B988806F08BFCE7E75F
S22401EDE02E4A9369126993420BD02C4A9168581C9061CA5C284B9A621A46D369002BFCD171
S22401EE00DEE7264B5B6973B1244B9B885B0043F00103214A5362D369002BFCD11F4B0322C7
S22401EE2083F82020CCE71C4A536843F440335360D369002BFCD1194B002283F8202083F8F0
S22401EE402120154A832111765B6A002BB8D0134A906A9847B4E7114A5369013BD2699A422E
S22401EE600CD00D4AD369002BFCD10B4B986A0B4BD968DA69541CDC61885499E7064A5368DF
S22401EE8043F4E0235360D369002BFCD1034B062283F82020E5E77047003400408C3C00203B
S22401EEA008B5534B1B78012B2ED008F06DFD012839D04F4B1B78012B03D14E4B1B78782BA4
S22401EEC041D008F061FD4C4B1B78012B4CD04B4B5B7B012B57D0464A1278002A7DD1022BD5
S22401EEE058D0474B1A6842F20F739A426CD8434B1B7B022B77D106F091FE414B00221A60B4
S22401EF00404B01221A7071E03A4B18787828CCD03A4B1B7B13F0FD0FC7D101F077FA364B6C
S22401EF2001221A70C1E7344B1B78012BC1D1334B1B7B13F0FD0FBCD1314B00221A60314B62
S22401EF4001221A7052E02D4B1B7B13F0FD0FB8D1782001F05BFA00232B4A1370284A136048
S22401EF60284B04221A7041E0244B1B7B23F00203184310F0FF0FAAD1214B00221A60214BD2
S22401EF8001221A7032E01E4B00221A601D4B02221A702BE0FDF7ECFD174B00221A70174B39
S22401EFA05B7B022B04BF154B5A73184B5B79022B06D0134B00221A60124B03221A7015E023
S22401EFC0124B00225A71F4E706F028FE0C4B00221A600C4B01221A7008E0094B1A6842F201
S22401EFE00F739A42F0D8074B03221A7008BD00BFED410020F141002004420020AC26002068
S22401F000C0400020F941002003420020F43F00202DE9F04F95B08146282200210DEB0200F2
S22401F02008F0EAFBB9F1010F40F08880002309930124009409AB0AAA28214C4807F02BF824
S22401F0400590224620214A4806F004FA82462823013BFDD1474B039320230793444B06939C
S22401F0604FF02808414B0493DFF80CB15D46002403E001341835162C21D028890028F8D064
S22401F080AF7C17F0400FF4D14246049906F092FB0028EED117F0020FEBD004EB44010BEB98
S22401F0A0C10107F0D1F80028E3D104EB4403324A02EBC3031A7D42F010021A75D9E74A46CD
S22401F0C04146039806F043FE2C4C04F1800500264B4681461F460AE0019600974346039ABE
S22401F0E02146304602F066F90834AC4203D02388002BF9D0F0E73B464F4699460093434658
S22401F100049A0799069808F0CCFC002818BF4FF0010A059B33B94FB9BAF1000F0AD115B016
S22401F120BDE8F08F484607F08BFDF4E7484607F09FFDF1E7484607F08FFDF0E7002409941B
S22401F140CDF8009009AB0AAA2146204606F0A3FF05904A462146204606F07CF982460394CB
S22401F16007940694A04604947EE700BF542F0020AC2300209C300020842B00206C380020A1
S22401F18010B582B0544B1B78072B00F28880DFE803F036041C48637E8659504C00224FF4FB
S22401F1A00051204608F0B4FB00224FF00071204608F0AEFB002003F0B1FF474B02221A700F
S22401F1C0474B00221A8002B010BD454B1B885A1C92B2092B02D9434901200870023340497D
S22401F1E00B80092AEFD9404A137803F0FD031370022007F0EBF8384B00221A70E3E70022E1
S22401F2004FF00071354808F083FB01A806F052FC0128D8D1354B019A1A602F4B03221A70C8
S22401F220D1E7324B187803F079FF4FF4005211462A4808F06DFB284B07221A70284B00221F
S22401F2401A80C0E7264A1388591C1180092BBAD9214B04221A70B6E70121022005F00CFC95
S22401F26000224FF000711D4808F052FB1E4A137843F0020313701D4B1978012007F0D0FE7F
S22401F280174B00221A80144B05221A709BE7144B1B88DE2B97D9104B06221A7093E7002195
S22401F2A0022007F0BDFE002003F038FF0B4C00224FF00071204608F02BFB00224FF40051C7
S22401F2C0204608F025FB0023034A1370044A1380022007F07BF876E7414200200080004189
S22401F2E0B841002042420020002400433841002008B5534B1A78002A0CBF012200221A709A
S22401F3000CD1504B5A88504B1A80504B1B78022B3ED0032B64D0012B0CD008BD04F046FB8B
S22401F32007F0DAFB4FF4C051062006F0C7FE07F0DFFBF2E7464B00221A80424B1A88A2F20C
S22401F34046239BB2B3F58C7F04D3A2F2FD639BB2E02B0BD83F4A138801339BB21380B3F558
S22401F360C87FDAD3394B02221A70D6E7A2F2452292B240F299539A42CFD9374A1388013373
S22401F3809BB21380632BC8D9304B03221A70C4E7304B00221A802B4B1B88A3F2823292B2A6
S22401F3A0B2F5567F0AD22A4A138801339BB21380312BB2D9254B01221A70AEE7A3F2452336
S22401F3C09BB240F299529342A7D9234A138801339BB21380632BA0D91C4B03221A709CE7AC
S22401F3E01D4B00221A80174B1A88A2F267239BB2B3F58D7F04D3A2F2DB639BB2DF2B0BD8DD
S22401F400144A138801339BB21380B3F5C87F84D30E4B02221A7080E7A2F2823292B2B2F5F2
S22401F420567FBFF47AAF0A4A138801339BB21380312B7FF672AF054B01221A706DE700BF10
S22401F4401742002058410020D641002016420020DA410020DE410020E241002030B40D46D1
S22401F460002956D0002854D053490C7F04F0FF01002C40F09E80514C646804F00704012CC1
S22401F4804DD04D4908604A6000244C618C610C6100284ED08D60002A4FD0474AD360464AA6
S22401F4A001211177454A127E12F0040F05D0434A916A117E11F0040FFAD1404A518B41F006
S22401F4C004015183117E41F0800111763A4AD1689268914204D9384AD1689068091A1161D6
S22401F4E0364A526812F0070F37D1334A91699268914226D2304A11680878304988629169A0
S22401F50001319161002B4CD02C4B04229A7501214CE0002B49D0002AA6D1002146E015B18E
S22401F52015F0010F42D1002BABD013F0010FA8D03CE0214900208860ADE71F4A0021D1608F
S22401F540ADE71D4A1269002ADCD01C4AFF21916219490A69013A0A61D4E7174A91684908FF
S22401F5609160116949081161D1684908D16091699268914208D2104A116808880F49886256
S22401F580916901319161BDE70B4A1269002AB9D00A4A4FF6FF71916207490A69013A0A61BB
S22401F5A0B0E70121054B997500E00021084630BC70470021FAE700BFB83C002000300040F7
S22401F5C010B50446554A682303FB002393F84A1006F0A8FB01281ED0504A682303FB0423EC
S22401F5E093F84A30032B60D004EB84034C4A02EB83035B7B042B07D0484A682303FB042305
S22401F60093F82830012B79D9444A682303FB04240323637010BD414A682303FB042393F8B8
S22401F6202830032B38D03D4A682303FB042393F84A30032B39D0394A682303FB042393F805
S22401F6402830022BD0D1682303FB04231B7E012B3BD0324A682303FB04231B7E012B0DD12F
S22401F6602E4A682303FB0423998C04EB84032C4A02EB83035B89073B9942C5DB204602F0DF
S22401F680C7FF264A682303FB04240123E3840023636502236370BDE7682303FB0424002397
S22401F6A0E384636502236370B4E704EB84021C4B03EB820303225A73184A682303FB04242E
S22401F6C00023636501236370A4E7682303FB0423998C04EB8403124A02EB83035B89073B77
S22401F6E09942B6DA204606F055FD0C4A682303FB042400236365032363708BE704EB840219
S22401F700074B03EB820303225A73044A682303FB042400236365012363707BE76C39002024
S22401F720AC260020F8B50446524A682303FB002393F8401006F0F6FA01282DD04D4A682389
S22401F74003FB0423002283F83C201A66204606F07DFE484A682303FB042393F83C301BBB1F
S22401F760682303FB042393F84030032B1ED104EB8402414B03EB820302221A730022DA7327
S22401F7803C49682303FB04F40B1983F82020DA651A6601230B550FE0364A682303FB04231C
S22401F7A0012283F83C20D1E7012B06D0682303FB04F4304B03221A55F8BD012819D0002810
S22401F7C0F4D12C4A682303FB0423DB7E9BB31146682202FB0412D27F9A421DD3682303FBF7
S22401F7E004F40B1900229A77DA651A6602230B55E2E704EB8402204B03EB820300221A73A5
S22401F8001C49682303FB04F40B1983F82020DA651A6601230B55CFE7164A682303FB042314
S22401F8201A7F01321B6E9342C0D3124A682303FB0423DB7F0DE00F4A682303FB04231A7F10
S22401F84001321B6E9342B1D30A4A682303FB0423DB7F084F682505FB04F57E190133F3771D
S22401F860204600F055FF0023F365336603237B55A2E700BF6C390020AC26002038B5044698
S22401F880514A682303FB002393F832302BB34E4A682303FB04239B7F012B21D0002B6FD166
S22401F8A0494A682303FB04239A8ADB6D934267D304EB8402454B03EB820302221A73002239
S22401F8C0DA734149682303FB04F40B1983F82020DA651A6601230B5558E004F099F8D6E72E
S22401F8E0682303FB04239B7E012B1CD0364A682303FB04239B7E012B57D9334D682202FB75
S22401F90004F2A91800238B7704EB84042F4800EB840402202073E37381F82030CB650B662F
S22401F9200123AB5432E0682303FB042393F820205B7E93422BD92448682303FB04F4031956
S22401F94000219977013283F82020D9651966022303551BE01C4D682202FB04F2A918002383
S22401F9608B7704EB8404194800EB840402202073E37381F82030CB650B660123AB5405E0B7
S22401F980682303FB04F4104B02221A5538BD0E4A682303FB042393F820205B7E9A42D9D2CA
S22401F9A0094A682303FB04239B7E002BE8D1064A682303FB04F413190121D9770021D96573
S22401F9C0196603231355E1E76C390020AC26002000B1704710B584B0484C0DF1070202A9EE
S22401F9E0E08803F00FFAA37B012B07D09DF80730003318BF01235BB904B010BDE37B012B63
S22401FA00F4D19DF80730082B14BF00230123F2E79DF808301B09032BEED8DFE803F0021771
S22401FA203459364A002382F828300DF1070329320DF10F0013F8011F02F8011B8342F9D17E
S22401FA409DF807202D4B83F83120D5E79DF80730082B04D0294B032283F82820CCE7274A91
S22401FA60012382F828300DF1070329320DF10F0013F8011F02F8011B8342F9D11F4B0822B6
S22401FA8083F83120B8E79DF80740082C0DD01B4B9A8C631E12FA83F3194A5289934204DA88
S22401FAA0164B032283F82820A6E7144A022382F828300DF1070329320DF10F0013F8011F7A
S22401FAC002F8011B8342F9D10C4B83F8314093E70A4A002382F832300DF1070333320DF100
S22401FAE00F0013F8011F02F8011B8342F9D19DF80720024B83F83B207EE700BF6C39002059
S22401FB00AC26002030B4474B474A1A60474A1A61012283F8402083F8412083F84220002188
S22401FB2083F8431083F8442083F8452083F8462083F8472083F8482083F8492083F84A10D3
S22401FB4083F84B20032483F84C4083F84D1083F8502083F8512083F8522083F8532083F886
S22401FB60542083F8552083F8562083F8572083F85910332083F8300083F83120412083F8AE
S22401FB803200142083F83300222083F83400202083F8350083F83610112083F8380083F84A
S22401FBA0390083F83A0083F83B0083F83C10204DC3F8805083F8C04083F8C12083F8C220A8
S22401FBC083F8C34083F8C42083F8C52083F8C62083F8C72083F8C82083F8C92083F8CA20F3
S22401FBE083F8CC2083F8CD2083F8CE1083F8CF1083F8DE2083F8DF4083F8B00083F8B10013
S22401FC0083F8B20083F8B30083F8B400052283F8B520772283F8B62083F8B71083F8BF1067
S22401FC2030BC704700800041CC2400020004000204C00040F0B540F2FF7681EA030C16EA98
S22401FC40115E1EBFB64516EA1355B54252D021EA465141F48011A1FB024723EA465343F4AC
S22401FC608013AE44A0FB03650CF0004C36197D41A1FB034747F10003A0FB0217F619654117
S22401FC8053F10003094218BF46F0010640F2FE74B3F5007F13D2AEF5806EA64523D24CEA61
S22401FCA00331280341EA155140EA16503203450872F1004250F1000051EB0E51F0BDAEF26E
S22401FCC0FF3EA6450FD24CEAC321E80241EA555140EA5650F202450872F1004250F1000049
S22401FCE051EB0E51F0BD1EEA0E0F2DD50CF000410020F0BD16EA115F04BF01F00041002000
S22401FD00004218BF41F0010116EA135F04BF03F000430022124218BF43F0010306EA13544B
S22401FD20B44218BFB64503D00CF000410020F0BD21F0004123F00043B1EB065F0CD8B3EBED
S22401FD40065F09D841B13BB10CF0004141F0FE4141F470010020F0BD40F20001C7F6F87100
S22401FD600020F0BD2DE9F04101224249424C434822720668B1F8403020889BB226F8103034
S22401FD80072081F82E0008886FF3410008803C48278801684D680C2101FB0751C97A042992
S22401FDA01DD96568DDB1257D04391544C9B2EDB22575A5691D44A56194F814E002FA01F519
S22401FDC0AE450ED1A56925FA01F126F817102D490978012907D0022924D0BDE8F08126F89C
S22401FDE017300022F3E70168238848680C2101FB0301C97A042905D9616819B122B10022F3
S22401FE00A26122750133238005F024FA30B92088FEF7CAF904236372BDE8F081E368BDE80D
S22401FE20F041184706680C252188726805FB0125AA7A02F00F00EA7A0625042A28BF0422F5
S22401FE40904238BF121AB0682CBF0022D2B205FB01010D4D13412D6898B24A88AD79561B06
S22401FE60B04202DD2A44904202DB4B80236998470223D0E7001C0043BC3D00201C000020C8
S22401FE8018000020604200201400002070B5404CA479032C02D00024204670BD801AC91A2B
S22401FEA080EAE075A5EBE075ADB281EAE173A3EBE1739EB21E2D01D82F2E62D907EE901AED
S22401FEC0F8EEE70A07EE900AB8EEE70A04F010FBDFED307AB4EEE70AF1EE10FA0BDBDFED7C
S22401FEE02E7AB4EEE70AF1EE10FA04D55A2D8CBF08240724D0E7DFED287AB4EEE70AF1EE3F
S22401FF0010FA0BDBDFED257AB4EEE70AF1EE10FA04D58C2E8CBF02240124BDE7DFED207AD1
S22401FF20B4EEE70AF1EE10FA0ADBDFED1A7AB4EEE70AF1EE10FA03D58D2E28BF0424ABE74A
S22401FF40DFED167AB4EEE70AF1EE10FA06DBDFED157AB4EEE70AF1EE10FA0DD9DFED127ACD
S22401FF60B4EEE70AF1EE10FA0DDBDFED0D7AB4EEE70AF1EE10FA08D55A2D8CBF0624052446
S22401FF808AE7002488E7002486E7002484E700BFF43E0020000034C2000034420000074370
S22401FFA0000007C300003443000034C310B5344B1B88C72B45D8334B1B88C72B41D8324B64
S22401FFC01B88C72B3DD8314B1B88C72B39D8304B1B88C72B35D82F4B1B88C72B31D82E4BA1
S22401FFE01B88B3F5967F2CD22C4B1B88B3F5967F27D22B4B1B88B3F5967F22D2294B1B88EC
S224020000B3F5967F1DD2284B1B88B3F5967F18D2264B1B88B3F5967F13D2254B1B88B3F5FF
S224020020967F0ED2234B1B88B3F5967F09D2224B1B88B3F5967F04D2204B1B88B3F5967FAD
S2240200400FD31F4901230B7041F20300FAF7E0FA1C4B1B8801339BB2C82B0CD8194A138057
S22402006010BD174900240C7041F20300FAF7D0FA144B1C80F4E7134B00221A80F0E700BF35
S22402008096410020984100209A410020B0410020B2410020B44100209C4100209E41002039
S2240200A0A0410020A2410020A4410020A6410020A8410020AA410020AC410020AE410020F9
S2240200C00E420020F64100202DE9F04F85B0814688469346414C04F50476012300934FF064
S2240200E0020A06E06B685B7D5B4527D01834B44264D027462389002BF8D02568002DF5D0C4
S2240201002B6A002BF2D042462946484600F066FD0128E7D0B8F1010F4AD0B8F1000FE5D15D
S2240201202B6A1B685B68B9EB032FDFD1286A05F0A1FD002808BF4FF0010AD7E7284604F0D9
S224020140C1FC01900028D1D1284605F091FF012804D0019B00934FF0040AC7E74FF0000324
S2240201608DF80F3094F812A00DF10F020121284603F0B2FC9DF80F30A3B1012809D0BA7CD6
S22402018052450AD12B6983B101209847DDF804A0ACE7284606F076FBF1E75146284604F06C
S2240201A08BFDEFE74FF0020AA0E7DDF804A09DE72B6A1B681B684B4598D1B7E76FF07F43B8
S2240201C0994503D0504605B0BDE8F08F009B012BF8D10021584605F059F9F3E7842B0020B9
S2240201E02DE9F04781468846174642EA012A00243F4E07F05FFCE3B2984267D9E5B20134E4
S22402020005EB850336F823305345F2D105EB8503374A02EB83035A88BDF820309A4201D083
S224020220132031E005EB8503314A02EB8303187906F0D8FE012801D07F2025E005EB85029B
S2240202402B4B03EB82035B7953B1B9F1020F1FD0B9F1030F2BD0B9F1010F04D0132013E0C1
S22402026004F044F9F1E705EB8502214B03EB82039B689847002834D01D4A142303FB052544
S224020280AB689847012821D005F0CCFFBDE8F08705EB8502164B03EB8203DB68984710B33F
S2240202A0134A142303FB0525EB689847EAE705EB85020F4B03EB82031B699847A8B10C4B21
S2240202C0142202FB05352B699847DBE7094B83F8019083F80280DF70032006F05DFF012033
S2240202E0D2E71220D0E71220CEE71220CCE700BFCC3700202810002008B506F005FC3E4B12
S22402030000221A7404F03EFE04F05AFE06F094F93A4BC2221A7705F0D5F906F09BF906F0EA
S2240203206FF906F07BF906F0A3F9354B4122C3F89C201A46D2F89C3013F0400FFAD0304B6B
S2240203404122C3F8A0201A46D2F8A03013F0400FFAD02B4B4122C3F8A4201A46D2F8A4304C
S22402036013F0400FFAD0264B4122C3F8E4201A46D2F8E43013F0400FFAD0214B4222C3F8E2
S224020380E8201A46D2F8E83013F0400FFAD01C4B4422C3F8F0201A46D2F8F03013F0400FBC
S2240203A0FAD0174B4122C3F820211A46D2F8203113F0400FFAD0124B4122C3F824211A46F4
S2240203C0D2F8243113F0400FFAD00D4B4322C3F828211A46D2F8283113F0400FFAD0094B27
S2240203E06FF07F421A614FF2FF725A61064A9A614FF460721A6208BD0014004000100040A9
S224020400001C00400008004056A80100374B00229A73012829D078284CD0354B1B7883B954
S224020420A0F11103DBB2012B59D9A0F17E03DBB2012B54D9312852D000232E4A53712B4ADE
S224020440D3732D4A7F2313702C4B1B7853709070264B1A6003221A8100225A7301221A739C
S2240204609A73274B00221A707047264B1B78012B12D01F4B1B781BB91E4A53711B4AD373D9
S2240204801A4B214A12881A81204A1A6000225A7301221A739A73E4E7154B1B782BB91346C5
S2240204A0144A5371114AD373DBE7104B00225A73DA73D6E7104A7F2313700C4B5968097844
S2240204C05170782191701A6003221A8100225A7301221A739A730E4B02221A60C1E7002312
S2240204E0044A5371014AD373BBE700BFAC260020F5410020F43F0020FC410020E9410020AF
S224020500ED410020E5410020EA41002028100020BC4000202DE9F04F89B0002878D0D0F8BB
S22402052004E00025D0F80090AC469EF8024099F801B067084FEA4B0303937B1C0093A3B23C
S2240205400693BEF800201FFA8CF39A4211D80BF10103DEF80810DEF80420DBB29C4298BF1E
S2240205600023C95C117002680020537009B0BDE8F08F1FFA8CF306225343D9F80820D11849
S2240205800191D35CC3F38203002B3BD1D9F804604A88039906EB4506029372529C422DD905
S2240205A05A00002107928846B218059201220EE09A450AD036F818700497059FB7F800A0E3
S2240205C0049F574516D10132D2B208F101085FFA88FA5445ECD8009F974204D98F4206D9F8
S2240205E00A44BA4203DB079BF35A029323460133DBB2D3E73CBF0131C9B2E6E7019BBDF89E
S22402060008205A80069B0CF1010C1D44ADB298E70B20ABE7D0B90023374A1380374A138056
S224020620374A1380374B9FED380A83ED000A83ED010A83ED020A83ED030A83ED040A83ED73
S224020640050A83ED060A83ED070A70472C4B1B8893BB10B4284B1988072923D84A1C92B2B7
S2240206601A8028488C00031983ED000A0346011D2144DFED257AB3EC017A77EE877A8B42C3
S224020680F9D1072A88BF11460ED807EE102AB8EE477ADFED1E6A37EE267A87EE870A5DF8CA
S2240206A0044B7047DFED187A154B01221A80134B00221A800A46E8E7104A11884B1C9BB2D2
S2240206C01380104A02EB810282ED000A072B02D90A4B00221A800B4B03F120029FED0A0A13
S2240206E0F3EC017A30EE270A9A42F9D1F4EE007A20EE270A704700BFC4410020C641002047
S224020700C8410020643D002000000000BD378635002874D130B40146394A012382F832301E
S22402072092F83D3043F0200082F841000E2B9ABF0133DAB20A46324B83F83D20314D2868A8
S224020740DA8F845C83F84240541CA4B2DC87045D83F84340941CA4B2DC87045D83F84440FB
S224020760D41CA4B2DC87045D83F84540141DA4B2DC87045D83F84640541DA4B2DC87045D91
S22402078083F84740941DA4B2DC87005D83F84800073292B2DA872B899A4226D31848807B04
S2240207A001280CD008339A1A154B83F84920154B9B7B012B1DD1134B0022DA7319E0D21AB8
S2240207C0002A0DDD0E4B1C7C00230D4805299CBFC31A83F848400131C9B20B468A42F5DC91
S2240207E0074B082283F84920E1E7054B082283F84920034B002283F8402030BC70477047C7
S2240208006C390020AC260020344B5B7B012B15D010B5022B19D0324B5B79022B15D0314BFA
S2240208201A6841F287339A4229D901232E4A13702C4A002111602D4A13701BE0294B0022B2
S2240208401A602A4B02221A707047FCF791F9284B00221A70214B5B7B022B04BF1F4B5A7338
S2240208601F4B5B79022B06D01E4B00221A601F4B03221A7010BD1A4B00225A71F4E71D4BB0
S2240208801B781BB9194B01221A70F3E7134C62681370194A13700120184A1070226840336D
S2240208A0137006F079FC0023124A1370104A1370637B022B0AD00A4B5B79022B09D0094BFC
S2240208C000221A60094B03221A70D3E700226273F1E7034B00225A71F1E700BFAC26002025
S2240208E0F43F0020C040002005420020F941002004420020FF410020E9410020F541002057
S2240209002DE9F0471646C2688A46C57919461F46104606F00FFC57454FEA151420EAE0707C
S2240209201FFA80F858D0791E104689B206F002FC002851DD1FFA80F90AEB0603013B9F42D8
S2240209404DD0791C104689B206F0F4FB002846DD82B2A7EB0A0091454FEA003087B240D3C2
S224020960A8EB020080B2821A09EB02010C2289B203F0E8FCA0F5805000B2022E384480B2E1
S22402098004D9711E002289B203F0DCFCB0F5805F28BF4FF4805015F00F0580B210D005EB23
S2240209A085050C22ED0085424FEA450198BF401BC1F580518CBF002080B289B203F0C2FC83
S2240209C040F6FF739842C4F10C0428BF184680B2204180B2BDE8F0874FF00009ACE70022A6
S2240209E0B7E7A8EB4901A2EB090011440C2280B289B203F0A7FCBFE7F0B52DED028B83B034
S224020A00102200212A4806F08CFB0C220021294806F087FB02220021274806F082FB032209
S224020A2069464FF4F06004F0ADF99DF80030042B28BF0023214A13709DF80230A3F1280262
S224020A40D2B2D72A28BF6E231D4A13709BB21D4A93839FED1D8AB0EE480A0020FFF7DAFDCE
S224020A6000221A4B1A701A4B83ED008A194B1A70194B1A80194C1A4811461A4D1A4E371DD2
S224020A8005E026F8321047F832105155013224F8021F20F8021FD3B2022BF2D9072BF4D9BE
S224020AA00133DBB20F2BF1D903B0BDEC028BF0BDF43E0020743F0020704100204F4200202D
S224020AC05042002000A0014100000000474200204841002048420020BE410020223D0020E1
S224020AE0423D002094400020403E0020F0B59DF814509DF818C09DF81C709DF820609DF8E8
S224020B0024E0A1B9002A66D1002B5ED150EA05031BD1BCF1000F4CD1002F41D1002E36D138
S224020B20BEF1000F22D101230A9A137055E0012953D1134351D102230A9A13704DE0002B13
S224020B404BD103230A9A137047E0012D15D0002D43D1BCF1010F2FD0BCF1000F3DD1012FF4
S224020B6020D0002F39D1012E13D0B6BBBEF1010F33D109230A9A13702FE046EA0E063E43D8
S224020B805CEA060329D105230A9A137025E0012E23D1BEF1000F20D108230A9A13701CE091
S224020BA0012F1AD156EA0E0317D107230A9A137013E0BCF1010F10D146EA0E0657EA06036A
S224020BC00BD106230A9A137007E0012B05D104230A9A137001E0012AB1D0F0BDF0B583B099
S224020BE00F6A002F6DD015460C460646384605F041F80346002865D06FF07F439E4208D0E5
S224020C00EEB9012D0ED03B685B68013318BF012358E0012D3B680CBF1B685B68013318BF60
S224020C2001234FE03B681A68B2F1FF3F05D05B68013318BF0123DBB244E00023FBE7294668
S224020C40204604F00DFD034600283BD001AB6A462946304603F0C8FC01280AD0012D28D08C
S224020C60236A1B685B68B6EB032F0CBF0123002328E0012D0CD0236A1B685B68009A934261
S224020C8015D3019A93422CBF00230123DBB219E0236A1B681B68009A934206D3019A9342F2
S224020CA02CBF00230123DBB20CE00023FBE70023ECE7236A1B681B68B34214BF00230123E5
S224020CC000E00023184603B0F0BD7047F8B5002866D003680C261D88002319469AB29542A3
S224020CE04ED800295ED0304C06F076FD2F48637A002B4FD106F070FD038843F00103038044
S224020D0006F06AFD012301626372294F0022294C1546012621FA02F3DB072CD5D05D00F072
S224020D203F0C10F0010F4FEA90134FEA5C0E4FEAC31304EB030023447044634490F830E077
S224020D4014BF66F3071E66F3030E80F830E083F8405093F8400040F0010083F8400093F8FC
S224020D60400065F3820083F8400093F8400065F3410083F840000132202ACBD10020F8BD8A
S224020D8006FB03F244680133A718A2587C6822431143A3E706F020FD036A0B430362B4E7C8
S224020DA00B20F8BD0220F8BDBC3D0020001C0043F25A02000080004110B43749CB6823F460
S224020DC0E0631B041B0C43F0BF6343F40033CB60BFF35F8F62B6314BE02283F80A234FF478
S224020DE08060186083F80B234FF40060186083F82E234FF48040586083F82F234FF40044F5
S224020E005C6083F830234FF48030586083F831234FF40030586083F832234FF48020586031
S224020E2083F833234FF40020586083F834234FF48010586083F835234FF40010586083F809
S224020E404F239C6083F85523986083F856234FF48000986083F86D234FF40050D86083F832
S224020E6077234FF40000D86083F879234FF00072DA604B6A43F480234B624B6943F010031E
S224020E804B614B6A43F400334B624B6A43F480334B625DF8044B704700ED00E000E100E09E
S224020EA02DE9F84F8046364B01221A54354D00242F46A146924610E0182303FB04731B7DE4
S224020EC013F0080F2BD047E030684368DB7E434537D001341835162C50D022462E462B8930
S224020EE0002BF6D004EB440307EBC3031B7DDB09EFD0A97C11F0420FE6D1286843685B7E8F
S224020F004345E1D101F0FB0B85F812B0BBEB010B18BF4FF0010B4368DB7E4345CCD0B27C30
S224020F208A4201D003F0C8FEBBF1000FD1D03146306805F089F90028CBD1306805F0A2FC83
S224020F40C7E702EB420307EBC3031B7D13F0080F08BFCB46E8D0CB4602EB420207EBC202B8
S224020F60137D13F0040FDAD1337C002BD7D086F81090B27C9142DAD0D346D3E7BDE8F88FD0
S224020F80AC400020842B002088B061EE837A21EE237A77EEC77A73EEE15A65EE805A77EE6B
S224020FA0A57A71EE435A65EEA05A77EEA57A21EE227A61EE826A37EE667A31EEE26A26EED4
S224020FC0006A37EE067A72EE416A66EEA00A77EE200AF5EEC07AF1EE10FA4CBF012300230B
S224020FE0F5EEC00AF1EE10FADBB24CBF01220022934236D122EEC37A33EE423A23EE213A45
S22402100037EE033A72EEE32A62EE812A73EE222A22EE232A32EE822AB5EEC02AF1EE10FAB3
S22402102013D4F5EEC07AF1EE10FA15DDF5EEC00AF1EE10FA13DD77EEA07AF4EEC27AF1EEC8
S22402104010FA4CBF0120002007E0F1EE677AF1EE600AB1EE422AE4E70020C0B202E00020D9
S224021060FBE7002008B07047002A62D02DE9F041134620B1012830D00020BDE8F0812E4A54
S224021080D2F8A420C2F3052201B301395FFA81F84FF0000CDFF8A4E000E0A446DEF8004099
S2240210A004EB021427686668A568E4681F605E609D60DC60614509D010330132D2B2082A4D
S2240210C008BF02460CF10104E045E6D102F03F02194BC3F8A8200120CFE7174AD2F8B4202C
S2240210E0C2F30522F1B101395FFA81FE0024DFF84CC000E00446DCF8040000EB02100768E4
S22402110046688568C0681F605E609D60D8608C4208D010330132D2B2082A08BF0022601C5C
S2240211207445E7D102F03F02034BC3F8B8200120A3E70020704700BF00040042A03D00209F
S22402114070B584B000240294ADF80240052A02D9042004B070BD1E4614460D4603A903F0CF
S224021160A7FB012801D00120F3E7039B19684B685B7DAB4201D00220EBE70DF1020302AAC6
S224021180204603F02FF8012801D00420E1E7029A53880899098899423BD31179022920D0AB
S2240211A0012D03D0042D01D00220D2E72A4601A9039B188903F040FA012803D00020089B05
S2240211C01880C6E7029CBDF802300233628801991944304605F0CBFB6388089A13800020B7
S2240211E0B7E7916839B130468847029B5B88089A13800020ADE7117B0029AAD03246039877
S224021200006800F0DFFB029B5B88089A138000209FE705209DE7FEE738B500222B4802EB3D
S224021220420300EBC303197D6FF3041119750132162AF4D1264B1B78012B06D00021084669
S22402124003F022FE0024214D14E00120FDF7E0FEF8E704EB440355F8330005F013FB04EB74
S224021260440305EBC3031A7D6FF304121A750134162C08D004EB440305EBC3031B7D13F0F6
S224021280100FF4D0E5E7134BB3F840214BF6BE239A4215D0104B0021197001225A709A704F
S2240212A0DA7019715A711622DA800C4B19700C4B20221A80FF229A70054B02221A7038BDC5
S2240212C0044B93F84221074B1A70E3E7842B00200A420020542F00208C3F0020683F002094
S2240212E0C84000200B42002010B504462F4A682303FB002393F828301BBB00EB80032C4A81
S22402130002EB83035B7B0BB1032B1CD104EB8403274A02EB8303DB7B7BB1244A682303FBD3
S2240213200423032283F82820204A682303FB042400236365012363700BE0204601F01CF943
S224021340F2E7012B06D0194B682202FB04340123637010BD00EB8003154A02EB8303DB7B2E
S224021360012B16D0002BEED100EB8003104A02EB83035B7B0BB1032BE5D1204601F014F856
S2240213800A4A682303FB04240023636503236370DFE7064A682303FB0024032384F82830A0
S2240213A00023636501236370D3E700BF6C390020AC2600202DE9F04F85B09DF838709DF8B8
S2240213C03CA0002403944468647DBC4204D00025284605B0BDE8F08F0191044603A902F02A
S2240213E0D1FC039B002B47D0A3681E68002E45D04FF001080025AB4620E00BF1020072880F
S224021400019B1918039B184405F0B1FA4D4608E00BF10200728801990144184405F0A7FA1A
S224021420012573889B441FFA8BFBB8F1050F19D0A36853F8286008F101089EB196F804900F
S224021440B9F1020FF1D0B9F1010FD6D0B9F1000FE7D1039B21881A889142D9D1BAF1000F18
S224021460DFD0D5E7002DB3D0019B1A88039B1A80384605F0FDFBABE70025A9E70025A7E76F
S2240214802DE9F84F804600242E4B1C54DFF8B8A05546D1461FE02B685B685B7E434526D187
S2240214A095F812B02BF0020343F04003AB7404EB44000AEBC00005F01DFDAA7C5A452ED166
S2240214C033681B690BB10220984733897BB901341835162C33D027462E462B89002BF6D0EC
S2240214E004EB440309EBC3031B7DDB09D3D133685B68DB7E434517D033685B689B7E4345B0
S224021500E5D17B00DA1909EBC202127D1F4409EBC70702F0FD036FF300033B75D7E75946D0
S224021520286803F0C9FBCBE707EB470309EBC3031A7D02F0FB026FF3C3021A75DCE7BDE811
S224021540F88F00BFAC400020842B002008B5284B1B68B3F5FA6F15D3264B1B7893B9264BF6
S2240215601B7B13F0FD0F11D17820FEF74FFF234A1378013313701E4B00221A60204B0422BD
S2240215801A700AE01B4B1B78012B07D01B4B1B78962B23D81A4B04221A7008BD164B1B7B4E
S2240215A0012BF3D0174B1B78782BEFD0164B00221A70114B5B7B022B04BF0F4B5A73134B2A
S2240215C05B79022B06D00A4B00221A600C4B03221A70E2E70D4B00225A71F4E704F01EFB40
S2240215E0034B00221A60064B01221A70D5E700BFC0400020ED410020AC26002003420020BC
S224021600F9410020F141002004420020F43F002010B52A4B1C6D24F4C05323F011034BB14D
S224021620264A1365264B1B6823B1254B59681B682046984714F0010F0DD0204B01221A65FC
S224021640D3F8A4001F4B1B682BB11E4B59681B6800F07F00984714F0100F0DD0174B1022BC
S2240216601A65D3F8B400174B9B682BB1154BD9689B6800F07F00984714F4006F0AD00F4B87
S2240216804FF400621A65104B1B681BB10E4B58681B68984714F4805F0ED0084B4FF48052CD
S2240216A01A65D3F8F400094B1B682BB1074B59681B6800F03F00984710BD00BF00040042BC
S2240216C0BC3F0020943E0020AC3F0020B43F0020F0B583B00446867C16F0080519D0057D36
S2240216E005F00303022B07D015F0010511D0437CFBB1002343740CE0437CFF2B1BD00133BF
S224021700DBB2437400684268127F9A4288BF012503D925B9284603B0F0BD01250DE0214690
S224021720206804F091FD0028F4D1206805F0AAF8F0E71D46EDE7006800250021617426F0E5
S2240217400C03A3740DF1070202F0C6F90746A8B900232374A27CB24203D03146206803F065
S224021760ABFA002DD6D0002FD9D0206805F08AF823685B68587D05F063FACBE70023237432
S224021780A27CB24208BF0125EFD001273D46E4E710B50446012808D0B0B9264B1B78012B65
S2240217A012D1254B01221A700EE0244B1B780E2B9ABF0133DBB2002320490B7041F21B008A
S2240217C0F8F726FF05F078FA1A4B1C701A4B1B78012B00D010BD1A4941F21D00F8F718FF1C
S2240217E0184C214641F21E00F8F712FF214641F21C00F8F70DFF144B1B78012B05D90023F6
S2240218000D4A1370104A1370E4E70C4B1B780E2B9ABF0133DBB2002308490B7041F21B00C5
S224021820F8F7F6FE05F048FA074A137801331370D0E700BF36420020374200203B420020B0
S224021840394200203A420020384200202DE9F04186B084222B4B1A7003238DF804308DF829
S224021860052001228DF8062018228DF8072004228DF808208DF8093000238DF80A308DF890
S2240218800B300B2704F062FE013F17F0FF07F9D1032400234FF0010806AA02EB430313F8E9
S2240218A0136CB5B29DF80E30AB4216D00DF10E023146204605F024FA8DF81000C0F3072325
S2240218C08DF81130C0F307408DF81200404604F015FD9DF80E30AB42E8D10137FFB23B463B
S2240218E006AA02EB470212F8144C002CD4D106AA02EB470212F8132C002ACDD1002006B0F3
S224021900BDE8F0814442002038B50346002947D0002845D0264D6A7A002A43D0042A43D07C
S22402192000684279013A062A40D8224CE960236000F058FB23684FF400011F4A1B68C2F808
S2240219408C115B795B01DBB282F87733D16005F043FF1A4991F82C3043F0040381F82C3043
S22402196005F03AFF072381F82E3005F035FF012291F82D3043F0010381F82D30104B1A700D
S22402198000232B8003F066FC044630B9288804236B72FCF709FC204638BD0220687238BDF2
S2240219A00B2038BD032038BD012038BD022038BDBC3D00201800002000E100E0001C00434A
S2240219C060420020F0B583B00024248904B10BB903B0F0BD1D4617460C4606461A460021DD
S2240219E0384605F009FF611E0529F1D8DFE801F00311173F351D012D08D0002462897B19D2
S224021A00110A03F8021C03F8012CE1E7FF233B70DEE73D440024A37B05F8013CD8E73D44CC
S224021A200024E37B05F8013CD2E700238DF8073073680DF10701587D04F08AFE40B97A198D
S224021A409DF80730003318BF012302F8013CBFE77B19002203F8012CBAE773681B7E002B8A
S224021A60B6D07B190024627C03F8012CB0E73D440024237C05F8013CAAE7FEE710B582B099
S224021A8000248DF800408DF801408DF802408DF803408DF804408DF805408DF806408DF81E
S224021AA0074000F00F0343F01003134A13706946A0B2F8F7ADFD0134652CF8D100200F4B0D
S224021AC018700F4B18700F4B18700F4B18600F4B18700F4B18700F4B18700F4B18700F4BFF
S224021AE018700F4B18700F4B18700F4B18700F4B187002B010BD00BF184200201C42002099
S224021B001D4200201E420020204100201F42002020420020214200202242002023420020AF
S224021B202442002025420020264200202742002010B504464FF42172002105F05DFE254ABB
S224021B40936943F001039361936913F0010FFBD0204A936943F0020393611F4B1C60196884
S224021B6089B241F0004141F40021C2F8A01004F180015960596889B241F0004141F40021FE
S224021B80C2F8B01004F58071D960D96889B241F08051C2F8C01004F500711961196989B2F8
S224021BA041F48011C2F8F01004F520745C6159690A4808605B699BB243F48033C2F884306F
S224021BC0936923F001039361936913F0010FFBD110BD00BF00040042A03D0020FF0700083F
S224021BE02DE9F84F80460F4691469A4641EA002B0024254E05F05CFFE3B298423AD9E5B259
S224021C00013405EB450336F823305B45F2D105EB45031D4A02EB8303187905F0E3F90128CF
S224021C2001D07F2427E005EB4503174A02EB83035B797BB105EB4503134A02EB83039B680B
S224021C40FBB105EB450502EB85056A88524504D0132410E002F04AFCECE7484698470446DA
S224021C60012808D1094B83F801809F70022005F093FA00E01224204604F0D4FA2046BDE80F
S224021C80F88F1224F7E700BF0C37002028100020F8B5C3B11D460E8900239C461C4602EBB9
S224021CA0C40732F83440B4423DD001339BB21C469D42F4D867464FF0000C3AE04FF0010CC5
S224021CC0BCF1000F1BD143680121587D03F0DEFB012025E03E4612E03E4610E001201FE0B7
S224021CE001339BB21C469D421BD902EBC40632F83440002CF4D101339BB2AB42DED2002E95
S224021D00ECD00B8933804B8973808B7C33710B7C73714B7CB3719DF8180004F091FF0020A0
S224021D20F8BD3E46CCE701339BB29D42D4D84FF0010CBCF1000FCDD100231C46D5E7FEE7D8
S224021D4000284ED110B4274B012283F8322026490889C2B283F8412009680C7883F84240CD
S224021D604C7883F843408C7883F84440CC7883F845400C7983F846404C7983F84740897904
S224021D8083F84810D8879B7B012B0ED00132154B83F84920144B9B7B012B1ED0114B002266
S224021DA083F840205DF8044B7047501CC4B2072C0ED80C48017C04F14003034441302044C6
S224021DC0C2F1060250FA82F203F8011F9342FBD1044B082283F84920DCE7034B0022DA73EA
S224021DE0DCE770476C390020AC26002008B5204B1B78DBB2012B05D01E4B1B78DBB2012BAD
S224021E000AD008BD1C491D48FFF77EFD0028F3D1174B00221A70EFE7164B00221A70FAF713
S224021E2013F9B8B91648FEF775FB58B91548F9F7ABFE58B91448FBF729F870B1134B04222F
S224021E401A700AE0114B02221A70EFE70F4B03221A70EFE70D4B01221A700A4B1B6893F9DF
S224021E600030002BB4BF024B094B01221A70C8E72D200020913E002065790200383F0020BD
S224021E80DC3F0020A43E0020EC3F0020D5410020B140002038B51D460132D2B2013A0F2AF1
S224021EA036D8DFE802F037080B0E1114171A1D202326292C2F3240F2D9242DE040F2A9341F
S224021EC02AE040F27A4427E040F24A5424E040F21B6421E040F253741EE040F6F4041BE054
S224021EE040F6FD2418E040F6055415E040F6DF7412E04FF499540FE041F232740CE041F672
S224021F00144409E042F2C61406E042F6B10403E02C6801E040F2712448B121B10648FBF76E
S224021F203DF92C6038BD2046FBF738F9F9E70020FBF734F9F5E700BFA0860100022801D975
S224021F400020704710B5044604F0ACFF224B23F83400022C0AD0204B33F83430852B1AD09D
S224021F601D4800EBC4040020606010BD022004F099FF852803D18520174B1882EBE70F20C4
S224021F8004F090FF852801D18520F5E7022004F089FF80B2F0E7104A02EBC4025368013314
S224021FA053604EF65F22934207D90B4800EBC4004EF6602343600020D7E7084B187838B9CF
S224021FC0074B1B78012B05D9022B08BF1846CCE70120CAE70120C8E7403E00200D42002057
S224021FE04742002038B50424244B00210A4661F305111D6964F30E351D611D6964F30A2528
S2240220001D615D6964F30E355D615D6964F30A255D618378402B17D1082363F30301182305
S22402202063F30C2242F01F0005F0D6FB144B82B2144882801B681B681B790F2B0CD96FF3F2
S2240220400B2141F480510BE0802B15D10A2363F3030141F04001E2E763F30B216FF30C31E8
S22402206005F0BAFB0322037A62F30303037205F0B3FB8161002038BD022038BD002000422A
S22402208018000020001C004370B586B00B9E0C9C05969DF82850003518BF01250495003350
S2240220A018BF01230393003218BF01220292003118BF01210191003018BF012000902378B9
S2240220C06278A178E078FEF711FD3378013B082B09D8DFE803F0050A0E12161A1E22260031
S2240220E0002003F0B7FC06B070BD002003F0B2FCF9E7002003F0AEFCF5E7002003F0AAFC3D
S224022100F1E7AC2003F0A6FCEDE7AC2003F0A2FCE9E7E12003F09EFCE5E7782003F09AFC03
S224022120E1E7AC2003F096FCDDE770B586B00B9E0C9C05969DF82850003518BF012504959C
S224022140003318BF01230393003218BF01220292003118BF01210191003018BF0120009080
S224022160E378A27861782078FEF7C0FC3378013B082B09D8DFE803F0050A0E12161A1E226D
S2240221802600002003F07EFC06B070BD292003F079FCF9E77D2003F075FCF5E7D22003F04F
S2240221A071FCF1E7372003F06DFCEDE7CB2003F069FCE9E7822003F065FCE5E7822003F0E2
S2240221C061FCE1E7822003F05DFCDDE7174B1A7812F0100F27D04FF4C87315490B60154970
S2240221E00B6015490B60642314490B6014490B6014490B60322314490B6014490B60144983
S2240222000B6014490B6014490B6014490B6014490B6014490B6014490B6042F02002034BFA
S2240222201A70002070470520704700BF18420020E0400020E4400020E8400020EC40002009
S224022240F0400020F4400020F8400020FC4000200041002004410020084100200C41002083
S224022260104100201441002018410020000098420000000000007F430000244200004E4365
S2240222800000AE42000007430000AE42000007430000294300004E430000294300007F4398
S2240222A0000047430000D44200007F43000098420000A841000007430000AE42000007436E
S2240222C0000029430000C04200007F4300004E430000AE4200007F430000404200007F4340
S2240222E00000374300004E430000294300000C430000B84200004E430000B84200004E43FB
S2240223000000244300000C4300002443244B1B78182B3ED92DE9F0470025214B1D70214C65
S224022320271F4FF055094FF008081AE004F10A0004F03CF8608084F800904246214634F83C
S224022340020C05F061FA14F8043C23F0010343F0020304F8043C0023237501351A34082DCD
S2240223601BD014F8043C13F0010FF6D094F814A005F016FB05EB450305EB8303534407EBC9
S2240223804303D881237D0133DBB22375042BE4D9CCE70133024A13707047BDE8F08700BF6A
S2240223A0113F0020C034002038B9244B032283F8282093F83130082B00D0704710B51F4A76
S2240223C092F8293003F00F0192F82A3043EA01231B494B810621918492899A4225D3072B4E
S2240223E000D810BD154A012182F82210144B586892F82B400470586892F82C404470586852
S22402240092F82D408470586892F82E40C470586892F82F400471586892F830204271597397
S2240224200021084602F00EF8DBE7054B05225A730221002002F006F8D3E700BF6C390020B7
S224022440AC26002070B588B000240694ADF81640022A02D9042008B070BD1E4614460D464C
S22402246007A902F025FA012801D00120F3E7079B19684B685B7DAB4201D00220EBE706AA8F
S224022480204602F041FD012801D00420E3E70DF1160206A9204602F031FC0C9B1A88BDF86F
S2240224A016309A4218D3012D03D0042D01D00220D1E7079B18890DF1160302930C9B019301
S2240224C000962B46069A214601F0ACFD012805D000200C9B1880BEE70620BCE70020BAE7C1
S2240224E000B1704710B5214B00249C76FF22DA767F211977012159779C77DA7783F8204034
S2240225001B4A14815481147354739473D4731474184A14715471032283F8282083F83C4036
S224022520022283F840209C84DC8783F8321083F8224083F83D40DC8483F84A205C665C65B8
S2240225409C65DC651C66204600F05EFF204602F0B8FA204604F05CFB204604F04DFB20463A
S22402256002F0F1FC204604F03BFB10BD6C390020AC260020F43F0020002843D1224B032240
S22402258083F8282093F8291001F00F0293F83130934234D9002A32D001F008011B4BDB7BFB
S2240225A00B432CD192B2194B5A81013A92B2062A21D85968144A92F82A000870596892F808
S2240225C02B004870596892F82C008870596892F82D00C870596892F82E000871596892F8B5
S2240225E02F004871596892F830208A7102225A730122DA737047054B03225A737047034BF7
S22402260003225A73704700BF6C390020AC260020002844D1224B032283F82820214BDB7B40
S224022620002B3CD11E4A92F8221092F8292002F00F02914203D01B4B05225A73704730B4C6
S2240226400E299CBF4B1CDBB2154A82F8223092F83110012910D90123124DD11891F8294086
S224022660918C68684454918C013191840133DBB292F831109942F0D80A4B5A89084B9B8C89
S2240226809A4206D8074B04225A730122DA7330BC70470829FBD0034B05225A73F7E770474E
S2240226A06C390020AC26002010B5244C214641F20500F7F7ADFF214641F20700F7F7A8FFB8
S2240226C0214641F20900F7F7A3FF214641F20B00F7F79EFF214641F20D00F7F799FF2146FC
S2240226E041F20F00F7F794FF214641F21100F7F78FFF214641F21600F7F78AFF214641F228
S2240227001900F7F785FF214641F21F00F7F780FF214641F22100F7F77BFF214641F2230021
S224022720F7F776FF214641F23300F7F771FF214641F25A00F7F76CFF10BD00BF3D4200208C
S22402274006EE900A07EE901AB8EE676A9FED1C7AC6EE077ABCEEE77AB8EE477A37EEC77A9F
S224022760B6EE006AB4EEC67AF1EE10FAFCEEE77A17EE903A4CBF5F336033DBB2114A1370C4
S22402278007EE903AF8EEE77A9FED0F7A67EE877A9FED0E7A77EE877A9FED0D6A77EEC67A9F
S2240227A0B8EE667A67EE877ADFED0A6A87EEA67A77EE067AFCEEE77A17EE903A53707047E8
S2240227C00000CC3F704100209A9989BE00C484430000204200007F4310B500EB8002214B4F
S2240227E003EB82031B7B012B06D0682303FB00F01D4B01221A5410BD04461A4B03EB820366
S2240228001B89072B13D81346164A02EB83031B7C002BEAD1FFF794FA134A682303FB04F4E5
S22402282013190021D965196603231355E3E700EB80030C4A02EB83031B7C002BD5D120462A
S22402284000F0E4FF084A682303FB04F4131901215977FF21D977D9760021D96519660323EA
S2240228601355C8E7AC2600206C390020234B1B7813B1827C13403ED010B50468002C34D0FE
S22402288021461E4B587802F0ADFF012802D00023184610BD6368194A92785B7D9A4201D0ED
S2240228A00023F5E7154BDB78012B08D0FBB92146124B187904F014FB03460028E8D00F4BCC
S2240228C05B79012B01D00023E2E7206A88B103F0D1F903460028DBD0084B197A204602F05A
S2240228E0BFFE031C18BF0123D2E70023D0E70023CEE70023CCE71846704700BF8C3F0020FA
S22402290038B500F03BFA214B1979C1F30301CBB21F4A927B9A422FD01C4BDA7818790009C7
S22402292000EB02101A4A10809D7CDC7C240904EB051454809C78C4F340041474DD791C7AA2
S224022940240904EB051494801D7B5C7B240904EB0514D48010819C7DD87D000900EB041028
S22402296050815C799879000900EB04109081DB7AC3F3C4035374917303F022FF012814BFD3
S22402298000200120024BD87338BD00BFF43D00206C3E0020224B30B51A680623946803FB91
S2240229A0004043888B4239D0156834BFC91A591AAB7889B2402B08BF490884292CD80529A9
S2240229C02CD98288C2F3013302F00F0403EB4300C3EBC003C2F30320C2F3031200EB400084
S2240229E003EBC303C0EBC000184400EB420080B2052C0CD8EB780B4AC3F3011332F81330F2
S224022A00594389B288422CBF0020012030BD0130053C80B2E4B2EBE7012030BD002030BDCE
S224022A2018000020E45A020010B49478FF2C1CBF01349470147844B90123137004235370EE
S224022A4000230B705DF8044B70475478022C1DD0032C23D0012C08D000230B700128F1D1DF
S224022A600323537000239370ECE7012809D090789DF804309842E5D30423537000230B7080
S224022A80E0E70323537000239370DBE701230B700028D7D1537000239370D3E794789C429B
S224022AA004D30223537001230B70CBE70028C9D10123537000239370C4E7FEE708B51F4B79
S224022AC01B78013BDBB2012B03D91D4B01221A7008BD1C4B187804F067FB01281DD0174BEC
S224022AE01B78013BDBB2012BEFD8164B187804F0AEFE0128E9D1134B187804F055FB0028B2
S224022B00E3D1782003F088F900230C4A13700E4A13600B4B04221A70DAE70A4B187804F087
S224022B2096FE0128DBD103F077F90023034A1370054A1360024B02221A70C9E7D941002028
S224022B40E1410020DD410020B840002010B504F02DFFC0F3CF23012B08BFA0F5805004B23E
S224022B6004F01EFF194B1B78012B13D0184B00221A70184B1B88834217D0174B00221A8058
S224022B8004F5FF639BB2B3F53E6F06D9104B01221A7002E00E4B01221A700E4B18800C491C
S224022BA041F20200F7F734FD10BD0B4A138801339BB21380B3F5487FE2D3054B01221A70C8
S224022BC0054B4FF448721A80DAE700BF144200200D420020EE410020F241002008B51D4BDB
S224022BE05B7B032B0BD0022B10D01B4B1A6842F20F739A4224D8194B02221A7008BD164B34
S224022C0000221A60154B01221A70F7E7F9F7B0FF134B00221A700F4B5B7B022B04BF0D4B05
S224022C205A73104B5B79022B06D00B4B00221A600A4B03221A70E1E70A4B00225A71F4E7B3
S224022C4002F0ECFF044B00221A60044B01221A70D4E700BFAC260020C0400020F9410020C3
S224022C6004420020F43F0020A0F582501C3807282DD8DFE800F027221D18130E0904154BE2
S224022C801B780B7000207047134B1B780B7000207047124B1B780B7000207047104B1B78D5
S224022CA00B70002070470F4B1B780B70002070470D4B1B780B70002070470C4B1B780B70DA
S224022CC0002070470A4B1B780B70002070470120704700BFF0410020EC410020E84100205E
S224022CE0E4410020E0410020DC410020D8410020D441002008B5194B9847194B9847EFF377
S224022D00108172B6174AD2F8883043F47003C2F88830BFF34F8FBFF36F8F01B962B6124A86
S224022D20936823F0010393601346DA6812F0010FFBD10D4B24225A6001229A6000F0A6F80B
S224022D400A4B23F07F03074A9360094B9847094B9847094B9847FBF7E3FCFEE76348020042
S224022D606348020000ED00E0006000410080010081400200634802006348020008B51E4B6D
S224022D801B78042B1CD803EB43031C4A02EB83035B6800209847184B1870042813D9164B43
S224022DA000221A70144B1B78154A12789A421DD003EB4303114A52F823300020984715E09C
S224022DC000200D4B18700E4B1B788342EAD003EB43030A4A02EB83039B6800209847064B33
S224022DE01B78042BE0D9044B00221A70024B1A78034B1A7008BD00BFF84100202851020047
S224022E00F441002008B541F26403984205D041F26503984219D0012008BD184B18780870A1
S224022E205878487098788870D878C870187908715879487198798871DB79CB71104B1B7857
S224022E40137004F099FC0020E6E70E4B187808705878487098788870D878C87018790871EF
S224022E605879487198798871DB79CB71064B1B78137004F089FC0020CEE700BF044000204F
S224022E80194200200C4000201A4200201E4B1F4A9342F0B438BF002103D203F8011B9342A4
S224022EA0FBD11B4AD2E9000150EA01034FF0000610D09468034602F10C076CB921B1014434
S224022EC003F8016B9942FBD13A46D2E9000150EA0103EED1F0BC704759B101F10C030C38F2
S224022EE0801A1A443B461C1813F8015B25709342F9D111F0030318BF012303EB910107EB0F
S224022F0081073A46E1E700BF1000002020000020808201000138C0B20F2834D8A9B32DE948
S224022F20F0471B4BD3F8C430C3F30443013001EB00150026DFF85C904FF00108D9F80C40B1
S224022F4018012218D1F800A0D1F804E0D1F808C0CF6844F800A0C2F804E0C2F808C0D76006
S224022F60103108FA03F216430133DBB2102B08BF00238D42E2D1BFF34F8F054BC3F8D06086
S224022F800120BDE8F087002070470020704700BF00040042A03D002030B583B0044603F0E8
S224022FA045FA0546204600F0ADFF012D09D0012818D0194A682303FB04240123A37003B068
S224022FC030BD0221204602F0E7FD0DF10701204602F0C0FB98B9104A682303FB0424022304
S224022FE0A370ECE7002DE4D10321204602F0D4FD094A682303FB04240223A370DFE701288A
S224023000D7D1204601F0F4F9034A682303FB04240123A370D3E700BF6C39002010B504463B
S224023020682303FB00F31C4AD35C032B2DD8DFE803F00223262902F0DBFE174A682303FB62
S2240230400423DB6D4FF6E752934205D81249682202FB04120233D3650F4A682303FB04235C
S2240230601B6E4FF6E752934205D80B4A682101FB04240233236610BDFFF7AEFBDDE7FCF7AD
S224023080FDFBDAE7FCF74EFBD7E7682303FB00F3014A0021D154D0E76C39002010B50446DE
S2240230A000F0FD03012B05D0022831D0602801D0122002E0022903D0132003F0B3F810BDE4
S2240230C0154B5C7000229A703221D9701A71C8225A71052004F060F8204603F02BFB022C97
S2240230E018BF0120E9D10FE00B4B02245C7000229A703221D9701A71C8225A71052004F0BF
S2240231004BF8204603F016FB782003F08BF8D6E70229E9D01320D0E72810002010B588B10C
S22402312001281DD0022829D01B4C4FF480421146204604F0EDFB4FF400421146204604F014
S224023140E7FB10BD144C00224FF48041204604F0DFFB00224FF40041204604F0D9FBF0E754
S2240231600D4C00224FF48041204604F0D1FB4FF400421146204604F0CBFBE2E7064C4FF449
S22402318080421146204604F0C3FB00224FF40041204604F0BDFBD4E7808000412DE9F041FC
S2240231A0042832D806461B4C04F504754FF00008474605E0FEF78CFA07461834AC4218D00A
S2240231C020462389002BF8D02368002BF5D05B68002BF2D01A7E012AEFD19A7EB242ECD16C
S2240231E05B7D042BE6D0012BE7D1FEF771FA8046E3E7B8F1000F02D0012003F021FD2FB19B
S224023200042003F01DFD002700E001273846BDE8F08100BF842B00202DE9F04107460E463D
S2240232201A4C1B4DE08858B3013880B2E080804600EB400305EBC3031B89002BF2D000EB55
S224023240400005EBC000FFF711FB0128EAD10F4B1B7A012B08EB48030D4A52F833301B6AAF
S2240232601B680EBF1B685B681B023B6008EB4808074B03EBC80898F812303370002003E02E
S224023280024B1622DA800120BDE8F0818C3F0020842B0020F8B51B4B5870997041EA002622
S2240232A00024194F04F002FCE3B2984226D9E5B2013405EB450337F82330B342F2D105EBED
S2240232C04503114A02EB8303187903F08BFE0446012801D0312412E00B4E6F007B1906EBEC
S2240232E083039B68094898473D4406EB8506708803F052FF022003F04FFF00E012242046F6
S224023300F8BD00BF28100020442900202B10002038B50023194A1360194C23606360A3605E
S224023320E3602361174D2B606B60AB60EB602B616B6105F1120104F1130004F071FB05F1F0
S2240233400F0104F1100004F043FB05F10C0104F10F0004F03DFB04F1120004F08DFB04F174
S224023360110004F08DFB084C204603F00FF9601E04F04CFBA01E04F058FB38BD28410020C8
S224023380583E0020283E0020C67902002DE9F0470023154A1370154A1370154A1380154C22
S2240233A0154D04F55F7A4FF00008DFF858900026124F54F8040B02F039F942464B46FCF7BA
S2240233C039FC32463B46FAF7BDFA02F0BBFF25F8020F5445EDD10021094804F0BDFA03F0CF
S2240233E0CFFBBDE8F08700BF3F42002040420020B641002030200020922D00200000A04098
S224023400117102000000A03F10B58AB004462422002101A804F0F0F90CB10AB010BD41F295
S2240234200503ADF8043001238DF806308DF80730AA238DF808309623ADF80A30ADF80C3006
S2240234401423ADF80E300B4B05930B4B06930B4B079341F26403ADF8223041F25B03ADF8B7
S224023460243041F26503ADF8263001A9002000F061FED2E72810002020000020043F00208E
S22402348000000200D83D0020B537000000000000000000000000000000070800E03D0020B6
S2240234A002023030032D6093000000000000000000160200EE3D00200C800000000000008F
S2240234C0000000000000000001000F00D83D002000000000000000000000000000000000A0
S2240234E0010F0900E73D002000000000000000000000000000000000C268F0B501EB410666
S224023500931985689F780C2303FB01535C681B896488E41A935DE41A436828460025A4B29F
S2240235201E88ABB29E4201D80020F0BD994219D09378BB4216D103787B33DBB2012B15D978
S2240235404368B0F808E05B889E450BD2A3EB0E0392F800E09BB2734504D9A3EB0E039BB2AF
S2240235609C4203D3013503320C30DAE70120F0BD00B1704700B585B00DF1070202A9174BF4
S2240235805889FFF73FFC9DF8083013F00F0222D003F0080151EA13131DD1114B1A711A688B
S2240235A09DF8091011701A689DF80A1051701A689DF80B1091701A689DF80C10D1701A68BA
S2240235C09DF80D1011719DF80E1051719DF80F10917102225A7105B05DF804FB6C390020C8
S2240235E0F43F002070B5194B1B78032B1DD0174B1B78012B23D0154B1C782CBB144B154A8D
S224023600106851689668D568186059609E60DD601069516918615961128B1A8300F05EF9E4
S224023620012808BF0324204670BD042002F04EFF0128DCD1054B02221A700424F3E7034B52
S22402364003221A700424EEE70424ECE714420020F43D0020D83D0020033804282ED8DFE88C
S22402366000F003090F151B00164B1B78012B19D000207047134B1B78022B13D00020704750
S224023680104B1B78032B0DD0002070470D4B1B78042B07D0002070470A4B1B78052B01D0A2
S2240236A000207047012901D000207047064B1878012805D9022818BF0020704700207047C3
S2240236C008467047534200204742002010B483B036238DF8003021238DF80130134B1B7890
S2240236E08DF80230124B1B788DF80330114B1B788DF804306A460DF105040020082112F8B2
S224023700013B58400B4610F0800F4FEA4000C0B218BF80F01D00013B13F0FF03F3D1A242B6
S224023720EDD103B05DF8044B704700BF2F420020314200203042002038B5184B1C682378D2
S224023740012B07D0022B1ED04FF40061002003F0E7F938BD114B9A68138801339BB2DE2B35
S22402376009D8138012880D4BDB6833F81210002003F0D6F9EDE700231380094BDF211980F3
S22402378002232370EEE7054B9B6800251D804FF40061284603F0C4F92570DAE79877020057
S2240237A0B8410020154B01229A611A46936913F0010FFBD0114B9A6942F002029A61104A47
S2240237C0DA612822C3F880209A6922F001029A611A46936913F0010FFBD1084B00229A6540
S2240237E00122DA65074A5A65074B03F11C01002203F8012B8B42FBD1704700BF000400424F
S224023800020B0004DDDDF23FA03D002068BB10B4164B012083F8320015490A8942F4805299
S224023820140A83F8414083F842200622DA8783F83D000A68117883F84310517883F84410E8
S224023840917883F84510D17883F84610117983F84710527983F84820082283F84920002234
S22402386083F840205DF8044B704770476C390020AC26002038B5164B1C78032C18D0144B45
S2240238801B78012B1DD0124B1B78FBB9114B124A106851689568D468186059609D60DC6045
S2240238A01069516918615961128B1A8304240BE0032002F00BFE0128E1D1054B02221A7057
S2240238C002E00324024B1C70204638BD0324FBE714420020F43D0020D83D002017490B78BC
S2240238E0174A107A4978527A914222D00023134A917B134A92F82720914218BF00230F4AA4
S224023900517A0F4A92F82220914218BF00230B4A917A0B4A92F82320914218BF0023074A43
S224023920D07A074A92F8242090420CBF184600207047834214BF00230123D8E7F43D002056
S2240239408034020000B583B08DF8070004F028F8323880B240F2CD73984203D900238DF8B6
S224023960073003E09DF80730022B04D00D4A1278022A09D103E00B4A1278022A0FD00A4952
S2240239800A7842F001020A70064A13700DF1070141F21000F6F73CFE03B05DF804FB13464C
S2240239A0F2E700BF3542002028420020174B01221A801A46136B13F0010FFBD14FF0801399
S2240239C01B689A0C02F07002D90A01F4E0610A43C3F302431A430D4BA3F848204FF4007285
S2240239E01A801B22DA7203221A7241F606029A800022DA80072283F82E20012283F82D203A
S224023A001A46136B002BFCD1704700BF0020004368BB08B5164B012283F8322093F83B30C9
S224023A20072B0DD9124A92F8333003F00F03937601219177022B03D8527F8A4201D093B12C
S224023A4008BD0B4A0021517792F83410D17692F8352012F0800F02D105490A77EFE7044A11
S224023A607F211177EBE70020FCF752FEE8E770476C39002010B50446164A682303FB00237C
S224023A805B78032B1ED8DFE803F00214171A02F0A5FB104A682303FB04235B6D4FF6E75245
S224023AA0934205D80B4A682101FB04240233636510BDFDF719FCECE7FAF7BEFFE9E7FBF735
S224023AC07FFDE6E7034A682303FB002300225A70DFE700BF6C3900202DE9F04143685F7D99
S224023AE0012F04D0002414702046BDE8F081164688460546012328220F4900F0FFFE044625
S224023B000121284601F002F8204310F0FF0F14BF012400240121284600F064F9002818BFBA
S224023B203C46B8F1000F02D101233370DCE7284603F0AEFFF8E700BF542F002030B40E4C5A
S224023B400E4D0FCD0FC42B6823700D4B1A680D4B1A600D4B0D4A92E80300186099800C4C6D
S224023B600C4B0FCB84E80F000B4C0C4B0FCB84E80F0030BC704700BF803E0020086F0200D6
S224023B80A87A0200DC400020A4400020607A0200D43E0020B8710200E43E0020C871020004
S224023BA0F0B4134B1E78134B43F82610124B43F82600124B1F789FB1050E114B7C1E5A1C16
S224023BC052FA84F4002213F8011BA94208BF0122A342F8D122B10136054B1E70F0BC704703
S224023BE0000E074BD8550137044B1F70F3E700BF45420020DC320020CC33002046420020E6
S224023C00203C0020144B01221A601A46D369002BFCD1114B4FF480725A601A46D369002B7F
S224023C20FCD10D4B2222DA600C4A1A601A46D369002BFCD1084B10225A831A46D369002B4D
S224023C40FCD1074B002283F8212083F82020024B83229A75704700BF003400401600100094
S224023C608C3C002070B51248FDF730F8114803F0EBF900240E4EA5B22946304602F076FC6A
S224023C802946304600F0A0FD0134102CF3D10A4D00240A4E2A46E1B2304602F0E5FD013421
S224023CA00635102CF6D1064802F0FDFE70BD00BF383F0020E43C0020D4390020A43E002092
S224023CC0EC3F002008B5134B187803F06DFA012809D0114B1A6841F287339A420ED80F4BA4
S224023CE004221A7008BD02F097F800230C4A1370094A1360094B02221A70F3E7212002F0F6
S224023D008BF80023064A1370034A1360034B01221A70E7E7DD410020B8400020E141002002
S224023D20D941002010B5134B1B78012B09D0124B1B78012B05D0022B10D0104B02221A7080
S224023D400BE000230B4A13700B4A137001240C4B1C7000F099FC094B1C7010BD0023054AF2
S224023D601370054A137000F08FFC044B02221A70F3E700BF0542002008420020094200209A
S224023D80064200206BB3F0B41E4600231C4602EBC40732F834500488A54206D001339BB2D9
S224023DA01C469E42F3D8002305E00F6001339BB29E4211D801237BB9184632F830400133AA
S224023DC09BB21846B34209D2002CF6D100F10050013802EBC0000860F0BC7047002CFBD184
S224023DE0F4E77047012901D00020704770B50588134B1888A84214BF002001200123104E28
S224023E0068B936F83320AA4214BF002401240133282B01D02046F3E7AA4200D070BD0C461E
S224023E2003F10053013B064901EBC300002241F833204260012002F01BFF2046EEE700BF83
S224023E409C30002010B5114B1B78042B03D8104A12789A4205D000200E4B1870044620466B
S224023E6010BD0D4B1B78042BF5D80C4A12789A42F1D102F055FA044603F09EFC0128084B75
S224023E800CBF012200221A70E9E700BF2A4200202D4200202E4200202B4200202C4200202C
S224023EA032420020012800D0704708B503F024FD114B1880114B1B78C0F30B00104A22F8D1
S224023EC0130013B1012B0BD008BD4FF4C051062002F0F4F8094B01221A7002F009FEF3E70C
S224023EE04FF4C051072002F0E9F8044B00221A7002F06AFBE8E700BFD04100205F4200209B
S224023F005841002000207047000000000000000065732D3852C1E03F182D4454FB21F93F6A
S224023F2066732D3852C1F03FE21C0651A6602BC0CBBCE2B97F8134C0636A8D5C3FFD20C0CC
S224023F40BD87B1D97ACDEABFA995C4BC7C884440A56D0B04128A5540D7A30D320ACA4D40EA
S224023F6010C74AE1490C2E4000B58BB08DED080ACDED090A8DED061ACDED071A8DED023A01
S224023F80CDED033A8DED004ACDED014AFCF7FCFFA8B99DED003ADDED013A9DED022ADDEDC2
S224023FA0032A9DED061ADDED071A9DED080ADDED090AFCF7E9FF003018BF012000E00120BB
S224023FC00BB05DF804FBFEE7154B01221A801A46136B13F0010FFBD14FF080131B681A0994
S224023FE002F07002D90001F4E0610A43C3F382031A430B4BA3F848204FF400721A80032295
S224024000DA721A724FF4C0529A800222DA80072283F82E201A46136B002BFCD1704700BF96
S224024020001C0043F0B583B00F4616461A46089D0A9C0023019301AB01F042FA0346E0B17C
S2240240402F7000236B7073681B681B7C53B96A7801326A700133DBB2726852F82320127C16
S224024060002AF4D0228801990631A81C02F07FFC23880233099A13800123184603B0F0BDA7
S2240240800E4A38B5002313600D4A0E4C13600E4A0E4D13600E4A13600E4A13600E4A536251
S2240240A013610123936003F02EFD03F02CFDAC4200D338BD54F8043B9847F8E76C41002068
S2240240C05C3B00206C820100583B002070820100503B0020543B0020603B002000B583B090
S2240240E00122694640F2817000F04CFE9DF80030082B28BF03230C4A13700C4A062151706E
S2240241001B0403F470230A49CB614FF485739381137843F002031370936813F0020FFBD100
S22402412003B05DF804FB00BF1F3F0020002400430018004010BB0A88114B9A81CA885A8273
S2240241400A899A824A89DA820A7B1A764A7B5A768A789A73CA78DA730A791A740A7F1A710D
S224024160CA8BDA800A8C1A814A8C5A81054B0A691A604A695A608A69034B1A60704700BFCC
S2240241806C390020AC260020F43F002010B5114B1B78022B05D0012B0ED00F4B01221A7047
S2240241A010BD00230D4A13700A4A137000F06CFA094B02221A70F3E70023084A1370054ADE
S2240241C013700124064B1C7000F05EFA024B1C70E6E700BF0842002009420020054200206A
S2240241E0064200208446886818B32DE9F04305680DB300273C46BE464FF0010809E0768879
S2240242003E44B7B2042C17D0013455F824509DB190B92878604503BF15601F8040467046B1
S2240242208D6855F8246096F80490B9F1020FE6D1E8E7002070470020BDE8F08310B5114C1D
S22402424040EA01212180104B01221A600F4B4FF480625A6102230E4A19462046FBF7FEF80E
S22402426018B102F0EDFD0028FBD1084B4FF480629A61074B1A88100240EA122080B21880FF
S22402428010BD00BFBA4100203C41002000800041BC41002038B50546114C22460146002091
S2240242A0FCF7E2FE0F4B1C60B5B10F4A04F10803013DE9B203F1100505EB011553F8081C38
S2240242C0C1F38A4142F8041C1C4603CC106051600C321033AB42F1D10020FAF757F838BD27
S2240242E0EC3800205C410020983A00202DE9F0410E4619461D46804602F01CFFB54220EA93
S224024300E07087B21AD9691E404689B202F012FF002813DD84B21644013EB54210D2691C8A
S224024320404689B202F006FF002809DD80B284428CBFE019C01980B2BDE8F0810024EAE75E
S2240243400020F4E759B10132D2B2030400D452B90B040DD5002322B113F4004F0DD04FF655
S224024360FF7318467047013A4000D2B280B2ECE701324900D2B289B2EAE75B00884228BF93
S224024380401A02F1FF329BB24FEA510128BF0133D2B224BF80B29BB2DDE7FEE7124B012296
S2240243A01A601A46936813F0010FFBD10E4B4FF498521A600221596158690C4A02435A614E
S2240243C0D96300225A649A64DA641A655A659A654FF4FA521A644FF001129A621A4693688B
S2240243E0002BFCD1704700BF00600141000E404008BB10B5104B93F84A3023B10E4B93F878
S224024400403063B110BD0D49A1F153040A460839208900F0C3FB012384F84A30F2E70849D9
S224024420A1F149040A460839208900F0B7FB012384F84030E6E770476C390020BF39002049
S224024440B5390020A8B9134B41F0300183F84B101A7E83F84C20DA8A83F84D209B7B012B43
S22402446008D00C4B032283F853200A4B002283F84A207047074B1A7C83F84E2083F84F2025
S22402448083F8502083F8512083F85220082283F85320EAE76C39002008B5124B1B78042BC7
S2240244A01CD8DFE803F0030F1215180002F0BCFB0D4B1B684FF6E752934202D802330A4ABC
S2240244C0136008BDFCF7A0F9F2E7FEF787FBEFE7FAF7E6FCECE7FDF739F8E9E7014B0022E2
S2240244E01A70E5E7F9410020C04000200120704770B510EE906A10EE100A01F097F804460E
S2240245000D46304601F092F845EC114B41EC100BF9F73AFB00220A4B51EC100BFBF78AFB10
S22402452005A3D3E90023FAF719F800F059FA00EE100A70BDAFF3008000000040FB210940AC
S2240245400080664070B44125057042244470432181704422C27045230371462646713026D3
S22402456086713126C6713226067233264672342686723526C67236260673372646733826A0
S22402458086733926C673057444748174C2740375012070BC7047FEE708B5114B1B78042BEB
S2240245A019D8DFE803F0030F1205150001F05EFF0C4B1B684FF6E752934202D80233094A2E
S2240245C0136008BDFEF77AFAF2E700F03DFCEFE7FFF778FBECE7024B00221A70E8E700BF98
S2240245E0E1410020B8400020012901D000207047F0B4104C2468A66837795FB906F1080423
S2240246000DE0156022793AB108463268013A1A60F0BC70470020F8E70846F6E708342646D9
S22402462054F8085C8542ECD02579002DF6D03946EAE700BFC4400020012A21D1F0B406466F
S224024640104B1B88834214BF0020012001230D4F60B937F83340B44214BF002501250133F9
S224024660282B01D02846F3E7B44207D103F10053013B044800EBC3030B601046F0BC704755
S224024680002070479C30002008B503F083F90D4B1870022800D008BD0B4B1B684AF6C13279
S2240246A01A800A4B1B78012B13460CBF13460023074A1380782001F0B5FD064B01221A7088
S2240246C001F0E6FD11420020D8400020E5410020FA41002010420020012800D0704710B5CC
S2240246E082B00F4B1B780E2B9ABF0133DBB200230B4C2370214641F21300F5F789FF227879
S224024700084B1A70FEF7E2FF8DF807000DF1070141F21200F5F77CFF02F0DAFA02B010BD5C
S2240247203C4200202F420020012800D0704710B582B00F4B1B780E2B9ABF0133DBB2002339
S2240247400B4C2370214641F21300F5F761FF2278084B1A70FEF7BAFF8DF807000DF10701B8
S22402476041F21200F5F754FF02F0B2FA02B010BD3C4200202F420020F8B5124B1B78EBB129
S22402478007460C4616468318B3F5006FC4BF4642F6B202F0F1FC0028FBD16EB1631E751EAC
S2240247A054FA85F5C4F1884401343C44E21813F8011F1170AB42F9D170B2F8BD4FF0FF3052
S2240247C0FBE700BF3E42002008B303681A888A421FD39B788268402B0DD106234FF40D70DC
S2240247E003FB01239880002006235943535C43F002035354704783F08003012B05D8062326
S22402480041F2342003FB0123ECE70220ECE70B2070470220704708B502F0A6FCFBF772F9B7
S224024820FBF76AFDFFF7EEF9FCF74FFA00F004FCFEF7B8FF01F066FC00F080FD00F01AFA9F
S22402484000F060FD00F0E0FAFFF748FCFFF7A6FDFFF7BAFBFFF7AAF803F08AF8FCF7ACFA16
S22402486008BD7047104B1B78022B10D007D9032B11D0602B13D10D4B10221A7004E0012B38
S2240248800DD10A4B01221A70084B18787047074B02221A70F8E7054B04221A70F4E7034B8F
S2240248A000221A70F0E700BF06420020074200202DE9F0410746884600230B600E4C04F59B
S2240248C0FC7602E0B44214D018342389002BF9D02368186A0028F5D003681B68BB42F1D110
S2240248E001F0C8F90028EDD0C8F800400120BDE8F0810020FBE700BF842B0020F8B50AB3E9
S224024900174606880022144631F83450013292B21446BA420FD2B542F6D10125184604F197
S2240249200054013C01EBC402002341F83430536002F086F904E0B5420CBF01250025EDD09B
S2240249402846F8BD0025FBE708B502F0F3FF28B90F4B00221A70FFF755F908BD01F046FD61
S22402496018B102F0E7FF012806D001F0B9FB38B9074B01221A70EEE7054B00221A70EAE759
S22402498002F0D8FF0128F3D1014B00221A70E2E71442002038B5049C0F480021416081609C
S2240249A0C1600E4D2860920462F31C0101604FF0000263F3030282714BB100220546A05C8F
S2240249C0A91808720132D2B291B29942F7D302490120FEF79FFA38BDDC3100206041002019
S2240249E001F000428B1AA3F16051B1F5801F0ADBB1F17F6F09D242EAC102C10071F10041AB
S224024A0042EB507070471046704701285B4113F5001F02D842F0FF407047C90041EA50703C
S224024A20104340F4800040F080407047D0B516461F460446D0E9062339463046F8F782FFEA
S224024A4032463B46FBF7F6F8D4E90423F8F77AFF02460B4630463946FBF7ECF8D4E90223E4
S224024A60F8F770FF32463B46FBF7E4F8D4E90023F8F768FFD0BD00BF30B400F01F05430944
S224024A8003F5020303F58073DB016C081A1992F83020D2B210F0010F19BF22F0F00242EA2E
S224024AA0011122F00F021143C9B21C4484F830102B4493F8402042F0010283F8402030BC79
S224024AC070477047104B1B68B3F1FF3F14D0A8B1026AAAB112681268B2F1FF3F12D0934211
S224024AE001D0002070474368587D074B1B79984214BF00200120704700207047002070474E
S224024B000020704700207047FC3F0020F8B5012902D000273846F8BD0D4B03F54076002755
S224024B203D4609E01D605D609D60DD601D615D610F4618339E4204D05C8802889442F8D1F1
S224024B40F0E7002FE6D0012002F086F8E2E700BFAC23002008B50E4BDB78012B08D00D4BC5
S224024B60DB78012B09D00C4BDB78012B0AD008BD074B987802F064F8F1E7064B987802F086
S224024B8077F8F0E7044B987802F066F8EFE700BFD0400020D4400020CC40002070B50F4B75
S224024BA01B7813F0100F17D0C0F30B035B2B02D00125284670BD16460446F5F729FD054675
S224024BC041F25B039C42F4D13278054B1A7002F0BBFD00F07FFEECE70525EAE718420020B7
S224024BE01B4200200623434310B50F4CE2185088E05290889180508080B281420CD0E35A57
S224024C00984209D0994206D0814206D9984203D8994228BF1946084610BD9842FCD3994212
S224024C2038BF1946F7E700BF123F002070B514461D460646D0E9062329462046FAF7FAFF3A
S224024C40D6E90423F8F77EFE22462B46FAF7F2FFD6E90223F8F776FE22462B46FAF7EAFF47
S224024C60D6E90023F8F76EFE22462B46FAF7E2FF70BD00BF0F4B01221A801A46136913F063
S224024C80010FFBD10B4B4FF4C0721A8001221A621A46136913F0200FFBD1064B00225A6224
S224024CA01A46136913F0400FFBD1024B4FF480725A81704700240040F8B12DE9F04106463F
S224024CC043691BB190460F465C7974B1BDE8F0811B6842463946308898470134E4B2736952
S224024CE003EBC4035D79002DF0D11A79002AEFD01B68414638469847EFE77047002313800E
S224024D000B68DBB15B681B68187C012815D030B45B7A02331380042308684068C558287C24
S224024D20012808D01088841C687A204410800433142BF1D1012030BC7047704700207047D3
S224024D40202919D80E4B18701C2917D810B589B1531E0B484C1E52FA84F213F8014F00F8BB
S224024D60014F9342F9D10131CAB20549462002F033F810BD0122F8E7002070470020704741
S224024D80043D00200F4B1B78BBB18318B3F5006FC4BF4242D2B29AB130B44B1E551E51FABF
S224024DA085F5C1F1884101311C18645C03F8014FAB42F9D150B230BC70474FF0FF30704705
S224024DC050B270473E42002010B5054C227832B9044B13B10448AFF300800123237010BDD3
S224024DE0843D0020000000000000000008B5034B1BB103490348AFF3008008BD0000000076
S224024E00883D0020000000000D4B01221A601A46136913F0010FFBD1094B10221A600322D1
S224024E201A7350229A8333229A72064A0021116001225A721A461369002BFCD1704700BFD3
S224024E4000A00141C43F002008B50A4B1A7B0A4B1B78134303D0094B02221A7008BD084B74
S224024E60187800F033FF074B00221A60034B03221A70F3E7AC260020ED410020E141002032
S224024E80DD410020B8400020042818D838B50C46054619B1012905D0012038BDFCF7F0FA53
S224024EA02046FAE7074B1B5C012B01D10020F4E7FBF7F6FF2846FEF771F90020EDE7012019
S224024EC0704700BFAC40002008B50E4B1B78032B0AD00C4B1B78012B0FD00A4B1B78002B90
S224024EE014BF0220032008BD022001F0F5F90128EFD10220034B1870F5E7024B03221A7014
S224024F000220F0E714420020CB68BBB14B6AC3B1CB78A3B110B400234C6AE45C844206D043
S224024F200133DBB2CC789C42F6D8002302E0CB681360012318465DF8044B704700231846B0
S224024F4070470023FBE7704708B549B90C4A1A2303FB00F0135C43F001031354002008BDA5
S224024F600A4607491A2303FB00F00B18DA8055221A71043008220144588802F045FCEDE756
S224024F80BC3400200C4B0D4A9A633B225A631A46D36B13F0040FFBD1074B022283F8302074
S224024FA01A46D36B13F0020FFBD1034A136C03F00303032BFAD17047001000406000010046
S224024FC00C4B0D4ADA642F229A641A46136D13F0040FFBD1074B022283F844201A46136D98
S224024FE013F0020FFBD1034A536D03F00303032BFAD17047001000406000010058B59DF8C1
S22402500014600C4C94F920400CB1002058BD094CA080E360049B6361A1602261A6709DF894
S22402502018302370002384F82130314600F062FB0120EBE78C3C00200B4B00221A621A777A
S2240250409A60DA60094B4FF400325A601A46D369002BFCD1054B03221A73054A1A601A46D3
S224025060D369002BFCD17047B83C0020003000400E00305008B50D4A682303FB00239B7859
S224025080012B0DD05AB242B1022B0CD0074B682202FB00300023837001E001F08DF808BDBD
S2240250A0FDF77AFFFBE700F003F8F8E76C39002010B582B004460DF1070100F04BFB012865
S2240250C007D0094B682202FB04340223A37002B010BD2046FFF78CF9034B682202FB04343A
S2240250E00123A370F3E700BF6C39002010B410F07F0400D198B90B480470417083709DF8AB
S2240251000430C3709DF8083003719DF80C3043711623C380027200205DF8044B70470120CF
S224025120FAE700BF8C3F0020B97A020065510200D9730200BD7A0200A1510200E973020017
S224025140C17A0200C94E0200F9730200C57A02007538020009740200C97A0200E5350200B4
S224025160CD7A020008B50D4B1B78032B09D00B4B1B78012B0ED0094B1878B0FA80F04009F6
S22402518008BD002001F0A8F80128F0D1034B02221A70F0E7014B03221A70ECE71442002091
S2240251A008B50D4B1B78032B0AD00B4B187801280FD0094B1B78002B14BF0120022008BD5D
S2240251C0012001F089F80128EFD1034B02221A70F5E703221A70F2E71442002000B583B08E
S2240251E08DF8070002F0DCFB323880B240F2CD73984284BF00238DF807300DF1070141F210
S2240252001500F5F705FA9DF80720024B1A7003B05DF804FB3042002008B50B4B1B78012B89
S2240252200BD00A4A1368591C1160052B06D8084B1B6813B1064B00221A6008BD01F0F8FA9A
S224025240024B00221A60F2E72942002040410020444100200C490D4A30B5086813880168AF
S2240252600C8806215943A3420AD285686D5C0631ED0702D401339BB2F5E71380002030BD5B
S22402528000230120138030BD18000020BC3D002030B49DF818409DF81C502C439DF81450B8
S2240252A02C439DF8105025439DF80C4025439DF808402C43234313430B43034314BF012240
S2240252C00022089B1A7030BC70477047F8B50C4C00252E460827267504F8046C24F8025CD0
S2240252E03A462146284602F096FA2378552B18BF66800835ADB21A34402DECD10020F8BD0F
S224025300C03400200C4B01221A601A46136913F0010FFBD1084B40F214521A6002221A73AD
S224025320FA22DA7600221A775A7733229A721A461369002BFCD17047003800400C4B012298
S2240253401A601A46136913F0010FFBD1084B40F214521A6002221A73FA22DA7600221A77DC
S2240253605A7733229A721A461369002BFCD17047003C004038B505460C4602F068FA0128E6
S2240253800BD1012C05D1074B1D70074B01221A7006E0132000F046FF02E0122000F042FFB6
S2240253A038BD00BFDD410020D941002000B583B00023019301A9FFF788FF019B73B15B6871
S2240253C09B686BB11A78012A03D0002003B05DF804FB5968002001F059F8F7E70020F5E7F3
S2240253E00020F3E74FF4001C1CEB410F98BF1CEB430F11D851EA030C50EA4C0C5CEA020C2D
S2240254000AD004D282428B4180414042704790429941804140427047002070474FF4001C6F
S2240254201CEB410F98BF1CEB430F11D851EA030C50EA4C0C5CEA020C0AD004D290429941E9
S22402544080414042704782428B4180414042704700207047B9B130B40D46002319461A4667
S22402546001EB410100EBC10440F831206260A260E2602261626101339BB21946AB42EFD3E3
S224025480012030BC7047002070477047012800D0704708B5084B1970084B93F842318B424C
S2240254A000D108BD054B4BF6BE22A3F8402183F8421101F0C5FBF4E70B420020542F002078
S2240254C0012A02D0002210467047F0B4084C04F540776588854204D01834A742F9D1002248
S2240254E003E065798D42F7D11C601046F0BC7047AC230020F8B507460A4C04F50475002641
S22402550002E01834AC420AD02389002BF9D02046FDF7ACF9012804BF0136B6B2F1E73E80CE
S2240255200020F8BD842B00200378072B01D90020704710B50146074C2370012240F281702A
S224025540FFF71AF923781B0403F47023024AD361012010BD1F3F00200018004000B583B0CB
S224025560019000F0E3FF01280ED072B6074A137A013303F001031372019942F8231062B6E5
S224025580012003B05DF804FB0020FAE7983F002008B5FDF7FBFE074A00231360536013810C
S2240255A0054A01211170054A03211170044A137008BD00BF983F002041420020434200206A
S2240255C042420020B0F57A7F14D8032901D90020704700B583B04008ADF806008DF8041045
S2240255E00198FFF7BBFF012814BF0020012003B05DF804FB002070474FF4001C1CEB410F8A
S22402560098BF1CEB430F0CD850EA410C08BF52EA430C08D0904208BF99420CBF01200020BE
S2240256207047002070470120704700BFC0F3C75191B142004FEA40704FEAD2014FEA31018F
S22402564001F16051B2F17F4F38BF704701F1605118BF41F40021704710F0004100207047E2
S22402566098B1036A9BB1012907D061B91B685868013018BF0120C0B270471B68186801303D
S22402568018BF0120F7E70020F5E7002070470020704770470A4B586C20F4605020F01800C7
S2240256A04004400C9B6913F0010F08D0044A936923F001039361936913F0010FFBD170477D
S2240256C000040042084B01225A711A46D37813F0010FFBD0054B064A1A621A46536813F079
S2240256E0040FFBD1704700BF00080040001C00400701010008B5094B00229A61DA61084BE5
S22402570083221A765A6822F480225A601A46D369002BFCD100F030FB08BD00BF8C3C0020FE
S2240257200034004008B5094B5B7A6BB1074A937A3321917203F0FF0033B1054B1B681BB1C2
S224025740034B59681B68984708BD00BF00A00141C43F002088B90A4A92F84A2012B90120D3
S22402576008707047064A92F840201AB902230B700120704700220A7070470020704700BF85
S2240257806C39002008B50A4B1B78012B0AD05AB22AB1022B09D0064B00221A7001E000F0D7
S2240257A053FA08BDFEF7F2FCFBE7FEF7BBFAF8E709420020A2B130B4154600231C4631F8D7
S2240257C0342001339BB21C46AB4203D28242F6D1012003E0824214BF0020012030BC7047BF
S2240257E00020704738B50C6A94B10546204600F041FA012801D0002038BD012D06D0A07B19
S224025800A84214BF00200120C0B2F5E70120FBE70020F1E708B542EA01230122114643EA86
S2240258200040FAF751FC30B104280CBF2220312000F0F8FC08BD024B01221A707820F7E75F
S2240258401342002008B50378272B01D8002008BD0146064A13709BB2054A9383012240F263
S2240258608270FEF789FF0120F1E700BF5042002000A0014108B503210020FFF7FDF8032156
S2240258800120FFF7F9F8054B03221A70FEF7BAF90021034802F048F808BD00BF14420020BA
S2240258A0494902000A4B187008441A280CDC6AB100B583B01346009101220549462001F045
S2240258C096FA03B05DF804FB0020704700207047043D002008B5094B1A684FF6FF739A42F5
S2240258E007D0074A137843F080031370F6F7A0FD08BD024B00221A60F3E700BF1C41002067
S2240259001D42002000B583B08DF8070002F048F8323880B240F2CD73984284BF00238DF888
S22402592007300DF1070141F20600F4F771FE03B05DF804FB00B583B08DF8070002F030F8FB
S224025940323880B240F2CD73984284BF00238DF807300DF1070141F20800F4F759FE03B000
S2240259605DF804FB00B583B08DF8070002F018F8323880B240F2CD73984284BF00238DF883
S22402598007300DF1070141F20A00F4F741FE03B05DF804FB00B583B08DF8070002F000F8F7
S2240259A0323880B240F2CD73984284BF00238DF807300DF1070141F20C00F4F729FE03B0CC
S2240259C05DF804FB00B583B08DF8070001F0E8FF323880B240F2CD73984284BF00238DF84D
S2240259E007300DF1070141F20E00F4F711FE03B05DF804FB00B583B08DF8070001F0D0FFED
S224025A00323880B240F2CD73984284BF00238DF807300DF1070141F21800F4F7F9FD03B090
S224025A205DF804FB00B583B08DF8070001F0B8FF323880B240F2CD73984284BF00238DF81C
S224025A4007300DF1070141F21C00F4F7E1FD03B05DF804FB00B583B08DF8070001F0A0FFDF
S224025A60323880B240F2CD73984284BF00238DF807300DF1070141F21D00F4F7C9FD03B05B
S224025A805DF804FB00B583B08DF8070001F088FF323880B240F2CD73984284BF00238DF8EC
S224025AA007300DF1070141F21E00F4F7B1FD03B05DF804FB10B5044601F016F901280CD09D
S224025AC072B6074A537A013303F00103537252F82300206062B6012010BD0020FCE700BFD4
S224025AE0983F002007001300350090003F1C0B05030103484904060708090A0B1011121349
S224025B00141516171B1E4243444546474C4D4E4F4041704708B5084B93F82E00012283F87F
S224025B202E20064B1B682BB1C0B2044B59681B681040984708BD00BF00200043A43F002042
S224025B4008B5084B9A8992B207494A604CF2FF329A819B890B6823B10B46486889681B6863
S224025B60984708BD00240040203F002008B5084B1968084801F0D2FE00F088FD002001F06F
S224025B804BF9042001F052F900F0D6FF08BD00BFB44000203F7A020060B9094B93F84030DA
S224025BA0012B08D0064B93F84A30012B04BF044B83F84A107047024B83F84010704700BF2C
S224025BC06C39002010B5044601F02CFE012800D010BD064A682303FB0423D88800F0C4FBFA
S224025BE00128F5D12046F9F7F3FEF1E76C39002010B5044601F01DFE012800D010BD064A9A
S224025C00682303FB0423588900F0AEFB0128F5D12046FDF7ADFCF1E76C390020074B1B78DF
S224025C2033B9074B00225A71064B0022DA737047044B00225A731A73F6E700BFF5410020FE
S224025C40F43F0020AC26002010B50023054A1370054A13700124054B1C70FEF715FD044B15
S224025C601C7010BD0542002008420020064200200942002003681B7A63B18388074AD25C82
S224025C8012F0010F08D1054AD35CC3F3400383F00103DBB2184670470023FBE7C43E00205B
S224025CA030B583B00C46154601A9FEF701FE012802D0012003B030BD019B1A685268527D17
S224025CC0A242F7D19B7C2B700020F3E7012805D008B5022803D0032806D008BDFEE70121E0
S224025CE0022001F0ADFDF8E7024B01221A7000F0CFFA00BF1242002008B5084B1A68084938
S224025D0009680A441A601B68B3F5FA6F00D808BD024B00221A6001F0F5FEF8E720410020E5
S224025D202441002088B938B50446022901D1012038BD0D4600F07AFB012D01D02046F7E751
S224025D40012814BF00200120F2E70120704789B130B40D4600231A46194600EBC20440F812
S224025D603210616001339BB21A46AB42F5D3012030BC704700207047002914BF03220422A1
S224025D80054B83F8202041EA4001044B59621A46D369002BFCD170478C3C002000340040D4
S224025DA010B5074A5168074BD86A4FF6FF74DC62DB6A136813B1136880B2984710BD00BFE7
S224025DC0CC3F002000600141084B1B7813F0800F07D1064A137843F0020313709368002BE3
S224025DE0FCD1024B01225A71704700BF0020004038B5084D682404FB00F42B190022DA6558
S224025E001A6601F00FFD012814BF00200120285538BD00BF6C39002010B50446012803D0C0
S224025E20204600F0FFF910BD034B1A78034B5A70012001F0B1F9F3E7DD410020281000201C
S224025E4030B484B00546074B6C460FCB84E80F000FCC28606960AA60EB60012004B030BC3D
S224025E60704700BFA873020008B5074B1B7813F0100F00D108BD054B01221A60FFF73CFF10
S224025E80F7F706FBF6E700BF1842002024410020F0B583B00546084617461E46089C032375
S224025EA00093621C3146FCF7BFFD337803B125783D70257003B0F0BD08B5074B1B78042B35
S224025EC006D00020054B1B78002B08BF184608BD032001F069FCF5E7524200202E42002034
S224025EE008B5074B1B78052B06D00020054B1B78002B08BF184608BD042001F055FCF5E799
S224025F00524200202E42002008B5074B1B78062B06D00020054B1B78002B08BF184608BD75
S224025F20052001F041FCF5E7524200202E42002008B5074B1B78072B06D00020054B1B783A
S224025F40002B08BF184608BD062001F02DFCF5E7524200202E42002008B5074B1B78082BF0
S224025F6006D00020054B1B78002B08BF184608BD072001F019FCF5E7524200202E420020DF
S224025F8008B5074B1B78022B06D00020054B1B78002B08BF184608BD012001F005FCF5E74E
S224025FA0524200202E42002008B5074B1B78012B06D00020054B1B78002B08BF184608BDDA
S224025FC0002001F0F1FBF5E7524200202E42002008B5074B1B78032B06D00020054B1B78F4
S224025FE0002B08BF184608BD022001F0DDFBF5E7524200202E42002008B501F01BF805387C
S22402600003280BD8DFE800F002040608012008BD0320FCE70220FAE70420F8E70020F6E7B1
S22402602000B583B08DF807000DF1070141F21400F4F7EEFA9DF80720024B1A7003B05DF82A
S22402604004FB00BF3142002008B5FBF7FFFB04490448FDF7A5FD04490448FDF7A1FD08BD20
S224026060F7780200010102465F7A02000100014600B583B001238DF80730836933B10DF1A5
S2240260800700984710B101238DF807309DF8070003B05DF804FB79B110B4541E0A44013AE6
S2240260A0002304F8013F0360436008309442F8D101205DF8044B704700207047074A9388DE
S2240260C09BB2014323F4F85323F01F030B439380136B13F0040FFBD1704700BF00200043F7
S2240260E0074B9A691B699A4201D000207047044B5869DB69984214BF00200120704700BF84
S2240261008C3C0020054A0023136093600449516006211160034A93601360704710E000E0E8
S224026120BFD401002C3F002008B5064B5868064A12689A6801329A601B6813B1014B1B685C
S224026140984708BD2C3F002010E000E008B5064B5968064A4FF48030D062D26A1B6813B172
S224026160014B1B68984708BDCC3F00200060014100B1704708B5FFF725FD0020FCF74EFF3B
S2240261800020FDF777FC0020FFF732FD0020FEF771FF08BD00B1704708B5FCF739FA054B47
S2240261A05B7B052B00D108BD00210846FEF74AF9F9E700BFAC26002010B5044601F032FBD7
S2240261C00128054B4FF0680202FB04340CBF02230023A37010BD00BF6C39002010B5074BD3
S2240261E0682404FB00340023636501F01BFB012814BF00200120607010BD00BF6C39002089
S22402620008B50023054A1370054A137000F084FA00F05CFE00F072FA08BD00BFE941002011
S224026220103E0020782805D0044B1870044B01221A707047034B00221A70F5E7F1410020C2
S224026240ED410020E541002043685B7D012B01D00120704700B583B000932823024AFBF747
S22402626017FD03B05DF804FB542F002008B5064B1B78012B054914BF012300230B7041F276
S2240262800100F4F7C5F908BD164200200C420020BFF34F8F0549CA6802F4E062044B1343B5
S2240262A0CB60BFF34F8F00BFFDE700BF00ED00E00400FA0508B50378032B01D9002008BDC5
S2240262C00146044A137001224FF4F060FEF754FA0120F4E74F42002010B543001A18D200ED
S2240262E00832054C191804EBC1010B46224489785878FEF725FD10BD8034020082B0FF23B4
S224026300019358B1411E1846019B5A1E0192002BFAD101900139B1F1FF3FF5D102B07047A5
S224026320064B187810F0010007D0054B1B78012B03D9022B0CBF18460020704748420020DB
S224026340474200200B0D40F21E42D21A09DBCB0243EA505040F00040202A28BF2022D04086
S224026360704749008041704708B541F26403984205D041F26503984204D0002008BD01F079
S224026380EBF9FBE701F0F0F9F8E700B583B08DF80700FDF79BF98DF807000DF1070141F2B6
S2240263A01200F4F735F903B05DF804FB831E0830002233F8021F0A448342FAD10248A0FB9A
S2240263C00230C0F38F007047CDCCCCCC00F01F03400900F5020000F5807003EBC01090F8DD
S2240263E0403003F0FE0380F840307047064B9A691B699A4201D000207047034B5869B0FA7E
S22402640080F04009704700BF8C3C002008B5054B01229A71044B1B681BB1034B58681B68F4
S224026420984708BD00200040D43F002008B10020704708B5044B1889F7F7BCFD012814BF3E
S2240264400020012008BD00BF6C39002040B9054B1889054BDB8F98428CBF002001207047EA
S22402646000207047AC2600206C3900200023044A1370044A1360044B01221A70704700BF60
S224026480D9410020B8400020E1410020B1F90C30B1F90A20D21AC01AC0EB0020C2EB4263C4
S2240264A000EBC31090FBF2F040B2704708B5FFF7DDFE054B1B7803B108BDFCF747FBF9F7F2
S2240264C075FD00F0E1FBF7E70C42002008B5064B4200111803EBC1010B464A68897858782E
S2240264E0FFF7E0F908BD00BF8034020008B500F0A1FD431E032B07D8DFE803F0030204030D
S224026500032008BD0220FCE70020FAE7012803D0054B00221A707047034B1B78002BFAD100
S224026520014B01221A7070473442002072B6064B187A01305B7A00F00100834214BF002054
S224026540012062B6704700BF983F0020054B1A68013205490B689A42FCD8034B1A68014BFC
S2240265601A607047544100205041002050B103681B888B4208D306238268594300200123D3
S224026580535470470B2070470220704710B504460078FEF77AFF207800F0D5FD2078FFF7FE
S2240265A078F82078FFF7B5FA10BD10B504460078FEF76BFF207800F0C6FD2078FFF769F83A
S2240265C02078FFF7A6FA10BD054A138823F002031B041B0C1380136B002BFCD1704700BFF2
S2240265E00020004310B429B1044B43F8301003EBC0035A605DF8044B704700BF943E002052
S224026600044B054A5A621A46536813F0080FFBD1704700BF001C004006010600044B054A9B
S2240266209A621A46536813F0100FFBD1704700BF001C004006013000044B054ADA621A460B
S224026640536813F0200FFBD1704700BF001C004001010400044B054A1A631A46536813F069
S224026660400FFBD1704700BF001C004008010C00044B054A5A631A46536813F0800FFBD13D
S224026680704700BF001C004006010300054A138823F002031B041B0C1380136913F0020FAC
S2240266A0FBD1704700240040054BDB7A13F0200F03BF034B83F8310001200020704700BFA2
S2240266C000380040054BDB7A13F0100F03BF034B83F8300001200020704700BF003C004086
S2240266E008B5054A92F82E3043F0010382F82E30F9F738FB08BD00BF001C004308B50023AA
S224026700034A1370034A1360FDF746FF08BD00BFE1410020B840002008B50023034A13701B
S224026720034A1360FDF7B8FE08BD00BFF9410020C0400020044B187000F07F00012818BFA4
S2240267400220024B187070470642002008420020012803D0043818BF01207047024B1B78EB
S2240267600B700020704700BF0B42002030B40546044C0FCC28606960AA60EB60012030BC87
S224026780704700BFE43E002008B50378012B01D9002008BD0146012240F28370FDF7ECFFA9
S2240267A00120F6E708B50023034A1370034A1370FFF760F808BD00BFF8410020F4410020D4
S2240267C008B50448F7F7DEF9C043C00F024B187008BD00BF808000411542002010B5054CEB
S2240267E000232370214641F25C00FCF73DFA207810BD00BF3342002010B5054C0023237037
S224026800214641F26200FCF72FFA207810BD00BF3342002010B5054C00232370214641F23A
S2240268205E00FCF721FA207810BD00BF3342002000B583B00022044B1978032000F060FAD5
S224026840002003B05DF804FB4442002008B5022000F07AFC10B94FF4907008BD022000F03C
S22402686073FCC0F34F00F8E710B548B142B10C2301245943836858185C544260002010BD86
S2240268800B2010BD08B528B1C2691AB1117811B15368984708BD526800889047FAE710B504
S2240268A00446002000F050FC000A2070002000F04BFC6070012010BD10B50446012000F05C
S2240268C043FC000A2070012000F03EFC6070012010BD10B50446022000F036FC000A2070E2
S2240268E0022000F031FC6070012010BD10B50446032000F029FC000A2070032000F024FC80
S2240269006070012010BD10B50446042000F01CFC000A2070042000F017FC6070012010BDF8
S22402692010B50446052000F00FFC000A2070052000F00AFC6070012010BD10B50446062079
S22402694000F002FC000A2070062000F0FDFB6070012010BD10B50446072000F0F5FB000ABC
S2240269602070072000F0F0FB6070012010BD10B43AB1431E8A1811F8014B03F8014F91429B
S224026980F9D15DF8044B704700B583B08DF807000DF107014FF48150F3F73AFE03B05DF813
S2240269A004FB00B583B08DF807000DF1070141F22200F3F72DFE03B05DF804FB00B583B0FE
S2240269C08DF807000DF1070141F21700F3F720FE03B05DF804FB00B583B08DF807000DF153
S2240269E0070141F21A00F3F713FE03B05DF804FB08B5002000F0A8FB08B9A92008BD00205A
S224026A0000F0A2FBC0F34F00F8E708B5012000F09BFB08B9CE2008BD012000F095FBC0F3D5
S224026A204F00F8E708B5032000F08EFB08B9862008BD032000F088FBC0F34F00F8E708B568
S224026A40042000F081FB08B9C72008BD042000F07BFBC0F34F00F8E708B5052000F074FB86
S224026A6008B9822008BD052000F06EFBC0F34F00F8E708B5062000F067FB08B9BA2008BDF3
S224026A80062000F061FBC0F34F00F8E708B5072000F05AFB08B9972008BD072000F054FBD0
S224026AA0C0F34F00F8E748B103683BB10020187058809880D8801881588170470B207047A3
S224026AC0044A138843F002031380136B002BFCD1704700BF001C0043044A138843F002038F
S224026AE01380136B002BFCD1704700BF00200043044A137D43F002031375136B13F4006F1B
S224026B00FBD1704700200043044B41F606429A611A46136913F0020FFBD0704700100040FD
S224026B20C1F30B01034B19821A46936813F0040FFBD1704700240043044A138843F0020329
S224026B401380136913F0020FFBD1704700240040044A136843F002031360136913F0020F20
S224026B60FBD1704700380040044A136843F002031360136913F0020FFBD17047003C004010
S224026B80044A136843F002031360136913F0020FFBD1704700A00141044A136843F0020384
S224026BA01360936813F0020FFBD1704700600141044A537803F0F00300F00F000343537020
S224026BC0704700BF00200040044B9B6813F0100F02D1024BA5221A73704700BF002000401A
S224026BE008B5044A682303FB002300229A70FEF741FA08BD6C39002008B5044A682303FB5D
S224026C00002300225A70FCF735FF08BD6C39002008B5682303FB00F3024A0021D154FCF7EF
S224026C20FDF908BD6C390020034B00221A60034B01221A70704700BFC0400020F9410020F8
S224026C40044B9B78834200D07047024B0022DA70FAE700BFD0400020044B9B78834200D0FF
S224026C607047024B0022DA70FAE700BFCC400020044B9B78834200D07047024B0022DA706A
S224026C80FAE700BFD440002008B5044900230B7041F20400F3F7BCFC08BD00BF0F420020A3
S224026CA008B500F0A7FE034A137843F04003137008BD00BF2542002008B5044A137843F0D6
S224026CC002031370F5F7B4FB08BD00BF1C42002008B5044A137843F004031370F5F7A8FBA6
S224026CE008BD00BF1C42002072B6044B187A5B7A984214BF0020012062B67047983F0020F9
S224026D0010B582B0144640F08000FDF797FA04B12080002002B010BD08B5002000F014FA17
S224026D2010B940F2531008BD002000F00DFAFAE708B5012000F008FA10B94FF4CE7008BD52
S224026D40012000F001FAFAE708B5022000F0FCF910B94FF4107008BD022000F0F5F9FAE749
S224026D6008B5032000F0F0F910B940F20D1008BD032000F0E9F9FAE708B5042000F0E4F9F2
S224026D8010B94FF4C77008BD042000F0DDF9FAE708B5052000F0D8F910B940F2051008BDA1
S224026DA0052000F0D1F9FAE708B5062000F0CCF910B94FF4BA7008BD062000F0C5F9FAE7C4
S224026DC008B5072000F0C0F910B940F22F1008BD072000F0B9F9FAE700B585B000230293D4
S224026DE001930093FEF70AF905B05DF804FB10B584B0002402940194069C0094FEF7FEF8FB
S224026E0004B010BD034BDB79DBB243FA00F000F00100704700240043034B98611A4613695C
S224026E2013F0080FFBD1704700240040034B18621A46136913F0200FFBD17047002400408D
S224026E40034B187E80F00200C0F34000704700BF00300040034B00229A601A6842F00102DB
S224026E601A60704710E000E008B5034B01221A70042000F0B9FC08BD2D20002000EB40002C
S224026E80024B03EB40035888704700BFD439002000EB4000024B03EB80031889704700BFEA
S224026EA04C360020034B9B6800EB400013F82000704700BFA43E00200128034B1B680CBF45
S224026EC018899888704700BFEC3F002008B5034B00221A70FEF756FC08BD00BF094200203C
S224026EE00B6A2BB1DB7B184214BF0120002070470020704710B504460089FEF757FAA073F7
S224026F00E0730023A38110BD30313233343536373839303030303030300000BF0346034A51
S224026F201068186092889A8001207047A440002008B50178437843EA01210020FEF704F8F9
S224026F40012008BD08B50178437843EA01210120FDF7FAFF012008BD08B50178437843EAF2
S224026F6001210220FDF7F0FF012008BD08B50178437843EA01210320FDF7E6FF012008BDDB
S224026F8008B50178437843EA01210420FDF7DCFF012008BD08B50178437843EA012105206C
S224026FA0FDF7D2FF012008BD08B50178437843EA01210620FDF7C8FF012008BD08B50178E2
S224026FC0437843EA01210720FDF7BEFF012008BD08B5034B19783120FEF7F4FA012008BD2C
S224026FE04F42002010B5044600F0D4FC30EA04030CBF0120002010BD08B5FFF7D3FB024B42
S2240270000022DA7308BD00BF6C3E002008B518B10846FFF7BAF908BD1046FFF7B6F9FAE78E
S2240270200128034B1B680CBF012202221A70704798770200034B1B78012B06BF014B187A3B
S22402704000207047743F002018B1034B1860002070470B20704700BF1C00002010B582B045
S224027060BDF810400094F9F7BBF802B010BD08B5112201464FF4A060FDF784FE012008BD78
S22402708008B5112201464FF4A060FDF775FB012008BD08B50422014640F21750FDF772FEFE
S2240270A0012008BD08B50422014640F21750FDF763FB012008BD08B51022014640F21B5015
S2240270C0FDF75AFB012008BD08B51022014640F21B50FDF757FE012008BD08B50122014651
S2240270E040F28370FDF74EFE012008BD08B550EA010314BF01200020FFF708FA08BD003042
S22402710018BF01201070003118BF01211970704708B50020FFF776FE00B908BDFCF70CFBC7
S224027120FBE7034628B122B1024403F8011B9342FBD170470C2303FB01014B6858880B8966
S224027140C01A00B270477047024A1A2303FB0020C0887047BC34002010B1024B1860596039
S224027160704700BFAC3F0020024B40F204521A80704700BF00400041024BD86AC0F380005F
S224027180704700BF0040004108B5FDF785F9FEF7F9FAFDF701FA08BD024A13881844108053
S2240271A0704700BFEA410020024B1878003018BF0120704711420020313233343536373834
S2240271C039303A3B3C3D3E3F48573035202020202020202020202020024B1B8803800120BC
S2240271E0704700BFF43A0020024B5B8803800120704700BFF43A0020024B9B880380012018
S224027200704700BFF43A0020024BDB8803800120704700BFF43A0020024B1B8903800120F6
S224027220704700BFF43A0020024B5B8903800120704700BFF43A0020024B9B8903800120D5
S224027240704700BFF43A0020024BDB8903800120704700BFF43A0020024B1B8A03800120B4
S224027260704700BFF43A0020024B5B8A03800120704700BFF43A0020024B9B8A0380012093
S224027280704700BFF43A0020024BDB8A03800120704700BFF43A0020024B1B8B0380012072
S2240272A0704700BFF43A0020024BDB8B03800120704700BFF43A0020024B1B8C0380012050
S2240272C0704700BFF43A0020024B5B8C03800120704700BFF43A0020024B9B8C038001202F
S2240272E0704700BFF43A0020024BDB8C03800120704700BFF43A0020024B1B8D038001200E
S224027300704700BFF43A0020024B5B8D03800120704700BFF43A0020024B9B8D03800120EC
S224027320704700BFF43A0020024BDB8D03800120704700BFF43A0020024B1B8E03800120CB
S224027340704700BFF43A0020024B5B8E03800120704700BFF43A0020024B9B8E03800120AA
S224027360704700BFF43A0020024BDB8E03800120704700BFF43A0020024B9B8F0380012009
S224027380704700BFF43A0020024BDB8F03800120704700BFF43A0020024BB3F84030038018
S2240273A001207047F43A002053573033303320202020202020202020024B1B78037001207C
S2240273C0704700BF1F3F0020024B1B7803700120704700BF4F420020024B03221A700020FB
S2240273E0704700BF14420020024B03221A700020704700BF14420020024B03221A70002076
S224027400704700BF14420020024B03221A700020704700BF14420020024B187800F00F0095
S224027420704700BF18420020024B187800F00100704700BF1F420020024B1878C0F34000C0
S224027440704700BF1F420020024B1878C0F38000704700BF1F420020024B1878C0F3C000D7
S224027460704700BF1F420020024B1878C0F30010704700BF1F420020024B1878C0F3401097
S224027480704700BF1F420020024B1878C0F38010704700BF1F420020024B187800F0010009
S2240274A0704700BF20420020024B1878C0F34000704700BF20420020024B1878C0F38000F5
S2240274C0704700BF20420020024B1878C0F3C000704700BF20420020024B1878C0F30010C5
S2240274E0704700BF20420020024B1878C0F34010704700BF20420020024B1878C0F3801095
S224027500704700BF20420020024B187800F00100704700BF21420020024B1878C0F34000D5
S224027520704700BF21420020024B1878C0F38000704700BF21420020024B1878C0F3C000F2
S224027540704700BF21420020024B1878C0F30010704700BF21420020024B1878C0F34010B2
S224027560704700BF21420020024B1878C0F38010704700BF21420020024B187800F0010024
S224027580704700BF22420020024B1878C0F34000704700BF22420020024B1878C0F3800010
S2240275A0704700BF22420020024B1878C0F3C000704700BF22420020024B1878C0F30010E0
S2240275C0704700BF22420020024B1878C0F34010704700BF22420020024B1878C0F38010B0
S2240275E0704700BF22420020024B187800F00100704700BF23420020024B1878C0F34000F1
S224027600704700BF23420020024B1878C0F38000704700BF23420020024B1878C0F3C0000D
S224027620704700BF23420020024B1878C0F30010704700BF23420020024B1878C0F34010CD
S224027640704700BF23420020024B1878C0F38010704700BF23420020024B187800F001003F
S224027660704700BF24420020024B1878C0F34000704700BF24420020024B1878C0F380002B
S224027680704700BF24420020024B1878C0F3C000704700BF24420020024B1878C0F30010FB
S2240276A0704700BF24420020024B1878C0F34010704700BF24420020024B1878C0F38010CB
S2240276C0704700BF24420020024B187800F00100704700BF25420020024B1878C0F340000C
S2240276E0704700BF25420020024B1878C0F38000704700BF25420020024B1878C0F3C00029
S224027700704700BF25420020024B1878C0F30010704700BF25420020024B1878C0F34010E8
S224027720704700BF25420020024B1878C0F38010704700BF25420020024B1878C0F3801008
S224027740704700BF25420020024A137803F0BF031370704725420020024B187800F001000A
S224027760704700BF27420020024B1878C0F34000704700BF27420020024A137823F0010346
S2240277801370704727420020024A137823F0020313707047274200203F420020404200202A
S2240277A0B6410020942D002007289ABF014B185C0020704794400020024B187800F00100E9
S2240277C0704700BF48420020024A136801331360704700BF50410020024B1A6B002AFCD124
S2240277E0704700BF001C0043024A138818441080704700BFD241002002440346934200D1FC
S224027800704703F8011BF9E708B500F5E06080B2FCF7B2FF08BD08B500F5E06080B2FDF70E
S224027820B1FA08BD08B5FFF7F7FDB0FA80F0400908BD08B5FFF7F0FDB0FA80F0400908BD3A
S22402784008B508B9012008BDFDF71EFBFBE70138C0B202288CBF00200120704710B50446A7
S22402786000F098F82070012010BD08B500210846FDF76AFB012008BD08B500210120FDF7A5
S22402788063FB012008BD08B500210220FDF75CFB012008BD08B500210320FDF755FB012006
S2240278A008BD08B500210420FDF74EFB012008BD08B500210520FDF747FB012008BD08B5FB
S2240278C000210620FDF740FB012008BD08B500210720FDF739FB012008BD08B5B0FA80F05B
S2240278E04009FCF721FF08BD08B5003018BF0120FCF7F2FE08BD7047014BB3F8400070472E
S22402790000200043014B186059607047A43F002003695A400A405A4002617047014B1860FE
S22402792099607047203F0020014B5862996270478C3C0020014B93F8210070478C3C0020DA
S224027940014B5868704700BF10E000E0014B1860596070472C3F0020014B186059607047DB
S224027960C43F0020014B01221A707047913E002008B5FEF7FBF8FCF775F908BD014B1B68A4
S22402798018787047EC3F0020014B1878704700BFF5410020014B1878704700BF06420020EC
S2240279A0014B1888704700BF6C3E0020014B5888704700BF6C3E0020014B587C704700BF92
S2240279C06C3E002003030000000000000000000000238B700B704B700370704708B508701D
S2240279E01078FEF7EBFF08BD014B1878704700BF41420020014B1868704700BF943A00202F
S224027A00014B194408797047943A002008B50078FEF706FB08BD08B50078FEF701FB08BDB5
S224027A2008B50131FFF7D4FF08BD08B50078FEF7C5FF08BD08B50020FFF732F908BD08B58F
S224027A40FFF712FA08BD7F2303700020704708B5FBF720FC08BD08B5FAF7C2F808BD7047F8
S224027A6032343037323200BF08B5FEF7B4FF08BD08B5F9F78DFE08BD08B500F00CF808BD72
S224027A8008B500F008F808BD83F00043F5F75ABF00B55DF804FB0023037070471070197053
S224027AA0704700207047704720240722302070471020704708207047002070470020704792
S224027AC0002070470020704700207047002070470870704708707047087070470870704787
S224027AE008707047087070470870704708707047087070470870704708707047002070475F
S20C027B00002070477047704731
S8040180007A
